:020000000C945E
:10000200E8040C9400000C9400000C9400000C9482
:1000120000000C9400000C9400000C94CF4B0C9444
:1000220000000C9400000C9455080C9400000C94F1
:1000320000000C9400000C9400000C9400000C943E
:10004200D0070C9400000C9466480C9400000C94A9
:10005200A0480C9400000C9400000C9400000C9436
:1000620000000C9400000C9400000C9400000C940E
:1000720000000C9400000C94364A0C9400000C947E
:10008200764B0C9400000C9400000000010002006A
:10009200040008001000200040008000000100025F
:1000A200000400080010002000400080000102044B
:1000B2000810204080005F4944000000000000005A
:1000C20000000000E50B8000100000005F526F741A
:1000D20061746500000000000000E50B8100010072
:1000E20000005F54617374656E58000000000000E8
:1000F200E50B0100040003005F54617374656E59DF
:10010200000000000000E60B0100060005005F444D
:10011200656661756C744B6579000000E80B01003F
:10012200800000002A436F64653000000000000078
:100132000000EF0B02000F2700002A436F646531B5
:100142000000000000000000E90B02000F27000081
:100152002A436F6465320000000000000000EB0BD0
:1001620002000F27D0122A4D61784D6F64756C0022
:1001720000000000ED0B0100100000002A5469731A
:1001820063684500000000000000EE0B0000010063
:1001920000005F4D795465726D4E720000000000E0
:1001A200F10B0100080001005F4D61737465725428
:1001B20065726D730000F20B0300080001005F45D9
:1001C2004D6F64650000000000000000F30B0300A7
:1001D200040000005F4543726564577472000000BA
:1001E2000000090C01007F003F005F5273304D6F29
:1001F2006465000000000000080C0100030000001C
:100202005F5634756E643500000000000000F40B88
:100212000000010000005F50756C736554696D65E4
:1002220000000000070C010064001E005F41736BB8
:1002320043726564697400000000F50B0000010060
:1002420000005F53656E64446562697400000000DB
:10025200F60B0000010000005F4372656469744D93
:100262006F6465000000060C0100010000005F439E
:1002720072656469744D617374657200F70B0000F6
:10028200010000002A5461626C655374617274004B
:100292000000F80B02000F2700002A5461626C650F
:1002A200456E640000000000FA0B02000F27E7030E
:1002B2002A4A6F6231000000000000000000FC0BBF
:1002C2000300080001002A4A6F62320000000000A9
:1002D20000000000FD0B0300080000002A4A6F62C4
:1002E20033000000000000000000FE0B03000800C5
:1002F20000002A4A6F623400000000000000000083
:10030200FF0B0300080000002A4A6F62350000005C
:10031200000000000000000C0300080000002A4A50
:100322006F6236000000000000000000010C0300B4
:10033200080000002A4A6F62370000000000000037
:100342000000020C0300080000005F4572726F7229
:1003520031000000000000000A0C04000A002E0018
:100362005F4572726F723200000000000000140CD0
:1003720004000A002E005F4572726F7233000000A3
:10038200000000001E0C04000A002E005F4572727D
:100392006F723400000000000000280C04000A0004
:1003A2002E005F4572726F7235000000000000007F
:1003B200320C04000A002E000000000000000000C1
:1003C2000000000000000000FF0000000000546177
:1003D200737465722020000000024C69745A202058
:1003E2002020000004044C65697454202020000081
:1003F200080750756C732020202000000C055075F2
:100402006C732030202000008C06546173742030FD
:1004120020200000800973657269656C6C20000001
:10042200100B73657269656C20320000500C5461C8
:1004320073742032202000004008546173742070CD
:1004420061720000140A3F3F3F3F3F3F20200000FF
:1004520000024D756C74696D617845636F20567347
:1004620020312E30300049443D0050726F642B0021
:10047200696E696369616C697A6172200000507209
:100482006F64756B74200000537061727465202074
:100492000000706F7274696F6E696572656E00003C
:1004A2002E666F6C67650000506F7274696F6E65BF
:1004B2006E207369636865726E000500C1110000E9
:1004C2000300D90B00000300C1110300170E030043
:1004D200D90B00000500E00800000A00C1110A0063
:1004E200170E0A00D90B0A00C1110A00170E2800C4
:1004F200D90B00003000436865662D4D656E7500AE
:10050200000031004B206C697374656E00000000BE
:1005120032004B206C6F65736368656E00003300B8
:100522004B20647275636B656E00000034005420CA
:100532006C697374656E00000000350054206C6FA6
:1005420065736368656E00003600542064727563DB
:100552006B656E000000460053797374656D000090
:10056200000000004100506F7274696F6E0000005D
:10057200000043004B72656469746500000000006E
:1005820044004B7265642E436C7200000000490007
:10059200496E666F000000000000000000000000CD
:1005A2000000000000000000000030005379737466
:1005B200656D000000000000370054657374000090
:1005C2000000000000003900506172616D657465C1
:1005D20072000000380050726F64756B7465000021
:1005E200000042004B656C6C6E65720000000000FA
:1005F200450056656E74696C650000000000470096
:100602002D3E4F73636172574C0000006300436FCD
:100612006C6F727300000000000000000000000018
:1006220000000000000000004572726F722000009E
:100632000000000000004F0C000010000000506598
:1006420067656C200000000000000000520C0000F2
:1006520001000000496D70756C73200000000000FD
:100662000000500C00001000000054696D654F75C9
:100672007420000000000000510C00001400000073
:100682002E202C30414243314445463247484933BB
:100692004A4B4C344D4E4F355051523653545537C8
:1006A20056575838595A2F393769000D0D34690D8C
:1006B2000D0D31691A0D0D3876000D0D35760D0DC3
:1006C2000D32761A0D0D3983000D0D36830D0D0D89
:1006D20033831A0D0D2D90000D0D21900D0D0D304F
:1006E200901A0D0D2B9D000D0D2F9D0D0D0D3D9D95
:1006F2001A0D0D0073656375726F203F00546F749D
:10070200616C0043616C6962726174696F6E006C46
:10071200656674200072696768742000746F7020C7
:1007220000626F74746F6D2000546573743A200018
:1007320056616E6E652000322E43686F69780054F0
:10074200657374006B65696E20454570726F6D004C
:100752004B230054230042450043450042410044DC
:100762005300564300494C00434300434200235088
:100772002241534349492D492F4F222C22312E30F9
:1007820030222C323030382D30312D30313B0023A5
:10079200482245636F222C22312E3030222C3230F7
:1007A20030382D30312D30313B0023532245636FD9
:1007B200222C22312E3030222C323030382D303162
:1007C2002D30313B00504F002C00504632333B500D
:1007D20055002564002B302B303B0000533F0000B6
:1007E20066616C7363686572205469736368200084
:1007F200546973636820766F6E204B2000466568EB
:100802006C6572200056656E74696C20616B746948
:10081200760054696D656F757400435349204E72BA
:100822002000436F6465200058313939313030007F
:100832004D4200505300504C5520203A00436F6403
:1008420065203A005469736368203A004B656C6C0A
:100852006E657220004D31004F31005350004350FD
:100862000044590062757379004D5000206765732A
:1008720070657272740025640000253032580025BC
:10088200303458002533642E253032640025356417
:1008920000256400253264002533640044440000CE
:1008A2004B2300425300422100424600542300548D
:1008B2004F004952004D5A00564300494B004252E4
:1008C20000435300426600004162726563686E75C0
:1008D2006E67004B656C6C6E65722000546F7461BC
:1008E2006C004D6F64756C2000202000433F006E49
:1008F20065696E006A6120200073656300496D704E
:1009020000504C553A20005370617274653A2000D1
:100912005072313A20005072323A200053656974A5
:1009220065203A20005479703A20003A20563A2045
:1009320020302B2030003A003A20544F3A20005306
:10094200703A004B2066726569204A6F62204A6FD6
:1009520062466C616773004B200066726569200015
:100962004A6F622020005620202045727220506774
:100972006C20496D7020544F005620004B656C6C02
:100982006E65723A004D49004D42004D43004D5094
:10099200004D4C0074657374202E2E004F4E0000E3
:1009A2002564002530325800253130640025642E3C
:1009B200253264004F4E000001002D4E414E0000D2
:1009C2004B00620CAA060100B10FBA090000F894AC
:1009D200EE27ECBBF1E0F5BFE5BFE0936C00F8E178
:1009E200F1BDE1BD8DE0A2E0BB27ED938A95E9F769
:1009F20080E090E1A0E0B1E0ED930197E9F7E2EC4D
:100A0200F9E085919591009761F0A591B5910590D6
:100A12001590BF01F00105900D920197E1F7FB01DE
:100A2200F0CFEFEFEDBFE0E1EEBFC0E0D3E00C941A
:100A3200B20908950895E0916300E07111F0E1E0D8
:100A42000895E0E00895E881E03011F01A9801C0BD
:100A52001A9A85C484C483C463C0089508950E9409
:100A62001D6410E0143130F40E94EC54A0E0A08325
:100A72001F5FF8CF30913A0810E0E091E60B1E17A5
:100A820008F500E0E091E50B0E17D0F4A02FE5E1A8
:100A9200EA9FF0010E94F254A12FEDE0EA9FF001DB
:100AA200E15D0E94F254E4E1F0E0FA93EA930E94DD
:100AB200F654E32FE0580E94FB543F5F0F5FE2CFF2
:100AC2001F5FDBCF10E0A5E01A9FF001EE59F34F54
:100AD200E081E03019F11A9FF001BF01DF01ED5909
:100AE200F34FE0810E94F254FD01EC59F34FE08193
:100AF2000E94F254F001EB59F34FE0810E94F2544C
:100B0200FB01EA59F34FE0810E94F254FB01EE59D6
:100B1200F34FE0810E94FB541F5FD5CF0E942464F3
:100B2200249608950E94045508950E9404550E9437
:100B32001055329606C00AC009C00E940838E6EF76
:100B4200F6E0FA93EA930E942833089588DF089525
:100B52000E9408380E941F550E94C33223960895AE
:100B62001A930A930E94245510E0E1E0E0935C0C92
:100B7200E0935D0C0E942E550E94F2540E94883729
:100B8200E0913D08E03041F4EFEFF6E00E94345589
:100B92000E9438550E940733A0913D08A130D8F039
:100BA200E0913D08E150EA930E9443550E944A5564
:100BB2000E944E55E12FEF5F0E94F2540E94883747
:100BC200E0913D08E1500E9453550E9457550E9402
:100BD2005C550E9407331E5FE0913D08EF5FE09392
:100BE2003D081C3020F4A0913D08AB3008F001C054
:100BF200C1CF79C31A930E94083810E0163050F51D
:100C02000E942E55EE0F0E94F2540E948837E1E0B6
:100C1200EA93E12FAA81EA0FEA930E946417E12F77
:100C2200A981EA0F0E9461550E942E55EE0FEF5FD7
:100C32000E94F2540E9488370E9469550E946E55A4
:100C4200E8E7EA930E9456370E9472550E947B554C
:100C52001F5FD4CF188122960895E881E064E7B936
:100C6200369A349BFECF349AE4B1F5B178C3E88169
:100C7200F981AA81BB81AE17BF0724F4EA1BFB0BE3
:100C82000C94610BA881B981EA81FB81EA1BFB0B01
:100C92000C94610B2A970E941B64EFE0E0936100C1
:100CA200E4EFE093620088EC90E00197F1F7ECE06A
:100CB200E093610088EC90E00197F1F70E947F5584
:100CC200E0935305F0935405E0915F05F0916005C0
:100CD200E0935105F0935205E0E0EA93BEDFE09322
:100CE2005F05F0936005EFE0E0936100E2EFE093CF
:100CF200620080EA8A95F1F7E3E0E093610088E51B
:100D020092E00197F1F70E948455E0934F05F0932A
:100D12005005E0915D05F0915E05E0934D05F0937D
:100D22004E05E2E0EA9399DFE0935D05F0935E05FC
:100D32000E948455A0914F05B0915005EA0FFB1F08
:100D4200A0915D05B0915E050E9489558F010E94B8
:100D52007F55A0915305B0915405EA0FFB1FA09156
:100D62005F05B09160050E9489559F01E0914F0592
:100D7200F09150050E949055FF93EF930E94845585
:100D82000E949055AF91BF91EA0FFB1FFF93EF9323
:100D9200E0915D05F0915E050E949055AF91BF9183
:100DA200EA0FFB1FE0935905F0935A05E0915305B2
:100DB200F09154050E949655FF93EF930E947F5540
:100DC2000E949655AF91BF91EA0FFB1FFF93EF93DD
:100DD200E0915F05F09160050E949655AF91BF9139
:100DE200EA0FFB1FE0935B05F0935C05A0915905A8
:100DF200B0915A05E8E2F0E00E9465610E2EA091E2
:100E02005B05B0915C05E8E2F0E00E946561E029D3
:100E120019F00E942137B1C0009355051093560571
:100E220020935705309358050E949C55D29724F47D
:100E3200A9E4B5E00E94A1550E94A755989724F411
:100E42000E94AC5598970CF010C00E949C551A97BE
:100E520021F4E1E0F0E00E94B1550E949C55989780
:100E620021F4E2E0F0E00E94B1550E94A755999763
:100E720024F00E94AC5599970CF47FC0A3E4B5E02E
:100E82000E94A155E0E3F5E760E070E00E94B655EC
:100E920040E050E0E0E0EE87EF87A0E0B0E00E94A3
:100EA2006B620E94A7550E94BF550E94C655AA8533
:100EB200BB858C859D85EAEAF0E060E070E00E94E7
:100EC20098617F936F93FF93EF93A2E0B0E00E944B
:100ED2006B620F01A0E0B0E00E94CB55AF91BF91D1
:100EE2008F919F910E9455610E94E8610E94C655B0
:100EF200A4E0B0E00E946B620E94AC550E94BF5514
:100F02000E94D255AE81BF8188859985EFE5F0E0D8
:100F120060E070E00E9498617F936F93FF93EF937C
:100F2200A6E0B0E00E946B620F01A4E0B0E00E9474
:100F3200CB55AF91BF918F919F910E9455610E94B5
:100F4200E8610E94D255EA85FB85E0933705F0936C
:100F52003805EE81FF81E0933905F0933A05E0917F
:100F62003705F0913805FA93EA93E0913905F0914B
:100F72003A05FA93EA930E949D360E942264609693
:100F82000895E6B3EF70A0E1EA9FF001AE2FE0B161
:100F9200E07FE295EF70EA2BAFEFEA2708950E9417
:100FA200D7550E941D64E3E6E2BFE1E0E71521F4B4
:100FB2000E9424642496A6C0E1E07E2E78940E94CA
:100FC200603668DE0E94571F0E94F248A4E8BBE028
:100FD2000E94A155A0913D05B0913E050E94116469
:100FE20014F40E94E55500E010E0A091A705B0912D
:100FF200A8058091A9059091AA050E94156424F480
:10100200A0913508A23009F00BC0A7EAB5E00E9412
:1010120041623197604070400E944B6201E010E0F3
:10102200A0913508A13011F401E010E0A09135083B
:10103200A33011F401E010E0A0913508A23021F4B0
:10104200E091840BE07449F0A0913508A23021F0C0
:10105200E091840BE07109F002C01A9801C01A9A5B
:10106200E091840BE87011F4C79A01C0C798A0916F
:101072003008B0913108EFEFF0E0EA27FB27EBBB35
:10108200AD98AD9AE0913008F09131080E944A6122
:10109200AFEFB0E0EA27FB27EBBBAE98AE9A77241E
:1010A2000E94246424962EC00E94D7551A930A9354
:1010B200E6E0E4BDE0E0EABBEFEFEBBBAF98000097
:1010C20000000000E9B3FE2FE0E08F01AF9AE0914B
:1010D2006500EB7FE0936500000000000000E9B3CB
:1010E200F0E00E0F1F1FE0916500E460E0936500E1
:1010F200EFEFEABB1A930A930E94C61E0E94D151D7
:1011020009911991E991EFBFF991E991B991A991E9
:101112009991899179916991F9901990099018950D
:101122000E94D1500E9498510E94EB3C0E94D01C18
:1011320008951A93A8950E947E34E13011F00C9420
:10114200F308E091AE05E1501E2FA091AD05A1304C
:1011520029F40E94EC54E081E03009F412C00E94AC
:10116200EC54E081E093C305ACE01A9FF001E75F25
:10117200FC4FBF01E081E260DB01EC931A930E9415
:10118200ED55A091AD05A23011F0A430D9F40E9422
:10119200EC54E081E093C405E5E1E093C305ACE0E3
:1011A2001A9FF001DF01E050FD4FE081E03031F0A5
:1011B200FD01E75FFC4FE081E27009F403C01A937E
:1011C2000E94F155A091AD05A33019F41A930E9423
:1011D2007725A091AD05A53029F4E091AE05EA93FB
:1011E2000E94C225E091F103E07889F0E091F103D9
:1011F200EF77E093F1030E942A38E091F103E07166
:1012020031F0E091F103E270EA930E94D33788DF74
:101212001EC21A930A930E94F555EF731E2F01E026
:101222000E9402561A930E947D160E940E560E9438
:101232004A550E94F6540E941356E12F0E945355BC
:101242000E9419560E9420564EC00E940256E88102
:101252000E9461550E94F6540E9413560E94235622
:101262000E9420567CC01A930A930E9428560E941C
:1012720028560E942D56EBE2F7E00E94345511E009
:101282001131A0F4E12F0E943156A0913008B091A3
:101292003108EA23FB23309739F0E2E3F7E00E94BA
:1012A20034551A930E9416331F5FEACF0E942856C4
:1012B2000E94135610E000E0023010F4103108F0E2
:1012C20012C00E943B56E03061F0E12F0E94F254BE
:1012D2000E940D330E943B560E94F2540E940D332D
:1012E2000F5F1F5FE9CF0991199108951A9310E0DA
:1012F200103190F41A930E947D16E4E6F0E0E09338
:10130200C70BF093C80BE12FEF5FE093C10B1A9369
:101312000E94A7161F5FECCF9AC1A881A13021F0CD
:10132200A0913A08A030D9F0A881A13011F40E940E
:101332000256E0913A08E03069F4A091E50BE091A1
:10134200E60BEA9FF001E0933A08E9E3F7E00E9436
:10135200345503C0E0E0E0933A080E94300521963C
:101362000895EFEFEBBBEABBEFE8E8BBE0E8E7BBD1
:10137200E0EEE5BBEFEFE4BBE5B3EF79E5BBE5B348
:10138200E066E5BBE0E0E2BBE1BBE3B9ECE9E2B970
:10139200E0EFE0936200E0E0E0936100E7E0E093D9
:1013A2006500E0936400E0E0E0BFE7E0E3BFE4E66D
:1013B200E2BFE0E0E1BFEFBDEEBDEDBDECBDE7BDDC
:1013C200E6BDEBBDEABDE9BDE8BDE0937900E0937F
:1013D2007800E3E0E5BDE6E0E4BDE0E0E3BDE093F4
:1013E2008B00EAE0E0938A00E0E0E0938900E0937A
:1013F2008800E0938100E0938000E2E1E0938700BF
:10140200E4E3E0938600E0E0E0938500E09384006B
:10141200E0938300E0938200E0936A00EABFE9BFB1
:10142200E1E4E7BFE0E0E0937D00EBB9E8EDEAB983
:10143200E6E0E0939500E0E0E0939000E7E6E9B9AA
:10144200E0E0E0939B00E8EDE0939A00E6E0E093B1
:101452009D00E0E0E0939800E3E3E0939900E0E888
:10146200E8B9E0E0E0BDE0E4E7B9E7E8E6B9E0B515
:10147200EF7EE0BDE0E0EDB9E0E2E0937000E0E095
:10148200E0937200E4E4E0937400EFE1E1BDEFE089
:10149200E1BD0E944156E0E0E0933508E8EEF3E05A
:1014A20060E070E00E94B655E0E0F0E0E0933D05B8
:1014B200F0933E05E1E0EA930E949E32E0E0E09381
:1014C200AB05E093AC0578940E9444560E947137B4
:1014D2000E9428560E9428560E948837E1E4F7E0CD
:1014E2000E9434550E944A560E944E370E94A5150A
:1014F20078940E9472320E94A815E030B1F40E94E2
:1015020050560E9455560E948837E6E4F7E00E9442
:101512003455A8950E945A56E2E3F0E00E946856BC
:101522000E945A560E944456F4CF0E944219E0305B
:1015320061F00E9428560E9428560E948837E2E7EE
:10154200F4E00E9434550E944A56E8E0E093E50B2D
:10155200E4E0E093E60B0E9428560E9428560E947F
:101562008837E4E5F4E00E9434550E9428560E9430
:101572001356E8E6F4E00E9434550E946C56EA9352
:101582000E941633EAE0F0E0FA93EA930E941356BF
:10159200ECE6F4E00E943455E0E2F3E00E94685683
:1015A200E0E0EA930E949E320E94C207E07469F072
:1015B200E2E0E093AB0B0E94C207E07211F0E3E0BD
:1015C20001C0E2E0E093AC0B0EC00E94C207E071E2
:1015D20019F0E1E0E093AB0B0E94C207E07219F050
:1015E200E1E0E093AC0BA9E0B0E0E2E00E947B62B4
:1015F200E1E0E093F60B9DDD0E940D2EFCCFFFCFC4
:10160200E0915D0BEA930E94174DE0915E0BEA9325
:101612000E94174D0895F4DF0E941F550E947156D3
:101622000E9471560E94785620C41A930E94634CFD
:101632001E2F103021F0E12FE150E0935B0BE0DF31
:10164200E0915B0BEF5F0E94F2540E947856199171
:1016520008950E941D6431E00E947E56A03320F05E
:101662000E947E56A43308F028C030E00E948456BF
:10167200E270E6951E2F0E948456E1700E2FA09113
:10168200750B1A1729F4E1E0EA27E093750B31E0B4
:10169200A091760B0A1729F0E1E0EA27E093760B96
:1016A20031E0E091760BEE0FE05DA091750BEA0F51
:1016B200EA930E94174D0E948A56E32F0E942464E7
:1016C200249608951A9310E00E948D56E9F10E9423
:1016D200321AE2E5F7E00E949356E091440C0E9430
:1016E200F2540E947856E5E5F7E00E9493560E9474
:1016F20097560E9478560E949E56A031E7E2BE0796
:101702004CF4E8E5F7E00E949356E091450CF09125
:10171200460C13C0EBE5F7E00E949356E9810E9464
:10172200A3560E949E56EA0FFB1F0E94A956E09103
:10173200450CF091460CE051F742FA93EA930E946D
:10174200464D0E94AE5611E00E94B256E12F8CC364
:1017520024970E941B640E94B2560E942A4CE130D8
:1017620010F40C94F80EE0915D0BEB3441F4E0912F
:101772005E0BE33219F40E94634C1E2F35C3E4352D
:10178200B9F4E0915E0BE33221F40E94634CEE83E4
:10179200FF83E0915E0BEF3451F40E94634C1E2FE5
:1017A2001A93EF81F885FA93EA930E94E2151CC31B
:1017B200E23411F00C941E0DE0915E0BE13259F40B
:1017C200AA85AF3F31F40E94B9560E9428560E9462
:1017D200F53E0E94F01AE0915E0BE134E1F40E94C2
:1017E200634C1E2F113071F4A0915108A13019F4ED
:1017F2000E948D5609F402C00E943D1AE0E0E09377
:10180200A70B09C0E1E0E093A70B0E94403FE093E1
:10181200A90BF093AA0BE0915E0BE534A9F4EEE577
:10182200F7E00E9493560E941A1AF3973CF00E9426
:10183200634C0E94A9560E94BC5601C0E0E3EA93A1
:101842000E94174D0E94AE56E0915E0BE634E1F421
:101852000E94C85619F40E94634CAF01E885F985CD
:101862000E94D4560E2F003420F0A091F70BA13025
:1018720059F40E94D8560E940F1BAA85AF3F21F44B
:101882000E94D8560E94F53EE0915E0BE23511F0BF
:101892000C94DF0C0E94C85619F40E94634CAF01ED
:1018A20030E0A091F70BA03021F40E946C56E13099
:1018B20009F023C00E94952FE030F1F00E94E0561B
:1018C200EC52F84F0E94E6560E94E056E852F84F5A
:1018D2000E94EB560E94E056EA52F84F10830E9493
:1018E200E056E952F84F40830E94E056ED52F84F1D
:1018F200A1E0A0830E94F1565FC00E948F2FE230C8
:1019020010F40C94DD0C0E94F9560E94E61B3E2F47
:101912003F3F29F00E94FF56A417B5070CF417C0E9
:101922000E940457E41BF50B0E9409570E940457BA
:10193200309739F4E0E0E093490C3A930E94721C2C
:1019420003C03A930E946B1C689420F803C0E0E045
:10195200E887E9870E940E57E150F84FDF010E94A5
:101962001457EA57F44FE081EC930E940E57EF5F51
:10197200F74F0E94E6560E940E57EB5FF74F0E9408
:10198200EB560E940E57ED5FF74F10830E940E57E1
:10199200E050F84FA5E00E941757E885F985309787
:1019A20059F00E94F956FA010E942C610E942057B8
:1019B2000E94D8560E94981A689422F8E0915E0B11
:1019C200E335D1F50E94634CE887F9870E942457DA
:1019D200DF01E050F84FE081E23081F4FD01EB5F7E
:1019E200F74F008011800E946C560E942A57EA1716
:1019F200FB0721F4A0915108A23009F01BC00E94FC
:101A02002457EF5FF74FDF010E943762DF01E8855D
:101A1200F985EA17FB0771F40E942457DF01E95F99
:101A2200F74FE081EA93FD01E150F84FE081EA933C
:101A32000E94F923689422F8D7C1E43411F00C947F
:101A4200890DE0915E0BE33559F4E1E6F7E00E947F
:101A520093560E94E8480E942D57E1E0E093540912
:101A6200E0915E0BE03511F00C94880D0E94315725
:101A7200E03011F40C94880D20E00E947E56A032D2
:101A820040F00E947E56A23221F00E947E56AB3375
:101A920009F43DC0E22FE03061F40E947E56A33289
:101AA20011F421E005C00E948456EA930E94C348C3
:101AB2002BC0E13049F40E947E56A43211F422E098
:101AC20001C020E010E020C0E23011F0E330E1F488
:101AD2000E948456EA930E94183FEF3FA1F0E12F43
:101AE200E295E07FEF930E948456EA930E94183FAA
:101AF200AF91EA0F1E2F2F5F243021F41A930E9418
:101B0200C34820E001C020E00E948A56B6CF6CC1D3
:101B1200E63511F00C94590EE0915E0BE334C9F5F1
:101B22000E94355730E0353070F40E943B57E08117
:101B32001E1739F40E944057EC930E943B57A0E0D5
:101B4200A0833F5FF0CF30E0303118F50E94465756
:101B5200E0811E17E1F4E4E6F7E00E949356E12FDC
:101B6200EF770E94F2540E944B570E9453570E94F3
:101B72001956FA93EA930E944B570E9457570E94B4
:101B820019560E945B570E944657A0E0A0833F5F10
:101B9200DBCFE0915E0BE33511F00C94320EE0E006
:101BA200EA930E94FA18E0E0E093AD0BE9ECFBE067
:101BB2000E945E57E093C20BE0E0E093C50BEBECB2
:101BC200FBE00E945E57E093C30BE0E0E093C60B9C
:101BD2000E94634CE093C10B0E94645711F00C9475
:101BE200320E0E94634CE093C40B0E946457C9F505
:101BF2000E94634C1E2F103019F0E1E0E093BE0BFF
:101C02000E94645771F50E94634CE093C70BF093F6
:101C1200C80B0E94645729F50E94634CDF01E4E679
:101C2200F0E00E94BE61E093CD0B0E946457C9F4BC
:101C32000E943557E0E0EA931A930E94F9230E2F8F
:101C4200013079F0E4E6F7E00E949356E12FE05884
:101C52000E94F2540E946A57E02F0E94F2540E949E
:101C62007856E0915E0BE53511F50E9435570E94DA
:101C72006457E9F40E94634C0E2F30E03530B8F41B
:101C82000E943B57E0811E1781F4013031F40E941B
:101C92007057EC91E068D001EC93003031F40E946F
:101CA2007057EC91EF77D001EC933F5FE7CF9CC088
:101CB200E934E9F4E0915E0BEC34C1F4E7E6F7E0D5
:101CC2000E949356E091DF05F091E005F070FA93DF
:101CD200EA930E94544D0E947857E091E005F0701B
:101CE200FA93EA930E94544D0E94AE567DC0E334AB
:101CF20011F00C94F50EE0915E0BE534B9F4EEE5CB
:101D0200F7E00E9493560E941A1AF3974CF00E9431
:101D1200634CE05FF84D0E94A9560E94BC5601C078
:101D2200E0E3EA930E94174D0E94AE56E0915E0BEB
:101D3200E634B1F441E050E00E94634C0E2F0E9461
:101D4200645719F40E94634CAF011A930E947C57A6
:101D5200E05FF84DFA93EA935A934A930E940F1B5D
:101D6200E0915E0BE33519F50E94634C3197E887E9
:101D7200F9870E94645719F40E94634CAF01E88509
:101D8200EA93FA01E058FF4FEA930E94F923E03008
:101D920041F4EAE6F7E00E9493565A934A930E946E
:101DA2007856E885EA93EFEFEA930E94F923E091EF
:101DB2005E0BE134C9F4EDE6F7E00E9493560E940F
:101DC200634C3197E887F987E885EA930E947D168C
:101DD2000E942D23E03011F0E1E301C0E0E3EA9339
:101DE2000E94174D0E94AE560E94E24BB6CC0E9452
:101DF20022642B960895A091730BA03529F4E091EB
:101E0200740BEA930E94A716A091730BA33529F4D1
:101E1200E091740BEA930E94E516A091730BAB3428
:101E220029F4E091740BEA930E942517A091730B99
:101E3200A63529F4E091740BEA930E944E17A09103
:101E4200730BA43511F40E94CC150E947F5708959C
:101E52001A9310E0103440F40E948557EE52F94F65
:101E6200A981A0831F5FF6CF1881229608950E9450
:101E72001B640E942A4CE13010F40C945912E09138
:101E8200730BA0915D0BEA1709F0B5DFE0915D0BD2
:101E9200E33211F5E0915E0BEC3449F4E0E0EA93B1
:101EA200D7DFEFEFE093770BE4E0E0933408E091C3
:101EB2005E0BE43581F4E0E0EA93CADFA091770B90
:101EC200AF3F31F0E091770BA9E0B0E00E947B6276
:101ED200E7E0E093340804C0EB3411F00C94B60F41
:101EE200E0915E0BE13221F4EBE4EA93B1DF3CC016
:101EF200E53211F480DF38C0E332D9F40E9488570A
:101F020031F00E9493570E94F1160E9499570E9445
:101F12009E57E081EB3461F4E0E0E093540CE093EF
:101F2200550C0E949E57A0E0A083EBE4E093730B54
:101F32001BC0E134C9F4EBE4E093730BA0915B0B9B
:101F4200A03890F40E94634C9F012093540C0E948D
:101F5200A45751F00E94634C9F010E94A45721F0A4
:101F62000E94634CE093550CA0C2E33511F00C942F
:101F7200FA0FE0915E0BE13221F4E3E5EA9368DFC8
:101F820037C0E332D9F40E94885731F00E94935748
:101F92000E94B8160E9499570E949E57E081E3352D
:101FA20061F4E0915B0BEA930E94DF180E949E5756
:101FB200A0E0A083E3E5E093730B1AC0EE34C1F412
:101FC200E3E5E093730BA0915B0BAA3088F4EAE09F
:101FD200EA930E94EF4C10E01A3050F40E94AA5784
:101FE2000E948557E15AF44FE081EC931F5FF4CFD2
:101FF2005CC2E63511F00C945010E0915E0BE132B8
:1020020021F4E6E5EA9324DF49C0E332D9F40E94E1
:10201200885731F00E9493570E9431170E949957B6
:102022000E949E57E081E63561F4E0915B0BEA93F2
:102032000E945B170E949E57A0E0A083E6E5E09312
:10204200730B2CC0E63531F40E94634C9F01209340
:10205200500C24C0E53471F40E94634C9F0120931C
:102062004F0C0E94A45729F00E94634C9F012093B9
:10207200520C14C0E43591F440E050E00E94634CED
:102082009F01022E032A11F042E050E00E94A45761
:1020920019F00E94634CAF014093510C06C2E43523
:1020A20011F00C941511E0915E0BE33231F40E94B1
:1020B200634C3197E0935B0BB6C0E03511F00C94A2
:1020C200141110E00E947E56A03250F00E947E56FB
:1020D200AD3331F00E947E56AB3311F01E3008F062
:1020E2000DC00E948557E15AF44F0F010E94845699
:1020F200D001EC931F5F0E948A56E4CF0E9485575D
:102102000E94B057EDE30E94B55711F00C941411E0
:10211200E4E5E093730B10E00E94BA5770960E94B8
:102122005062EF3FA0E0FA0711F40C9414110E94E0
:10213200C0570E94BA57FA93EA930E94F751E030CF
:1021420011F00C9412110E94BA570E94C55729F43B
:102152000E94634CE093770B64C0E138A0E0FA0779
:1021620039F40E94634CA8E0B0E00E947B6259C03F
:10217200309721F0E130A0E0FA0769F40E94BA57E3
:102182003E960E945062FF93EF930E94634CAF9180
:10219200BF91EC9346C0E230A0E0FA0771F40E94CE
:1021A200BA573E960E945062FF93EF930E94634C8F
:1021B200AF91BF91ED93FC9334C0E330A0E0FA07F6
:1021C20069F40E94BA573E960E945062FF93EF93C1
:1021D2000E94444CAF91BF91EC9323C0E430A0E045
:1021E200FA07F9F40E94BA577296E491EA930E94B0
:1021F200EF4C0E94BA573E960E9450624F0100E097
:102202000E94BA570E94CC5764F40E947C57E15A4C
:10221200F44FE081D401EC93F40131964F010F5F4A
:10222200EFCF1F5F79CF41C1E03511F00C94561208
:10223200E0915E0BE332D1F40E94885731F00E94A4
:1022420093570E947D160E9499570E949E57E081E3
:10225200E03561F4E0915B0BEA930E94FA180E9468
:102262009E57A0E0A083E0E5E093730BE0915E0B44
:10227200E33221F0A0915B0BA03408F016C1E0E537
:10228200E093730BE0915E0BE13221F4E0E5EA9317
:10229200DFDD0BC1E134C1F40E94634C1E2F00E06C
:1022A2000B3088F40E94D4573B96E491E11749F42D
:1022B2000E94D4573A96E491A091BE0BEA2BE09388
:1022C200BE0B0F5FEDCFF1C0E63559F5E0E0E093CC
:1022D2005C0B0E94DA57EA0FFB1FFF93EF930E94F9
:1022E200634CAF91BF91EC93EBE2EA930E94F54B02
:1022F200E03059F00E94E057EA0FFB1FFF93EF9383
:102302000E94634CAF91BF91EC930E94E657A0915B
:102312005C0BA33018F40E94A45709F401C0D9CF72
:10232200C4C0ED34D1F4E0E0E0935C0B0E94EC57C2
:10233200EA0FFB1FFF93EF930E94634CAF91BF9193
:10234200EC930E94E657A0915C0BA33018F40E9414
:10235200A45709F401C0EACFA8C0E434C9F5E0E00B
:10236200E0935C0B0E94634C9F01E2E0EA930E94BF
:10237200024CAF01E3E70E94B55769F40E94F2579D
:10238200BF01D901E4E6F0E00E949361E40FF51F7A
:10239200DB01ED93FC93E9E40E94B55769F40E94D6
:1023A200F257208331830E94FC57EA0FFB1F0F0173
:1023B2000E94FC570E9402580E94E657A0915C0BB3
:1023C200A33018F40E94A45709F401C0CBCF6DC00A
:1023D200EE3491F4EAE0EA930E94EF4C10E01A30F6
:1023E20050F40E9409580E948557E15AF44FE08147
:1023F200EC931F5FF4CF59C0E33449F40E94315784
:102402000E94634CE093B90BF093BA0B4EC0E335D4
:1024120089F40E94634C9F0100240216030624F4EF
:102422002B30E0E03E070CF004C0F9013197E09355
:10243200BB0B3BC0E53529F40E94634CE093BD0B16
:1024420034C0EF3491F40E94634C1E2FECE2EA9305
:102452000E94F54BE12FE295E07FEF930E94634CDF
:10246200AF91EA0FE093BC0B20C0E035F1F4E0E05D
:10247200E0935C0BA0EDBBE00E940F580E94135842
:10248200FF93EF93E2E0EA930E94AE4CAF91BF91CB
:10249200ED93FC930E94E657A0915C0BA23018F4D6
:1024A2000E94A45709F401C0E5CF0E94E24BE1CC9F
:1024B200E0E0E0935E0A0E942264269608950E945C
:1024C2001D640E942A4CE13010F40C94D614E09161
:1024D2005D0BE332A9F4E0915E0BE03519F4E0E71D
:1024E200F7E009C0E83419F4E1E9F7E004C0E335A4
:1024F20031F4ECEAF7E0FA93EA930E94284D52C2D3
:10250200E43511F00C941913E0915E0BE43229F4D6
:10251200E3E2F0E00E9418588AC0E33211F485D851
:1025220086C0E03511F00C9418136AD8A0915B0BA9
:10253200A33210F00C9418130E941C580E94935658
:10254200EDE3EA930E94174D0E941C580E94C55762
:1025520039F40E946C560E94F2540E94464D67C0A4
:10256200E138A0E0FA0739F40E9424580E94F2549C
:102572000E94464D5CC0309721F0E130A0E0FA079E
:1025820059F40E941C583E960E945062E0810E94BB
:10259200F2540E94464D4BC0E230A0E0FA0759F4D3
:1025A2000E941C583E960E945062DF010E942958E8
:1025B2000E94464D3CC0E330A0E0FA0751F40E946D
:1025C2001C583E960E945062E081EA930E94634D3D
:1025D2002EC0E430A0E0FA0751F50E941C583E9646
:1025E2000E9450624F0110E00E941C5872960E9495
:1025F20050620E942E58AE17BF0774F40E9485578E
:10260200E15AF44F0F01D401EC91D001EC93F401A3
:1026120031964F011F5FE8CF0E941C5872960E94AC
:1026220050620E94B0570E94C0570E94C64DBAC164
:10263200E33569F5E0915B0BEA930E94B816E091ED
:102642005E0BE43229F4EAE0F0E00E9418581EC062
:10265200E33219F40E94160B19C0EE34B9F40E9449
:10266200010B10E01A3060F40E948557E15AF44FD2
:102672000F010E94AA57EC91D001EC931F5FF2CF99
:102682000E9431580E94C64D0E94AE568BC1E6355B
:1026920011F00C948913E0915B0BEA930E943117BD
:1026A200E0915E0BE43229F4E0E1F0E00E94185878
:1026B2002EC0E33219F40E94160B29C0E53459F4F6
:1026C2000E94010BE0914F0C0E94F2540E946A5743
:1026D200E091520C19C0E63529F40E94010BE091F9
:1026E200500C12C0E43599F40E94010BE091510C98
:1026F200E03011F0E1E301C0E0E3EA930E94174DFC
:102702000E943558E091510CF0E00E945B574AC19B
:10271200E03511F00C94A914E0915B0BEA930E944E
:102722007D16E0915E0BE43229F4E0E4F0E00E94D1
:1027320018580DC1E33219F40E94160B08C1E13496
:1027420011F00C94E7130E94010B12E0A091BE0B52
:10275200ECEDEA233E2F00E00B3068F40E94D457E0
:102762003A96E491E31729F40E94D4573B961491C8
:1027720002C00F5FF1CFE12F0E94F2540E947856FF
:10278200E091BC0BE03099F0E7ECF7E00E94935641
:102792000E9439580E94464DEAECF7E00E94935697
:1027A200E091BC0BEF700E94F2540E943E58E091FF
:1027B200BD0BE03051F0ECECF7E00E949356E09153
:1027C200BD0B0E94F2540E943E58C1C0E43469F528
:1027D2000E944358A0915C0BA33030F5E0915C0B52
:1027E200E03011F00E9435580E94FC57AE0FBF1F17
:1027F200EC91E17051F4A7ECBBE00E940F580E94EB
:1028020019560E944958E3E709C0A7ECBBE00E94B1
:102812000F580E9419560E944D58E9E4EA930E940B
:10282200174D0E94E657D6CF8EC0ED34B1F40E9408
:102832004358A0915C0BA33078F4E0915C0BE0303C
:1028420011F00E9435580E94EC570E9451580E9484
:10285200464D0E94E657EDCF76C0E63501F50E945F
:102862004358A0915C0BA330C8F4E0915C0BE030BC
:1028720011F00E9435580E94DA570E9451580E9466
:10288200464DEBE2EA930E94174D0E94E0570E94E8
:1028920051580E94464D0E94E657E3CF54C0EE3491
:1028A200B1F40E94010B10E01A3060F40E948557C7
:1028B200E15AF44F0F010E940958EC91D001EC93B8
:1028C2001F5FF2CF0E9431580E94C64D3CC0E334D4
:1028D20099F40E94010B0E94C057E4EDF7E0FA93CD
:1028E200EA930E9455580E945A580E945F580E94CB
:1028F200C0570E94C64D27C0E03579F40E94010BF3
:102902000E9423560E9449580E943558E091D20BEA
:10291200F091D30B0E94495816C0E33531F40E945E
:10292200010BE091BB0BEF5F0BC0EF3481F40E940F
:10293200010B0E9439580E946A57E091BC0BEF705C
:10294200F0E00E944D58EBE3EA930E94174D2AC033
:10295200EB3441F5E0915B0BEA9342D2E0915E0BDE
:10296200E43229F4E0E8F0E00E9418581BC0E33298
:1029720019F40E94160B16C0E134A1F40E94010B57
:102982000E9464580E946A570E9464580E946A57C3
:10299200E091550C0E94F2540E94464DE7EDF7E09B
:1029A2000E9493560E94E24B8CCD0E94B2560C9428
:1029B200BA180E946958EBE5F9E00E9471580E942A
:1029C200B2560E947658E181E43471F40E9476583E
:1029D20002800E946C56E05DE01529F00E94765854
:1029E200E281EA3209F401C057C00E947B580E947A
:1029F2007658E1810E947E580E947658E2810E94B8
:102A02007E580E9484581C910E94765833960E94E8
:102A12007158E12FE23131F40E948958E6E0EC93DB
:102A220026DA3AC0E13131F40E948958E2E1EC93AE
:102A320046DD32C0EF30A9F40E948958EEE0EC93F3
:102A42000E942A0BE13039F4A0915008A03019F00D
:102A52000E948D5609F402C00E943D1A0E948F58AE
:102A62001BC0EE30C9F40E948958EFE0EC930E943B
:102A72002A0BE13089F4A0915008A03019F00E948D
:102A82008D5609F402C00E943D1AE0E0E09350081E
:102A9200EFEFEA930E94A90B55C01A930E94965831
:102AA200E7E5F8E00E947158EAE7EA930E94174DC1
:102AB2000E94845811971C91E12FE23131F4E6E033
:102AC200EA930E94174DD3D937C0E13131F4E2E1E4
:102AD200EA930E94174DF3DC2FC0EF3099F40E9465
:102AE2009B580E942A0BE13039F4A0915008A03083
:102AF20019F00E948D5609F402C00E943D1A0E94EC
:102B02008F581AC0EE30C1F4EFE0EA930E94174DDD
:102B12000E942A0BE13081F4A0915008A03019F0F4
:102B22000E948D5609F402C00E943D1AE0E0E09333
:102B32005008EA930E94A90BA0915308AA3211F0FF
:102B42000E94A14E199108950E947F5708951A93E9
:102B52000A9310E0E4E6F0E00E946856A8950E940D
:102B62004238E03021F4E0EA0E949F5809F002C0A6
:102B720001E001C000E00E9452381F5F003011F4F2
:102B8200153008F001C0E6CFE02F099119910895A0
:102B92000E94A4586CC40E94A4580E94B15808957F
:102BA200A881B9810E94116424F4A83EE3E0BE0723
:102BB2000CF005C00E94B7580E94B23860C3E0E032
:102BC2005EC3A881B9810E94116424F4A83EE3E0A7
:102BD200BE070CF005C0EA81E03011F4EFEFEA83A2
:102BE2000E94B758ED81EA930E94E13861C10E94C8
:102BF2001D6420E030E0283EE3E03E077CF4A89527
:102C02003A932A93CDDF1E2F1F3F29F0EFEFEA936D
:102C12003A932A93D6DF2F5F3F4FEDCFAAC21A9382
:102C22000A93E0E0F0E0E093B20CF093B30CAA81D7
:102C3200A03458F40E94C058E55FFB4F8F010E94F8
:102C4200C758E2EBFCE00E94D058E091B20CF09140
:102C5200B30C2CC11A931FEF1F5F1A93E0DFA981F7
:102C6200BA81EA17FB0711F0113408F001C0F4CF62
:102C7200E12F18811DC1EA81EF5FEA83EA93CFDF7A
:102C8200A881B981EA17FB0719F0AA81A13408F0DB
:102C920001C0F1CFEA810CC10E941B6410E0103424
:102CA20030F50E942E58E8E2F0E00E949361E05075
:102CB200FC4FAF01E0EAEA93FA017096FA93EA93C5
:102CC2000E94B238EC713E2FE0EAEA93FA01739661
:102CD200FA93EA930E94B2380E2F303119F4EE8142
:102CE200E01709F002C0E12F03C01F5FD8CFEFEF5A
:102CF2000E942264279608950E941D64E091AD0B04
:102D0200AC81EA1711F1A03488F40E94D458A8E2E9
:102D1200B0E00E949361E050FC4F8F010E94D758AF
:102D22000E940239EC81E093AD0B0FC0EFEFE0930C
:102D3200AD0B30E03A3030F40E94E058EDE2EC9313
:102D42003F5FF8CF0E94E058EC933AC01A930A937F
:102D52000E94C058E050FC4F8F01AA81A03430F489
:102D62000E94D758E0E2EA930E9467399FC00E940E
:102D72001D64E091D60BAC81EA1711F10E94D45880
:102D82000E94E658AC81AA3040F40E94EE580E949C
:102D9200D058EC81E093D60B13C0EFEFE093D60B43
:102DA20030E03A3048F4A7EDBBE0EE27A30FBE1F98
:102DB200EDE2EC933F5FF5CFA7EDBBE00E94F9583F
:102DC2000E942464259608950E94FE580E94E658A7
:102DD200AA81AA3020F40E94EE580E94B15866C01F
:102DE2001A930A93E091530CAA81EA1761F10E94A7
:102DF20003590E94065908F50E94C758E4E5FCE011
:102E02000E94D058EA81E093530CE0E0E093E105A0
:102E1200A091550CA13020F0A091550CA83008F0DB
:102E22000BC0ACEFBBE0E091550C0E940E59AE0F07
:102E3200BF1FEC91E093E10506C0EFEFE093530C66
:102E4200E0E0E093540C32C00E94FE580E94065902
:102E520030F40E94C758E4E5FCE00E94B15826C055
:102E62001A930A93E0914E0CAA81EA17A9F00E94E4
:102E720003590E94115940F40E9419590E94D058D6
:102E8200EA81E0934E0C08C0EFEFE0934E0CE0E0D5
:102E9200E0934F0C0E94245909C00E94FE580E94E0
:102EA200115920F40E9419590E94B15819810881C0
:102EB20023960895E0E0E0934F0CE881EF5F0E94D3
:102EC20024592196089524970E941B640E942C592C
:102ED200E0E0E0933D0CAB85A13010F0A63008F0A5
:102EE20007C0EB850E940E590E943F590E94455926
:102EF200EB85E03069F5E0E0EE83EF83E887E98770
:102F020040E050E020E030E02530E0E03E07B4F45D
:102F1200F9010E943F590E9445590E9469554E0F7E
:102F22005F1F0E947255AE81BF81888599850E947C
:102F320027610E94D2552F5F3F4FE6CF40933E0C50
:102F420050933F0CEE81FF81688579850E94595923
:102F52000E9422642C9608951A930A93AB81A130A1
:102F620010F0A63008F01DC0EB810E940E590E949D
:102F720045610E944161DF010E940359AE0FBF1FEC
:102F8200E8E0F0E00E949361E050FA4E8F01E0EA3F
:102F9200EA930E9462591A930A93ECE3FCE00E94BE
:102FA200B15819810881E7C01A930A93EA81EA931A
:102FB200A3DE0E941A1D0E2F10E01017D8F5EB8128
:102FC200EA93EB81EA937FDFAEE3BCE00E94A15576
:102FD200A091400CB091410C8091420C9091430C15
:102FE2000E9423560E9455610E9427610E945959EE
:102FF200EB81EA93EB81EA93AFDFEB81E093440C40
:103002000E945558309761F40E946C560E94A35654
:10301200EF5EF84DDF010E940359EA0FFB1F02C069
:103022000E945558E093450CF093460C0E94675954
:103032001F5FC3CF198108819EC00E941D6400E0FA
:103042000B3058F4E02F0E9453550E9457550E94AE
:1030520071590E9446620F5FF3CF0E9471590E941C
:10306200765900E0003418F50A9346DEE0913E08F6
:10307200EA930A9328DFE091BB0B0E9453550E940A
:103082004561EA0FFB1F0F01E091BB0B0E945355F4
:103092000E9457550E943B62DF01CB010E9472558C
:1030A2000E942761D0010E9446620F5FDBCFA09190
:1030B2003508A33011F00C94A21830E0303110F032
:1030C2000C94A2180E947F590E948259C1F500E017
:1030D2000A30A8F5E32FE05DEA93EEEDF7E00E94F7
:1030E2008759E02FE05D0E948E5939F513E0E02FF9
:1030F2000E9453550E944561EA0FFB1FFF93EF9315
:10310200E02F0E9453550E9457550E943B627F93C5
:103112006F93FF93EF93EDB7FEB7FA93EA931F9382
:103122000E941A4E1F91AF91BF918F919F910E9461
:103132002761AF91BF910E9446620F5FC9CF3F5F87
:10314200BDCF00E00A30A8F4E02F0E9453550E9440
:1031520057550E943B62A0914508B0914608809164
:103162004708909148080E9427610E9476590F5F94
:10317200E9CF0E942464249608951A93A895A98100
:10318200A63058F40E942C5910E0103430F4E98132
:10319200EA931A93E1DE1F5FF8CF70C01A9311E031
:1031A200163020F41A93E9DF1F5FFACF84C3E1E0FF
:1031B200E093540CE093550C0C948A1D1A93A89535
:1031C20010E0183050F40E94AA570E948557E65723
:1031D200FB4FE491EC931F5FF4CF0E949359E0936D
:1031E200DF0B0E949A59E093E00BE0E0E093E10BE1
:1031F20045C01A93A89510E0183050F40E9409585F
:103202000E948557E058FB4FE491EC931F5FF4CF87
:103212000E949359E093B60B0E949A59E093B70B20
:10322200E0E0E093B80BE0E0F0E0E093D00BF09345
:10323200D10BE2EDFBE00E945E57E093BB0BE0EBAB
:10324200E093BC0BE0E0E093BD0B10E01330B0F470
:103252000E94A1590E94A459AEEBBBE00E94AD5955
:10326200A1ECBBE00E94AD59A4ECBBE00E94AD59B9
:10327200ADECBBE00E94AD591F5FE8CF18812296EA
:1032820008950E941B6400E083DCA091E20BB091E0
:10329200E30BA633E2E1BE07C1F1E3E50E94B259B6
:1032A2001A3030F41A938ADF1A938EDD1F5FF8CF3B
:1032B200E0E50E94B259103430F41A939ADF1A935F
:1032C20045DD1F5FF8CF0E947709EBE40E94B259F7
:1032D200103830F41A936BDF1A93B6DD1F5FF8CF04
:1032E200E1E4EA930E94563759DFE4E5EA930E944B
:1032F2005637A9E0B0E0E0E00E947B62E6E3F2E14B
:10330200E093E20BF093E30B01E010E0133210F0D4
:103312000C94F5190E94BA573E960E9450629F0182
:103322000E94BA573E960E945062AF010E94BA575D
:1033320070960E945062309721F0E130A0E0FA07C7
:1033420089F4D9016C910E94BA5772960E94506218
:10335200A62FB0E0EA17FB0724F40E94BA570E9496
:10336200B75940C0E230A0E0FA07C9F4DA016D9122
:103372007C910E94BA5772960E945062E617F70734
:103382002CF0DA010E943762FF2342F40E94BA57FE
:1033920074960E945062DA01ED93FC9323C0E330ED
:1033A200A0E0FA0749F4D901AC91AF3F21F40E94A1
:1033B200BA570E94B75916C0E430A0E0FA0791F458
:1033C200D901AC91AF3F71F400E00E94BA570E945C
:1033D200CC5744F40E94BA570E94B7592F5F3F4F0F
:1033E2000F5FF3CF1F5F92CFD6DB10E0103160F496
:1033F2001A9336DDA0914F0CA13120F01A935ADDB9
:103402001A934BDD1F5FF2CFE02F0E9422640C94CF
:10341200031FE881EF5FE883A881A43610F0E0E0A3
:10342200E883E8810C948A1D0E94BC5930960C9462
:103432008A1DA091570CBB27E091560CB5C0F9DF4D
:10344200329774F00E94C359E091560C0E94C659FB
:103452000E94B158E091560CEA93DBDFE093560CE0
:1034620008950E94C359E091570C0E94C659FA93DD
:10347200EA930E9402390895EFEFE093440CEFEFD4
:10348200FFEF0E94A956EFEFFFEFE093470CF09396
:10349200480C0E94C359E091570C0E94C6590E94E1
:1034A200B158E091570CEA93B4DFE093570C0895BA
:1034B2000E941D64E0E0E093560CE093570C10E08C
:1034C20030E0343680F5A8950E94C3593A93ACDFB8
:1034D200FA93EA93E4E4FCE00E94D05800E0A09161
:1034E200440CA13010F0A03808F001C001E0E12F37
:1034F200E03041F4013029F43093570C3093560CEC
:1035020011E00FC0E13031F4003019F43093560C61
:1035120012E007C0E23029F4013019F43093570C5D
:1035220013E03F5FCECF0E9424640C94551F1A9380
:10353200A091F30BA870D1F010E0E981FA810E940A
:103542002E58AE17BF0794F4ED81E093440CEB8143
:10355200FC81E851FC4F0E94A956E0E0F0E0E093C4
:10356200470CF093480C6BDF1F5FE7CF18810C9478
:10357200031FE881EF5FE883A881A43610F0E0E042
:10358200E883E8810C948A1DE881E150E883A881F0
:10359200A43610F0E3E6E883E8810C948A1DA0913A
:1035A200590CBB27E091580CF0E031960E94CE599D
:1035B200EC59FF4FDF01E4E6F0E00E94F06108956C
:1035C2000E94BC59E050FE4F0C948A1D0E94D359B0
:1035D2000E94D959E881EA937DD10C948A1D1A93ED
:1035E20006DBE1E0E093A80B66C1A89510E0143673
:1035F20080F41A9368D1A091490CAF3F31F40E9434
:10360200E059AF3FEFEFBE0711F01A93DFDF1F5F04
:10361200EECF0E94E559689420F84DC164970E944C
:103622001D641091590CA98DAA23E2F5E091580C62
:10363200E11719F0A98DAA230AF033C01A9343D1D6
:103642000E94E059EA8DFB8DEA17FB0729F4EC8D05
:10365200A091490CEA1709F021C00E94FF56E88D9B
:10366200F98D0E942C61EA17FB0764F40E9404574B
:103672000E94EB590E940957E0E0E88FE98F1A9304
:1036820029D10CC00E9404570E94EB59E88FF98F90
:10369200E0E0F0E00E9409570E94F0590E94F659BA
:1036A200C5CF43C0E091580CE11729F0A88DB98D20
:1036B2000E9411640CF01DC01A9305D10E94E059BA
:1036C200EA8DFB8DEA17FB0729F4EC8DA091490CDA
:1036D200EA1709F00BC00E9404570E94EB590E949E
:1036E20009571A93F7D0E0E0E88FE98F0E94F65964
:1036F200D9CFA88DB98D0E941164BCF4EC8DE093F2
:10370200490CEA8DFB8DE0934A0CF0934B0CE88D4B
:10371200F98D0E940957E091580CEA93DBD0E091B1
:10372200580CEA9326DFE093580C39DF7E9714F0A9
:103732000C94DE1B1091580C0091580C1A9324DF44
:103742001E2F1A93C0D0A091490CA13010F0A038BE
:1037520008F01DC00A9318DF0E2F1017C1F00A934C
:10376200B9D030E0333098F40E947F590E94FB595F
:1037720031F0FD01EB53FA4FE0811E1709F005C04D
:103782000E947F590E94035A00833F5FEBCFE09172
:10379200590CE11799F6101781F00E94D3590E9433
:1037A200D959102F0A93F0DE0E2F0A9393D0E0918D
:1037B200590CE017B9F71093590C689420F8E88D6A
:1037C200F98D0E9424646D9608951A93A89510911C
:1037D200590CE091580CE117C9F00E94085A0E9456
:1037E200116464F4EB81A091490CEA1739F40E9448
:1037F200E059E981FA81EA17FB0709F004C0E12FD9
:1038020018810C94551F0E94F659E3CFEFEF1881EF
:103812000C94551FA895E091580CA881EA17F1F075
:10382200E881EA9350D00E94FF560E94116484F40A
:10383200E091E105E87031F4E0914B08A091490C68
:10384200EA1731F40E940C5A0E94D456E03408F070
:1038520002C0E8815EC10E94115ADDCFEFEF59C16B
:103862001A93A8951091590CE091580CE117E1F0C8
:103872000E94085A0E9411648CF4E091E105E870FC
:1038820031F4E0914B08A091490CEA1739F40E94F7
:10389200E059E981FA81EA17FB0709F002C0E12F3A
:1038A20071C20E94F659E0CFEFEF6CC21A931091E9
:1038B200590C1A93AFDF199108950E94115AE881A9
:1038C200EA93A8DF26C10E94C3590E94175A0E9498
:1038D200D0581FC10E94C3590E94175A0E94B15862
:1038E20018C1E091590CA881EA1741F40E94FF56D1
:1038F200109721F4A091490CA03009F01CC0E88176
:10390200EA9364DE0E94115AE881E093590CE09137
:10391200580CA091590CEA1719F0E881EA93D3DF09
:103922000E94FF56109721F4A091490CA03009F093
:1039320001C0E5CF03C0E881EA93CCDFEAC00E9470
:103942001D640E94E55910E030E0343628F5A89550
:103952003A93B9DF00E0A091490CA03808F401E0E5
:10396200E12FE03041F4013029F43093590C3093C7
:10397200580C11E00FC0E13031F4003019F43093EB
:10398200580C12E007C0E23029F4013019F43093E8
:10399200590C13E03F5FD9CF0E94246485C20E9474
:1039A200205AA43009F464C110914B0800912D0DE6
:1039B200E0914D08E03059F0E0934B08689424F808
:1039C2000E94255AE0E0E0934C08E0E520C0E09137
:1039D2004C08E03021F0E0934B08E2E518C0E0E04B
:1039E200E0934B08E0932D0DE091E80BE03031F0CD
:1039F200E091E80BE150EA930E94F116A091540C79
:103A0200A17039F0E091E80BE0934B08E4E4E09315
:103A12002D0DA0914B081A1721F4A0912D0D0A1714
:103A220011F0689423F824C1A091BE0BECE1EA23C3
:103A32000895A091BE0BA07411F0E2E00895A09148
:103A4200BE0BA07859F40CC0A091AD0BAF3F31F082
:103A5200EBDFE43019F0E8DFE03111F4E0E0089543
:103A6200E1E008950895A881AF3F09F451C0DCDF79
:103A7200E43011F4E1E04DC04BC0A881A23019F44A
:103A8200D3DFE83011F0E1E044C042C0E881F0E069
:103A9200EE52F94FE081E13010F0E43108F002C05B
:103AA200E1E037C035C0A881A13118F0E881E051CA
:103AB200E883E8810E9431560E942B5AA091F40BB0
:103AC200A13018F0A881A43009F006C0E6E9F0E0C0
:103AD2000E9450620E942B5A1CC0A881A13010F093
:103AE200A13108F007C0E8810E940E59EA50F34F55
:103AF200E0810FC00DC0A881A13010F0A13108F003
:103B020007C0E8810E940E59EA5FF24FE08101C0CE
:103B1200E0E0219608950E941D64E0E00E94246482
:103B2200259608951A930A9310E0103130F40E94FA
:103B3200365A0E94A4591F5FF8CF10E01031A8F541
:103B42001A930E9431170E942E58AA50B34FE09147
:103B5200500CEC930E942E58AA5FB24FE0914F0C8A
:103B6200EC93E091520CE03059F00E942E58AA5F7B
:103B7200B24F0E948557EA5FF24FE081E068EC9312
:103B8200E091500CE1500E2F0F3F69F0E02FA6EBB1
:103B9200BCE00E943B5ABF01E091510C0E94A35627
:103BA200DB01ED93FC931F5FC9CF62C01A930A93A6
:103BB20010E0103130F40E9485570E943D5A1F5F79
:103BC200F8CF10E0103440F51A930E947D161A9334
:103BD2004ADFE130F9F4E091C10BEA937EDFE15074
:103BE2000E2F0F3FB9F00E947C57EE59F94F108308
:103BF200A02FB0E0AE58B94FE091C10BEC93E02F8B
:103C02000E94425A0E94465AE091C70BF091C80B9B
:103C1200ED93FC931F5FD6CF2BC00E94205AA23097
:103C220041F0A0913508A83021F0A73011F0A5305D
:103C320009F41EC010E01530C8F40E9485570E9496
:103C42004B5AA7EDB6E00E94AD59ACEDB6E00E942A
:103C5200AD5900E0033040F40E94505A0E94535A7A
:103C62000E94A4590F5FF6CF1F5FE5CF0E945C5AF6
:103C72000991199108951A93E981E058E98310E0B6
:103C82001530C0F4ACEDB6E0EE27A10FBE1FAC912B
:103C9200E981EA1751F4A7EDB6E0EE27A10FBE1FA6
:103CA200AC91E0914B08EA1709F002C0E12F03C082
:103CB2001F5FE6CFEFEF1881229608951A93EA81EB
:103CC200EA93D9DF1E2F1F3F19F1ACEDB6E00E9437
:103CD2008557EA0FFB1F0F01ACEDB6E00E946C5A4C
:103CE200EF77D001EC930E948557EE52F94FA981EC
:103CF200A083E9810E94715A0E94765AEF77DB0114
:103D0200EC93E9810E94715AE75FFC4FA1E0A08326
:103D1200E12F38C01A931FEFE091F80BF091F90BE5
:103D2200A981BA81AE17BF073CF0E091FA0BF0917E
:103D3200FB0BEA17FB070CF411C0E981FA81FA9335
:103D4200EA930E94D1151E2F103031F01F3F21F04F
:103D5200E0914B08E11711F4E1E014C01F3F39F480
:103D6200E2EEF7E0FA93EA93EB81FC8106C0E2EF20
:103D7200F7E0FA93EA930E948557FA93EA930E9436
:103D82002D05E0E01881239608950E941D64E091BC
:103D9200DF05F091E005AC81BD81EA27FB279F0199
:103DA200E091AB0BE03089F410E0183070F4F901C7
:103DB200E17039F00E942E58AE51BA4FEC91EF5F8C
:103DC200EC930E947B5A1F5FF0CFE091AC0BE03086
:103DD20089F418E0103170F4F901E17039F00E94B1
:103DE2002E58AE51BA4FEC91EF5FEC930E947B5A82
:103DF2001F5FF0CFEC81FD81E093DF05F093E005DA
:103E02000E942464269608951A930A9310E00E9451
:103E120085570E94825A11F00C944F1F00E0023025
:103E2200F0F40E94875A0E948A5AAFEFB6E00E94CD
:103E320085570E948A5A0E94975A0E948A5A0E9463
:103E4200505A0E94535A0E94A459ACE2B7E00E9411
:103E520085570E94535A0E94A4590F5FE0CF0E94D7
:103E6200875A0E949A5ADB01AE0FBF1FEA81FB817B
:103E72003996EC930E94505A0E94A05AAE0FBF1F6F
:103E8200E2E3F0E0ED93FC930E942E58AE52B94F5C
:103E9200EA81FB81EC59FF4FEC9304C01F5F1530A0
:103EA20008F4B5CF198108812496089524970E94B9
:103EB2001B644091DF055091E005FA010E944A61BE
:103EC200AFEFB0E0EA272E2F10E0103110F00C9483
:103ED200EF1FA091AB0BA13011F4183038F0A09174
:103EE200AC0BA13011F4183008F436C00E9485578B
:103EF2000E94A75AC1F0003810F0003B08F001C040
:103F02000F5F003921F40E948F2FE03009F407C0BF
:103F12000E940E570E94B55AE0E00E94C55A00382E
:103F220008F400E814C0003208F40F5F003121F4F5
:103F32000E948F2FE03009F407C00E940E570E94A2
:103F4200B55AE1E00E94C55A003B09F400E00E9424
:103F52008557EA5EF24F0083A091AB0BA23011F4B9
:103F6200183008F039C00E9485570E94A75A71F094
:103F7200003810F0003B08F001C00F5F003911F467
:103F82000E948F2F003808F400E821C0003208F4A4
:103F92000F5F003131F40E948F2FE03011F020309A
:103FA20009F412C02093440C0E948557E558FC4F37
:103FB2000E94A9560E946759A091AC0BA33021F42C
:103FC200E12F0E94F25420DF003B09F400E00E943E
:103FD2008557EA5EF24F00831F5F77CFE0E0F0E0A3
:103FE200E0933208F0933308E0913908EF5FE093F1
:103FF2003908E091070CA0913908EA1751F4E091D1
:10400200070CF0E0A0E0B1E00E946462EA1BE093DA
:104012003908A0913508A13019F0A93009F0BCC0C7
:10402200A091840BB091850BE4E1F0E00E94F06175
:10403200309719F4E1E0E0933B0800E00031A0F58D
:104042000E947C57EE50FA4FE081E03059F10E9415
:104052007C57EE5FF94F0E94CE5A0E947C57EE5E6B
:10406200F94F0E94CE5AE02F0E9457570E941358D0
:104072000F01E02F0E9457570E941956DF010E943C
:104082007C570E94D25A0E94D65A0E947C570E94A4
:10409200D25A0E94E05AE02F0E9453570E94465A79
:1040A2000E94A1550F5FCACF0E94E55A21F00E94DB
:1040B200F555E07809F44EC00E94F555EF733E2F96
:1040C2003A930E947D16A091BD0BA03049F4BCDC4E
:1040D200E13031F4E0913608EA93CFDCE03009F4C4
:1040E20039C00E94EB5AAE0FBF1FEC91EC71EC305D
:1040F20021F4E0913908E07861F40E94F15AD3DCAE
:10410200A4ECBBE0E09136080E94FB5AEC91EA93E2
:10411200CADCE32F0E9453550E94465A0E94A155C1
:104122000E94F15ADADC1E2F1130A0F00E94FF5AD1
:104132000E9413580F010E94FF5A0E941956DF0174
:10414200E12F0E940E590E94D65AE12F0E940E5969
:104152000E94E05A10E01031F8F40E948557EE599F
:10416200F94F30813F3FB1F00E948557EE58F94F29
:104172000E94CE5A0E94FF5A0E9413580F010E94B9
:10418200FF5A0E941956DF010E943B560E94025BB1
:104192000E94E05A1F5FDFCFA0913508A23039F0AC
:1041A200A83029F0A53019F0A73009F0DDC1E0E010
:1041B200E0933C0800E0053010F00C94B5220E9418
:1041C2007C570E94825A11F40C94B322E0913C086D
:1041D200EF5FE0933C080E94E55A91F00A9356DCA7
:1041E200E03069F00E947C57EE52F94FE081A091D5
:1041F2004B05B0914C05F0E0EA17FB0709F4B2C198
:10420200E0E0E887E98740E050E04330E0E05E0725
:1042120014F00C9453220E94095B0E949A5A0E9445
:104222000C5BE27041F40E94125B0E94A05A0E9451
:10423200155B309709F40CC10E94195BE07811F00C
:104242000C9405220E94095B0E949A5A0E940C5B00
:10425200E17069F40E94125B0E94A05AAE0FBF1F68
:10426200FA010E94465A0E94205B31966AC00E945F
:10427200265B0E949A5A0E940C5BEA932EDCE15064
:104282001E2F0E943B56E03049F50E94295B0E9496
:10429200A1550E94365A0E941956309759F00E9431
:1042A200295B0D901C900E94365A0E941956E01507
:1042B200F1050CF012C00E947C57E95BF24EE491CA
:1042C200E03021F00E947C570E942E5B0E947C57B6
:1042D2000E944B5AE2E0E093280D22C00E94125B3A
:1042E2000E94A05AAE0FBF1FFA010E941358FF93FB
:1042F200EF930E94125B0E94A05A0E94155BDF019D
:104302000E943B56F0E00E94CE59AF91BF91ED93CF
:10431200FC930E9485570E94E05AE12F0E94365B6F
:104322000E94125B0E94A05A0E94155BFF234AF46E
:104332000E94125B0E94A05AAE0FBF1FFA010E9498
:10434200A4590E94095B0E949A5A0E940C5BEC716C
:10435200EC3021F4E0913908E078E9F40E94125B34
:104362000E94A05A0E94155B7E973CF40E94095B52
:104372000E949A5A0E940C5BE072A0EFB6E00E9483
:104382007C570E949A5A0E943A5B0E943F5B0E94AD
:104392009A5A0E943A5B0E94265B0E949A5A0E9495
:1043A2000C5B0E94425B81F10E947C57E95BF24EFA
:1043B200E491E03081F00E947C570E942E5B0E94C3
:1043C2007C57EE52F94FE0810E94715A0E94765A50
:1043D200E058DB01EC93ACEDB6E00E947C57EA0FAB
:1043E200FB1F0F010E94195BE058D001EC93E3E040
:1043F200E093280D0E94265B0E949A5A0E940C5B51
:10440200EA9379DBE093290D0E94475B0E94A05A50
:104412000E94155B3097E1F00E94475B0E94A05A10
:10442200AE0FBF1FFA010E94465A0E94205B0E94F3
:10443200475B0E94A05A0E94155B309749F40E9484
:10444200125B0E94A05AAE0FBF1FFA010E94A4592C
:104452000E94125B0E94A05A0E94155B3097F9F4E9
:10446200E885F9853196E887F987042E052A49F40B
:104472000E94095B0E949A5A0E944A5BED7FD0011A
:10448200EC93E1E0F0E0E417F50749F40E94095BE0
:104492000E949A5A0E94525BED7FD001EC934F5FCB
:1044A2005F4FB3CEA885B985139711F00C94B32250
:1044B2000A93ECDAE03021F00E947C570E942E5BD6
:1044C2000E948F2FE030A9F00E940E570E945A5B83
:1044D200E8E0EC930E94195BAE81BF811496EC93E5
:1044E2000E947C57EE52F94FE081AE81BF810E945B
:1044F200C55A0E947C570E944B5AACEDB6E0EE279B
:10450200A00FBE1FEC930E94095B0E949A5A0E9460
:10451200625BEC71E83031F50E948F2FE03011F1CF
:104522000E940E570E945A5BE3E0EC93AE81BF817A
:10453200EFEFEC930E94265B0E949A5AE60FF71F58
:10454200E281AE81BF810E94675B0E943F5B0E9455
:104552009A5AE60FF71FE281AE81BF810E946C5B1F
:104562000E94715B0F5F27CEA0913508A23029F01F
:10457200A83019F0A53009F05FC010E0103110F03A
:104582000C941D230E948557EE59F94F30813F3F0D
:1045920011F40C941B230E948557EE58F94F0E9488
:1045A200CE5AE12FA2E8B6E00E943B5A0F010E94C8
:1045B200795BDF010E943B560E94025B0E94E05A37
:1045C2000E94795BDF010E941164C4F4E12F0E9412
:1045D200425A0E941956DF010E9411647CF40E9423
:1045E2007E5B0D901C90E12F0E94425A0E94195648
:1045F200D001AE1BBF0B0E9411640CF01BC0E12F57
:10460200A2E8B6E00E943B5ABF010E947E5B0D9079
:104612001C90E12F0E94425A0E941956DF01F001BC
:10462200EA1BFB0BDB01ED93FC933A93E5E0EA9383
:104632000E949D341F5FA2CFE0913808E03041F420
:10464200E0913208F0913308E0933008F09331089A
:104652000E9422642A9608950E941B64E5D9E031E3
:1046620011F40C949C2320E030E040E050E010E094
:10467200133060F50E94A1590E941956309721F11A
:10468200A1ECBBE00E946C5A0E9431562E2B3F2BAC
:10469200A1ECBBE00E946C5A0E94425B19F00E949E
:1046A200835B22C2A4ECBBE00E946C5A0E9431568A
:1046B2002E2B3F2BA4ECBBE00E946C5A0E94425B63
:1046C20019F00E94835B10C21F5FD2CF00E0053059
:1046D20030F50E947C570E94825AF9F010E01330A4
:1046E200E0F40E94265B0E949A5ADB01AE0FBF1FC4
:1046F2000E946C5A0E9431564E2B5F2B0E943F5BE8
:104702000E949A5ADB01AE0FBF1F0E946C5A0E9490
:1047120031564E2B5F2B1F5FE2CF0F5FD8CFF901CF
:10472200E423F523309739F0E1E0E093280DE0E04F
:104732000E942264D9C1E1E00E942264D5C1E091C5
:104742002B0DE03011F40C94F823E091080CE130C9
:1047520059F4A0912B0DA13311F4EFE001C0E0E078
:10476200EA930E94C34843C0E23059F4A0912B0D52
:10477200A13311F4E6E001C0E5E1EA930E94C348E7
:1047820036C0E33041F5A0912B0DA13319F50E94FB
:104792008A5B0E94915B0E94955B0E94995BE8E5AF
:1047A200EA930E94174DE0E40E94A45BE8E3EA93D7
:1047B2000E94174DE2E4EA930E94174DE1E4EA9366
:1047C2000E94174DE0912A0D0E94F2540E947856E1
:1047D2000E946A4F0CC00E948A5BE9E4EA930E943D
:1047E200174DE0912B0D0E94AB5B0E943D4F089547
:1047F2000E941D6430E0A0913508A23029F0A83053
:1048020019F0A53009F038C134E0AD81A03410F0C0
:104812000C943B25E0914B08E03011F4E2E062C1D8
:10482200ED81EA930E947D16FFD8E03131F4E1E395
:10483200E0932B0D84DFE1E055C106D9E03011F49D
:10484200E3E050C109DFE13011F00C943B2535E083
:1048520010E00E9485570E94825A11F00C94342570
:1048620000E0033010F00C94F8240E94875A0E9452
:104872009A5A0E94AF5BEA0FFB1F0F010E94B35BC3
:10488200D001EC93AFEFB6E00E9485570E949A5A8E
:104892000E94AF5BEA0FFB1F0F010E94BA5BD001BF
:1048A200EC930E94975A0E949A5A0E94AF5BEA0FB9
:1048B200FB1FBF01A091BE0BECEFEA230E2E0E945C
:1048C200C15BE029DB01EC93AFD8E43159F40E94DB
:1048D200975A0E949A5A0F010E94AF5B0E94C95BCD
:1048E200ED7F0AC00E94975A0E949A5A0F010E94B5
:1048F200AF5B0E94C95BE260DC01EC930A93BDD816
:10490200E03011F40C94D8240E94875A0E949A5ADB
:10491200DB01AE0FBF1F0E94D55BEA93DED82E2FBC
:10492200213048F0E22F0E940E590E94E05AE22FF5
:10493200E1500E94365B0E94505A0E94535A0E94D4
:1049420013580F010E94DA5B0E941956D001ED93B1
:10495200FC93013031F4E091C90BF091CA0B30970E
:1049620009F009C00E94975A0E949A5A0E94DD5B80
:10497200E062D001EC93023031F4E091CB0BF09184
:10498200CC0B309709F009C00E94975A0E949A5A9C
:104992000E944A5BE062D001EC930E94975A0E9407
:1049A2009A5A0E94525BE062D001EC9306C00E94C8
:1049B200505A0E94535A0E94A45936D8EC3019F426
:1049C200E0E0E0933908ACE2B7E00E9485570E942C
:1049D200535A0E941358BF01ADECBBE00E94D55B55
:1049E2000E94A356DB01ED93FC930F5F3ACFA09197
:1049F2003508A23011F0A53019F4AC81A03808F0C6
:104A020007C0E0914B08EA93EE81EA930E94D51722
:104A12000E948557EE52F94FAC81A083A7EDB6E014
:104A22000E948557EA0FFB1FA0914B08A083ACEDB3
:104A3200B6E00E948557EA0FFB1FAD81A083AC81CF
:104A4200A03838F4EC810E94715AE75FFC4FA1E074
:104A5200A0830E94975A0E949A5A0E94DD5BED7FC2
:104A6200D001EC9331E01F5F313011F0153008F0C6
:104A720001C0EFCEE32F36C0A0913508A13091F5E9
:104A820010E0103178F50E948557EE50FA4FE08120
:104A9200E03031F50E948557EE50FA4FAC81A08389
:104AA2000E942E58AE5FB94FE091C10BEC930E9469
:104AB2002E58AE5EB94FE091C40BEC93E12F0E94E9
:104AC20053570E94A459E12F0E9457570E94A4599C
:104AD2000E9485570E94D25A0E94E05AE1E002C029
:104AE2001F5FCFCF0E942464269608950E94205A09
:104AF200A23021F0A0913508A53021F40E94E35B99
:104B02000E94F155A0913508A830B9F50E94E35BE7
:104B12000E94ED55EA81ACE0EA9FF001E050FD4FC2
:104B2200E081EF771E2FA091060CA03049F40E947D
:104B320085570E94EE5BDF010E943762309709F0D1
:104B420016C00E9485570E94035A00810E94855711
:104B52000E94035AAFEFA0830E9485570E94EE5B2A
:104B62000E94F35B1A930E942B05689420F8E0914F
:104B7200060CE03011F0689420F819810881239620
:104B8200089564970E941D64A0913508A23039F4FB
:104B9200E0914B08EA93E98DEA930E94D517A09120
:104BA2003508A83011F00C943A260FEF30E030317E
:104BB20048F40E947F59EE59F94FE081AE2FE88DFB
:104BC200EA1709F402C03F5FF2CF0E947F59EE5507
:104BD200F94F00810F3F11F40C943A260E947C5742
:104BE2000E94035A10810E94085A0E941164F4F430
:104BF200ACE4BCE00E94205B0E947C570E94EE5B0A
:104C02000E94FF56A083B1831A930E946B1C0E94DC
:104C12007C570E944361E953FA4F20810E94F85B5E
:104C22002A930E94FF5B2A930E94F1550E94045727
:104C32003097F9F40E947C570E94035AAFEFA08389
:104C42000E947F590E943D5A0E947F590E94055C32
:104C52000E947C570E94EE5B0E94F35BE0E0F0E072
:104C62000E9409570E94F0590A930E942B056894EA
:104C720020F80E942464699608951A9310E0103176
:104C8200A0F40E948557EA5FF24FE081EF77AE2FE2
:104C9200E981EA1729F4E12FEF5F0E94425B09F4F0
:104CA20002C0E1E003C01F5FEACFE0E01881229674
:104CB20008951A930A930E940A5C0E94115C0E9452
:104CC2004A3FE030F1F00E94165C10E01031C8F467
:104CD200A091300DAF5FEA2FEF70E093300DEF5FE0
:104CE200EA93CBDFE03059F0E3E0E093280DE09166
:104CF200300DF0E0EF5FFF4EE093290D02C01F5F21
:104D0200E5CF0991199108951A93E091DD05F0918B
:104D1200DE05E093260DF093270DE8E7F0E0FA9325
:104D2200EA93ECEDF0E0FA93EA930E94553710E033
:104D3200103110F5E12FEF5FEA939FDFE030D1F001
:104D42000E942E55EA5F0E94F2540E948837EFEFCC
:104D5200F7E00E943455AAE0BCE00E948557BD01ED
:104D6200AAE0B0E00E946B61E60FF71FFA93EA93A4
:104D72000E944A551F5FDCCF25C39BDFA091280DFF
:104D8200A13021F4E7E0F8E00E941D5CA091280D1B
:104D9200A23021F4E4E1F8E00E941D5CA091280D0C
:104DA200A33059F4EFEFF7E00E94255CF0E0E05009
:104DB200F04FFA93EA930E942D05A091280DA4309A
:104DC20041F4ECE1F8E00E94255C0E94F2540E945A
:104DD2002D05A091280DA53029F4E091290DEA9323
:104DE2000E942609A091280DA63041F4E4E2F8E0E1
:104DF2000E94255C0E94F2540E942D05E0E0E0939F
:104E0200280D0895A881B9811196E1E0EC930E94E2
:104E12000C5AA881B9811296ED93FC930E941A1D37
:104E2200A881B9811596EC930E946C56A881B9812C
:104E32000E94675BE091AE05A881B981EC93E09195
:104E4200490CA881B9811496EC93E091AD0BA8812D
:104E5200B9811896EC9343C464970E941D64E98D4E
:104E6200EA930E94641CAA8DAF3F29F40E940C5A57
:104E72000E94D456EA8FEA8DEA930E947D160E9420
:104E82001A1D3E2FA88DAF3F21F00E94251DE03054
:104E920009F001C08BC00E94FF560E947F59AE17D5
:104EA200BF071CF0D9DBE13009F080C0E091F50BBF
:104EB200E03021F10E946C56E13041F00E948F2FC8
:104EC200E03021F00E94A52FE03009F004C00E94DA
:104ED2000E570E942A5C0E946C56E13021F40E9417
:104EE200952FE03009F409C00E94E056EE52F84FC7
:104EF200FA93EA9387DF0E94F15656C0EA8DEA934D
:104F02000E94315C1E2F113011F00C94D527A09114
:104F1200F70BA13059F4E0914B08EA930E940C5A26
:104F2200FA93EA93EFEFFFEF0E9420570E94FF5699
:104F32000E947F590E94CE590E940957689420F816
:104F4200E091060CE030A1F40E947C570E94EE5BD7
:104F52000E94FF56A083B1830E94F85B0E947C5797
:104F62000E944361E953FA4FE081EA930E94FF5B9A
:104F72000E940457309741F4E0E0E093490CE98D38
:104F8200EA930E94721C04C0E98DEA930E946B1C92
:104F9200E0914B08EA930E945558FA93EA93E32F63
:104FA2000E94F2540E94981AE1E001C0E0E00E94DF
:104FB20024646B96089550DBE13031F4AFD7E030D2
:104FC20019F0C2D7E03009F00BC00E945558E093A7
:104FD2004A0CF0934B0C0E940E570E942A5CB9C2F5
:104FE200C1C21A930A93E091290DEA930E944D16C9
:104FF2001E2F1F3F11F40C944628E0912B0DE03038
:1050020011F00C9445281A930E947D16E5E0E09376
:10501200280D1093290DA0913508A23031F40E9479
:10502200365C0E948B1EE13009F00EC0A0912C0D5F
:10503200A13331F4E0914B08EA931A930E94D517F9
:10504200E1E3E0932B0DA2C3A0913508A83089F4C7
:105052000E945558FA93EA930E94311C0E2F0F3F7B
:1050620041F0EFEFEA930A93EA93F6DEE03009F0BB
:105072008DC3A0913508A53021F49DDFE03009F001
:1050820085C3E0E3E0932B0D06C0E0E3E0932B0D34
:10509200E4E0E093280D7AC3E0915B09E093290DE7
:1050A2000E943D5C08951A93E6E0EA930E94C34889
:1050B2000E948A5BA0915B09A83541F4EAE2F8E01C
:1050C2000E9493560E94955B0E943D4FA0915B09FE
:1050D200A335F1F410E0A0913508A83021F0A230F8
:1050E20011F0A53009F411E3E3E5EA930E94174DAC
:1050F2001A930E94475C0E94475C0E94475C0E9490
:10510200174DE0E0E0932B0D0E94955B0E943D4F0E
:10511200A0915B09A93451F40E944C5CE093290DE3
:105122000E948456E0932C0D5CDF09DB4BC11A937D
:10513200A0915B09A13841F4E0916109E03421F4C6
:10514200E0916209E43409F029C0E0915C09E0933E
:10515200820BE0915D09E093810BE5E6F9E00E94A4
:1051620071580E942A4CE130C8F0A0915D0BA23424
:1051720091F4E0915E0BE53421F40E94634CE093DC
:10518200290DE0915E0BE13431F40E94634CE0930F
:105192002A0D0E943D5C0E94E24BE3CFA0915B0985
:1051A200A13821F4E0916409E43409F019C0A09116
:1051B200830BA03029F0E6E4E0936309E03009F4C0
:1051C20005C0E091830BEF5FE093830BA091830B0B
:1051D200A43418F0E0E0E093830BE1E0E0937E0B6F
:1051E200A0915B09A93829F4E0E0E0937E0BE093FB
:1051F200800BE8C0E1E00E94535C0E9428560E94A6
:105202002D560E9428560E9428560E948837E4E9AB
:10521200F4E00E943455E09136080E94565CE2EABE
:10522200F4E00E943455E2E0E0935D0C08951A9395
:1052320010E0103458F4E12F0E9453550E94A459F3
:105242000E945A5C0E94A4591F5FF3CF10E01031F4
:1052520030F40E9485570E94E05A1F5FF8CFE9811F
:10526200E03009F406C0A0913608AF5FE3E00E9487
:10527200ED61E09336080E945C5A30C21A930A9399
:1052820010E0103410F00C948B291A930E947D16B2
:1052920000E0E12F0E9453550E9419563B97CCF033
:1052A2000E945D5C0F01E12F0E9453550E94195626
:1052B200D001ED93FC930E94EB5AEA0FFB1F0F0102
:1052C2000E94EB5AAE0FBF1FEC91EE7FD001EC9320
:1052D20001E00E945A5C0E9419567597A4F00E9440
:1052E2005D5C0F010E945A5C0E941956D001ED9339
:1052F200FC930E94EB5AEA0FFB1F0F010E94EB5A2C
:105302000E94025801E0013019F41A930E94A71674
:105312001F5FB7CF3BC21A9323FE03C00E94625C99
:10532200D2D50E94B234E030E1F1E0E00E94675C45
:10533200103808F5113219F40E94625CC4D51D348C
:1053420029F40E946E5CE3E0E09334081B3261F4BE
:105352000E94785CEAE2EA93E5E3F8E0FA93EA93E2
:10536200E09136080E947E5C1F3221F4E1E0EA936C
:105372000E948E093FDF1038A0F00E94825C89F003
:10538200A091AD05A23031F4E091BD0BEA930E94E9
:105392008E0930DFA091AD05A43019F4E3E0E0936B
:1053A20034080E94E55A21F00E94F555E03808F4CD
:1053B20009C0E0913B08E03029F00E940A09E0E0D0
:1053C200E0933B08199108950E948A5C0E948E5CCA
:1053D2000E94535C0E9428560E948837A091370889
:1053E200A23021F4E8E3F8E00E943455A091370896
:1053F200A13021F4EFE3F8E00E943455E091370840
:10540200E03021F4E6E4F8E00E9434550E94965C14
:105412000E9428560E9488370E949B5C0E94A05CD2
:105422003197FA93EA930E94A55C0E94C7370895C8
:10543200E1E003C0E0E001C0E2E0E0933708C4DF4E
:105442000895A881A03310F0AA3308F01DC00E946D
:10545200AC5C0E94B15CAAE0B0E00E949361DF0103
:10546200E8810E94B65CEA0FFB1FE0934108F093CB
:105472004208E2E0E0935D0C0E94965C0E9428568E
:105482000E942D560E949B5CA881A33461F40E9465
:105492008E5CE0935D0C0E94965C0E9428560E94EE
:1054A2002D560E949B5C50C1A0E023FCA1E0A030DD
:1054B20019F0A881A03009F016C0E89423F8E7E0BB
:1054C200E09334080E94FB37A0914D08A03019F4F4
:1054D2000E94B95C09F407C0E7E0EA930E94B9565A
:1054E200F2D4E89424F824FE18C00E94BE5CEAE5D7
:1054F200F0E00E94C55C19F0A881A13069F40ED5D4
:10550200E03051F00E94CB5CE981EA93E0914B08D4
:10551200EA930E94365CD7D40BC00E94BE5CE8EED0
:10552200F3E00E94C55C21F40E94D25CE0934C0837
:10553200D6C0E091EB0BF091EC0B0E94D65C11F41B
:10554200E2E00895E091E90BF091EA0B0E94D65C4B
:1055520011F4E1E00895E091EF0BF091F00B0E945D
:10556200D65C11F4E0E00895EFEF0895A0913508BC
:10557200A23021F40E9408380E949C05A0913508AF
:10558200A83009F4FAD4A0913508A53009F401D164
:10559200DBC01A93E2E0EA930E949E32E2E0E093DB
:1055A2005D0CE981EA934DDFA981AF3721F4E091E7
:1055B200E105E37009F403C0E2E0E0933408A98155
:1055C200A13239F0A33421F40E94AC5C109709F0A7
:1055D20016C0A0913708A33009F42EDFA091370836
:1055E200A23019F4E1E0EA93C1DFA0913708A030BC
:1055F20021F4A091EE0BA13009F001C01BDFA981BB
:10560200AD3311F00C94642B0E94FB37E091370804
:10561200E030B9F4E0914108F0914208FA93EA933C
:105622000E948B1E1E2F113051F4E0914108F0911F
:1056320042080E94DA5CE0E0EA9398DF01C0FADEF9
:1056420042C0E13081F475DFEF3F49F0E3E00E94B0
:10565200DF5C0E946E5C6DDFE093400803C0E1E016
:10566200EA9384DF30C0E23001F50E94AC5CA034E2
:10567200E0E0BE07C4F4E0914108EA930E947D167F
:105682000E940838E2E00E94535C0E9428560E9461
:1056920088370E940E560E944A550E949E05E3E0FA
:1056A200E093370801C0C8DE0EC0E33061F4E09138
:1056B2004108EA930E947D16E0914108EA93EFEFD8
:1056C200EA9396D8B9DEA981AD3409F4B1DEA98195
:1056D200AF3221F4E1E0EA930E948E09188122960A
:1056E2000895E091BD0BE33631F4A0913508A23064
:1056F20009F4A0DE12C0E23611F49EDE0EC0A091C3
:10570200AD05A23029F4E091BD0BEA930E948E0907
:10571200A091AD05A43009F48BDE08950E940E1EFF
:105722000E940838E0E0E0933708A881A13039F4FC
:105732000E94B95C21F0A091EE0BA03009F402C0E6
:1057420079DE02C00E949C05219608951A930A935D
:105752000E94E55CD9F00E94F25CC0F00E94825C7B
:10576200A1F41A930E94FA5C89F40E94365C0E94AA
:105772008B1EE13021F40E94251DE13009F004C0A6
:105782001A930E94315C0E2F01C0ABDF099119916F
:1057920008950E940E1EE89421F8E0E0E0933A0892
:1057A2000E949C0508951A930E94E55C49F00E94AC
:1057B200F25C30F00E94825C11F4FDDB01C091DFEB
:1057C2001BC40E941D640E94E55C11F40C943A2CE7
:1057D2000E94B5343E2F3A93DCDEA091060CA03035
:1057E20021F4303810F0313808F00CC03F770E94B5
:1057F2007F590E94035A00810F3F21F0EFEFEA9395
:105802000E94015DA091060CA03011F0303808F41E
:1058120030C03F773A930E947D16E091BD0BE03095
:1058220039F53A930E94FA5C81F50E94251DE13018
:10583200F1F40E941A1DE03061F43A930E94315C47
:10584200E03031F0E0914B08EA933A930E94D51789
:105852000EC0A0913A08E32FEA1BAAE4B7E00E9427
:10586200FB5A0C910F3F19F03A930E94015D01C05F
:1058720038DF20FE0AC0E091060CE03019F4BED3F6
:10588200F4D401C04BD5E89420F80E9424642496F5
:1058920008950E941B64A0913508A33011F40C9462
:1058A200092EE0915508ED3411F00C942C2DE09165
:1058B2005608EA3511F00C94E12C24FC81C0E091E9
:1058C2005708E0532E2FE0915808E0533E2FE9E5A8
:1058D200F8E00E9471580E947E56AB3429F40E946F
:1058E2008A560E94634C0E2F0E947E56A43529F4DC
:1058F2000E948A560E94634CAF01E091F10BE317BC
:1059020031F5E0E0E093B50C0E94CB5C4093430894
:1059120050934408A0914C080A1759F0E7E0E0932D
:10592200340800934C082093B40CE0E0E0934B0859
:105932000DC0A091B40C2A1721F0A0914A08A03002
:1059420009F004C0209334082093B40C35C0A09110
:105952004C08A03049F4A091F20B0E947F59E25505
:10596200FF4FE491EA2309F40CC0E7E0E093340826
:105972002093B40CE0E0E0934B08E0915408E093EC
:10598200B50CE0915408A091B50CEA17A9F4409324
:1059920043085093440800934C080E94CB5CA091AA
:1059A200B40C2A1721F0A0914A08A03009F004C0D3
:1059B200209334082093B40C273011F40E94255A06
:1059C200E0915608E93439F4E7E00E94DF5C0E9476
:1059D200D25CE0934B08E0915608E03039F4E4E001
:1059E2000E94DF5C0E94D25CE0934B08E091560873
:1059F200E03519F4E1E0E0933408E0915608EC3424
:105A020049F4E4E0E0933408E0915708E053EA9364
:105A12000E94FB05E0915608E334E9F4A09157088F
:105A2200A13320F0A0915708A93308F014C00E94B6
:105A3200075DE0913E08EA930E94BE18E091540887
:105A4200EA93E7E5F8E0FA93EA930E9471590E941B
:105A520054620E94CD4EE0915508E03521F4A091A8
:105A62003508A13009F003C00E94785CC3DBE091E5
:105A72005508EF3459F4E0915608EE3439F4E091C8
:105A82005408EA93EAE5F8E00E940D5DE0915508BA
:105A9200E33579F5E0915608EF3359F5A0915708AF
:105AA200A03360F0A0915708A93340F4A0915808A0
:105AB200A03320F0A0915808AA3308F01AC00E941F
:105AC200075DE0915808E0531E2F103011F40E9438
:105AD2001E18E0915408EA93EDE5F8E0FA93EA9390
:105AE200E12F0E9453550E9457550E945C550E9417
:105AF200CD4EE0915508E33411F00C94CE2DE09197
:105B02005608EF3311F00C94CE2DE0915808E03393
:105B120019F4EFEFE0933F08A0915708A03320F06B
:105B2200A0915708A93308F01BC00E94075DE091BD
:105B32003F08EF5FE0933F08E0913E08EA93E0916F
:105B42003F08EA930E946417A0913E0CB0913F0C6B
:105B5200109721F4A0913F08A03408F001C0E7CFCC
:105B6200E0913F08EA930E947D160E949658E0E673
:105B7200F8E00E9493560E9469550E945A580E946A
:105B8200B34D0E9472550E9454620E94B34D0E940E
:105B92000E560E94D84D0E94A14EE0915508E43461
:105BA200B9F5E0915608E43499F514E0E1E0E093A8
:105BB2005409103538F40E948557ED5AF74FE081A9
:105BC200E03208F41AC00E948557ED5AF74FE0817F
:105BD200E33259F40E948557EC5AF74FE081E053C3
:105BE200EA930E94C3481F5F06C00E948557ED5A80
:105BF200F74F0E94135D1F5FDCCFE0915308EA93D9
:105C02000E948E4EE3E6F8E00E9493560E94A14E57
:105C12000E942264269608951A930A930E94175DA1
:105C220011F40C94862EE0913408EF770E2F009336
:105C320034080E9408380E945056E4E0F0E0FA93DB
:105C4200EA930E948837013021F0A0913508A130F3
:105C520009F00BC0EAEAF4E00E9434550FDB0E941F
:105C6200115C0E94D1340E940838073041F40E942E
:105C72000E1EE0E0E09337080E942E0545D804305E
:105C820031F4E6E6F8E00E9434550E949D050830A2
:105C920019F40E941D5D71D1053019F40E941D5D39
:105CA20078DD013051F4E89423F8E0E0EA93BFDABA
:105CB200009335089FDA0E949C05093071F4E0E0F8
:105CC200EA93B5DAE0E0E0933A08E89423F80E9418
:105CD2009C050A93E1E0EA93E7DB023081F4E0E01D
:105CE200E0933A08E0E0F0E00E94DA5CE89423F8FE
:105CF2000A93E1E0EA93D8DBE1E0EA930FDD0330B7
:105D020011F40E94054800933508A0913508A73088
:105D120011F00C943B2F0E940A5CE4E6F0E00E9432
:105D2200275DE03021F0A0913708A03009F00FC0C4
:105D32000E94165CE091260DF091270DA091DD05E1
:105D4200B091DE05EA17FB0711F00E9485260E943A
:105D5200B234E030F1F0E2E00E94675C1A9371DB4A
:105D62001D3409F465DB1D33A1F40E94FB37E1DB2E
:105D7200EF3F49F0E3E0E09334080E946E5CD9DB28
:105D8200E093400806C0E7E8E0933408E0E0E093DF
:105D92003708A0914B08A03031F0E0914B08A09158
:105DA2004A08EA1709F457C0E0914B08E150EA9318
:105DB2000E94F116A091540CE1E0EA23E13021F4B3
:105DC200E091E105EF7C09F429C0E0E0E0934A08A4
:105DD200E091B40CE03019F0E09334081EC012E0F8
:105DE200E091E105EC7009F018E0E091E80BA09178
:105DF2004B08EA1781F0E091E105E07439F011E017
:105E0200EAE2EA93EBE6F8E00E940D5DE091E1053B
:105E1200E07809F019E0109334081DC00E94083898
:105E22000E942E050E945056E4E0F0E0FA93EA93B5
:105E32000E948837EBE4EA930E945637E0914B08C0
:105E4200EA930E941633EEE6F8E00E943455E091A0
:105E52004B08E0934A08A0914B08A03021F4A0918E
:105E62004A08A03009F406C0E0E0E0934A08E7E8F7
:105E7200E0933408A0913508A33011F40E94FF4545
:105E8200A0913508A13009F446DAA0913508A23074
:105E920009F45CDCA0913508A83009F492DCA091E9
:105EA2003508A53009F47FDCA0913508A93049F402
:105EB200E0E0E0933C08E0913508EA93E0E0EA9301
:105EC200F3DA0C94ED320E940E57E050F84FA6E040
:105ED200A0830E940E57E150F84FAB81A0830E942D
:105EE2000E57ED5FF74FAA81A0830E940E57EF5F16
:105EF200F74FA881B981A083B1830E94715B0E9490
:105F0200EB3C0C943F33E881EF5FE883A881A53036
:105F120010F0E0E0E883E8810C94C132A0912F08F0
:105F2200BB27E0912E0805C0A0912D08BB27E09168
:105F32002C08F0E031960E94CE593596DF01E5E05B
:105F4200F0E00E94F06108951A9310912F08E091F9
:105F52002E08E11781F0A9E01A9FF001E050F84FF6
:105F6200E081E13011F0E23011F4E1E045C01A9332
:105F7200CADF1E2FECCFE0E03FC01A930E940E1E34
:105F820010E01130B0F40E9485570E94035AAFEF1F
:105F9200A0830E9485570E942B5D0E9485570E9414
:105FA200325D0E9485570E94EE5B0E94F35B1F5F89
:105FB200E8CF10E0103130F40E9485570E94055C52
:105FC2001F5FF8CFE091E105E37019F00E94B95C20
:105FD20009F402C0689401C0E89421F8EFEFE0935D
:105FE2004908E091060CE03029F408D03ED1E8944B
:105FF20020F802C00E942F05199108950E941B6487
:1060020030E0313050F40E947F590E94325D0E948C
:106012007F590E942B5D3F5FF4CF30E00E94571CF6
:106022001E2F1F3F11F0313008F061C050E000E038
:106032000E947C570E94035AE0811E17E9F40E94D5
:106042007C570E94EE5BDF010E9437620E94FF567E
:10605200EA17FB0761F00E947C570E94EE5B0E94E8
:10606200FF56A083B1830E947C570E94395D51E0A4
:106072000E947C570E94405D503099F500E00E94DA
:106082007C570E94035AE081EF3F59F50E947C57EA
:106092000E94035A10830E947C570E94EE5B0E946A
:1060A200FF56A083B1830E947C570E944361E7534D
:1060B200FA4FA091490CA0830E947C570E94475D31
:1060C200FF93EF930E940C5A0E94D456AF91BF9156
:1060D200EC930E947C570E94395D0E947C570E947B
:1060E200405D1A930E945E1C1E2F3F5F9ACF00E014
:1060F2000130D8F40E947C570E94FB5931F4FD0113
:10610200EB53FA4FE081EF3F09F40DC00E947C5738
:106112000E94395D0E947C570E94035AAFEFA08310
:106122000A930E942B050F5FE3CF40E04031E0F578
:1061320050E000E0013060F5503041F50E947C579C
:106142000E94475D20812A930E947D160E947C57FF
:106152000E944361EA53FA4FE081E13059F42A93F5
:106162000E94341DE13031F4A42FAF5FE091C10BE6
:10617200EA1709F00BC00E944C5DEE59F94F2083DB
:106182000E944C5DEE55F94F008351E00F5FD2CF74
:10619200503041F40E944C5D0E943D5A0E944C5D79
:1061A2000E94055C4F5FC2CF0E9422640C94F134BE
:1061B2000E941D64AC81BD81EBE4EC93EC81FD8116
:1061C20031960E944F5D0E944361E753FA4FE0818E
:1061D2000E94565D00E0AC81BD810E94D55BE0303B
:1061E20011F00F5FF8CF0E945C5DE0E2EC930F5F6D
:1061F2000E94625D0E944F5D0E94EE5BDF010E9481
:1062020037620E945A580E945F58EE81F0E00E9465
:10621200475D10811A930E947D1600E0AC81BD811A
:106222000E94D55BE03011F00F5FF8CF0E945C5DF9
:10623200E8E7EC930F5F0E945C5DE0E2EC930F5F96
:1062420030E03A3058F40E94625D0F010E94E0583B
:10625200EC91D001EC930F5F3F5FF3CF0E945C5D46
:10626200EC930E9424642796089564970E941D640B
:1062720000E010E0113050F40E9485570E94035A4A
:10628200E081EF3F09F40F5F1F5FF4CF013021F08F
:10629200A0914908A03009F406C0E0E0E093490863
:1062A200EA930E942C05013021F4A0914908A13003
:1062B20009F406C0E1E0E0934908EA930E942C0544
:1062C20010E0113038F50E9485570E94FB5931F0D9
:1062D200FD01E853FA4FE081E03009F419C01A9346
:1062E200FE013596FA93EA9363DF0E9485570E9476
:1062F200475D30813A930E947D161A93FE013596CE
:10630200FA93EA930E94A9050E9485570E942B5D89
:106312001F5FD7CF0E942464689608950E941D646F
:1063220030E0343168F4A2E7B7E00E94F958AAE4F9
:10633200B7E0EE27A30FBE1FEFEFEC933F5FF1CF65
:106342000E94571C0E2F0F3F11F40C94F1310E9442
:106352000C5A0E94D4561E2F1F3F31F0E0913A088A
:106362001E1710F0103408F036C0A0913A08E12F41
:10637200EA1B3E2F343130F5A2E7B7E00E947F5985
:106382000E94695DAC910E940457B0E0EA0FFB1FC6
:10639200D001EC930E94725DAC91A43620F00E9471
:1063A200725DE3E6EC93AAE4B7E0EE27A30FBE1F0B
:1063B200AC91AF3F39F4AAE4B7E00E947F59EA0FEB
:1063C200FB1F00831A930E940C5AFA93EA930E94CD
:1063D2003C161E2FC1CF0A930E945E1C0E2FB3CF14
:1063E20030E0343110F00C946F32A6E8B7E00E942E
:1063F200785DAF3F11F40C946D320E947D5D0E9476
:106402007D16A091BE0BA07849F40E94725D0C909B
:10641200AEE5B7E00E94835DE01509F45DC0A6E831
:10642200B7E0EE27A30FBE1F2C91ACE02A9FF0012C
:10643200E55FFC4F0F010E94725DEC91D001EC937D
:106442000E947D5D0E943C1EEF3F41F0ACE02A9F1E
:10645200F0010E94765AE058DB01EC930E94725DD3
:10646200EC91E030B1F0ACE02A9FF001E95FFC4F23
:10647200DF01E091BC0BE295EF70EC93ACE02A9F58
:10648200F001E85FFC4FDF01E091BC0BEF70EC9391
:106492000EC0ACE02A9FF001E85FFC4FA7E0A083AA
:1064A200ACE02A9FF001E95FFC4FA8E0A0830E94C4
:1064B2007D5D0E943C1EEF3F19F0ECE0E0935E0C24
:1064C200AEE5B7E00E947F590E94695DEC91D00170
:1064D200EC932A930E94ED553F5F83CF0E94246480
:1064E200CDC0E7E0E09334080E94C915A8950E9448
:1064F200591AA8950E94A01CA895EFEFE093D60B1D
:10650200E093AD0BE093530CE0934E0C0E942458A1
:10651200EE7FE03029F0A8E0B0E0E0E00E947B628C
:10652200E6E1FDE0FA93EA93E0EAEA93E0E1F0E0E3
:10653200FA93EA930E94E9510895E881E03021F448
:10654200E2ECF4E00E94885DA881A13021F4ECEB3A
:10655200F4E00E94885DA881A23021F4E8ECF4E026
:106562000E94885DA881A33021F4E6EDF4E00E9448
:10657200885DA881A43021F4ECEDF4E00E94885DEE
:10658200219608951A9310E00E948D5DE03039F053
:106592000E948D5DEA930E9456371F5FF5CF43C17B
:1065A2001A930A93E0E0E0936105E093620510E03C
:1065B200143190F400E0033068F4A3E01A9FF00174
:1065C200E859FA4FDF01EE27A00FBE1FE0E2EC937D
:1065D2000F5FF1CF1F5FECCF0991199108951A93C4
:1065E20011E0E981E11788F00E948557E255FF4FDB
:1065F200E491AA81EA2319F0E12FE05D01C0E0E213
:10660200EA930E9456371F5FECCF0DC10E94905D46
:106612000E94955DB7DF1AC10E94905D0E94B95D2C
:106622000E945F580E94C05D1DC10E94905DE6E914
:10663200F8E004C00E94905DEAE9F8E0FA93EA9378
:10664200EE850E94565D0E94C05D2B9608951A93B6
:106652000A9300E010E00E94C55DE03021F00832AC
:10666200E0E01E070CF008C00E94C55DEA930E949C
:1066720056370F5F1F4FEFCF198108812496089577
:106682001A930A9300E010E0F801AB81BC81AE0FCF
:10669200BF1FAC91A03021F0EA810E94CC5D0CF0CA
:1066A2000CC0F801AB81BC81AE0FBF1FEC91EA9325
:1066B2000E9456370F5F1F4FE7CF1BC10E941D6418
:1066C20010E0E1E3E0935309E89431F80E94D15DD0
:1066D200EEE9F8E00E94935600E0E09166050E179D
:1066E200D0F40E947C57E859FA4FE081E03248F436
:1066F2000E94D55D0E947C57E859FA4FE081E05D27
:1067020005C00E947C57E859FA4FE081EA930E9443
:10671200174D0F5FE2CF0E94D95D9F010E949A0838
:106722003A932A93E8ECF0E00E94275D0E2FA0E056
:1067320031FCA1E0A03011F4003009F001C0EECF2D
:1067420031FE0AC0E0E0E0936605E89431F8E1E04A
:106752000E9424640C9495381F5F123008F4B1CF64
:10676200E0E0E09366050E9424640C949538E09181
:106772006505E03021F4E881EA930E94C348A091C4
:106782006505A13021F4E881EA930E949C4BA09117
:106792006505A230F1F4E0916605F0E0E859FA4FA0
:1067A200A881A083E0916605EF5FE0936605E09122
:1067B2006705EF5FE0936705A03218F4EF5FE0939F
:1067C2006705A0916705A73321F478DFE0E0E09345
:1067D20067050C94F937A0916505A13039F4E8EC0E
:1067E200F0E00E946856E9E1E0939900A091650506
:1067F200A23021F463DFE0E0E0936705E0E0E0939C
:1068020065050895EDE0EA93B2DFEAE0EA93AFDFCF
:1068120008951A9310E0E9811E1728F4EA81EA9399
:10682200A6DF1F5FF8CF188123960895EDE201C01D
:10683200EDE3EA93E8E2EA93ECDFE4DF08950E94F5
:10684200905D0E94955DE0E0EA930ED02E96089549
:106852000E94905D0E94B95D0E945F58FE010E94F5
:10686200DD5D02D02C9608951A930A9310E0EA8116
:10687200E03011F408E201C00A81AB81BC81EE274D
:10688200A10FBE1FAC91A03011F0101708F007C085
:10689200AB81BC810E946C5A0E94E25DEECFEA811C
:1068A200E03039F0EA811E1720F4E0E20E94E25D56
:1068B200F9CF1FC01A930A9310E0EA81E03011F475
:1068C20008E201C00A810E94E75DE03011F0101772
:1068D20008F005C00E94E75D0E94E25DF4CFEA8104
:1068E200E03039F0EA811E1720F4E0E20E94E25D16
:1068F200F9CF1981088125960895E091AC05A09100
:10690200AB05EA17B9F0AFEAB5E0F0E00E94465AEB
:10691200EC91E093AE05E091AC050E94EF5DE18160
:10692200E093AD05A091AC050E94F25DE093AC0549
:10693200E1E008950C945538E091AB050E94EF5DBB
:10694200A981A083E091AB050E94EF5D3196A881F9
:10695200A083A091AB050E94F25DE093AB050C947D
:10696200B038E091C40508951A93E091C405E0306F
:1069720059F40E949A080E94175D21F4A091C4055F
:10698200A03009F001C0F5CF1091C405E0E0E0931A
:10699200C4050E94175D09F011E2E12F0C94C4377F
:1069A2000E941D640E94403F8F010E949A08EC8160
:1069B200FD81E00FF11FFF93EF930E94403FAF91E3
:1069C200BF91AE1BBF0B9D010024021603061CF4EF
:1069D2000E94175D09F001C0E8CFE0E00E94246444
:1069E200269608951A930E94F75DE050FD4FA0E0AD
:1069F200A0830E94F75DE65FFC4F108117FF09C07C
:106A0200E12FEF73A5E1EA9FF001E253FB4FA0E013
:106A1200A08316FF09C0E12FEF73ABE0EA9FF001FC
:106A2200EE50FC4FA0E0A0830E94F75DE65FFC4FB2
:106A3200A0E0A0830E94F75DE75FFC4FA0E0A08387
:106A42000C94AF380E941D6430E0EE81ACE0EA9F06
:106A5200F001E65FFC4F108116FF1AC0E12FEF73C1
:106A62000E2FAC81BD810E94785DA03011F03A30CA
:106A720008F00AC00E94FC5D0E947F590E94035EDA
:106A8200D001EC933F5FEDCF0E94FC5D0E94F9586C
:106A920017FF1AC0E12FEF730E2FAC81BD810E9448
:106AA200785DA03011F0343108F00AC00E94095E0E
:106AB2000E947F590E94035ED001EC933F5FEDCFAD
:106AC2000E94095E0E94F9580C94DD38A0970E943A
:106AD2001B64EDA5FEA5A9A9BAA9EA0FFB1FAF0188
:106AE200E0E0F3E0EE83FF8310E01431C0F5AE8105
:106AF200BF81AC91A03049F1EE81FF81A381B481C5
:106B0200EFA5F8A9EA17FB0701F5EE81FF81A18144
:106B1200B281E9A9FAA9AE17BF07BCF0EE81FF81E5
:106B2200A181B2814A175B0784F00E94105EAE0F0A
:106B3200BF1FE9A9FAA9AE17BF073CF00E94105E79
:106B4200AE0FBF1F4A175B070CF402C01A934ADF4D
:106B5200EE81FF813C96EE83FF831F5FC6CFE0E0AC
:106B6200F3E0EE83FF8310E0143110F00C945B36F7
:106B7200AE81BF81EC91E03011F00C945436EAA55D
:106B8200EC93E9A9FAA9AE81BF811196ED93FC932A
:106B9200EFA5F8A9AE81BF811396ED93FC93EDA505
:106BA200AE81BF811596EC93EBA5AE81BF8116969F
:106BB200EC93E091F003A0915E0CEA27AE81BF81D5
:106BC2001796EC93E0915F0CAE81BF811896EC931F
:106BD200E091600CAE81BF811996EC93AE81BF81CA
:106BE2001A96E0E0EC93AE81BF811B96EC93E887A6
:106BF200E8A5F9A5309751F00E94195EEAA5FBA518
:106C0200FA93EA93E4E1EA930E943D52EEA1FFA1D6
:106C1200309751F00E94195EE8A5F9A5FA93EA931C
:106C2200E4E1EA930E942952E0E0EC8F0E94195EAF
:106C32000E9414523E2F3B30C0F000E00E941E5EC4
:106C420011F0053008F002C00F5FF8CF0E941E5EFF
:106C520061F4A5E10A9FF001E253FB4F0E94265E18
:106C6200E058AE81BF811A96EC93E0E0EA8B3130B6
:106C7200C0F000E00E94315E11F0043108F002C061
:106C82000F5FF8CF0E94315E61F4ABE00A9FF00122
:106C9200EE50FC4F0E94265EE05CAE81BF811A96E8
:106CA200EC93E12F08C0EE81FF813C96EE83FF83D7
:106CB2001F5F5ACFEFEF0E942264E39608951A9362
:106CC2000A930E94395E3097A9F1E0913D05F09157
:106CD2003E05309769F50E94395E0E945062E0934A
:106CE2003D05F0933E05309731F4E0E0F0E00E947C
:106CF200885DE0E01AC00E943E5E0E94395E0E94FA
:106D02005062F595E7958F01D801E0E0F1E00E942D
:106D1200BE61E0938700D801E0E0F1E00E94F061FB
:106D2200E09386000E943E5EE0E4E0938B0002C0A6
:106D32000E94E5550C94093A0E941D6400E020E08F
:106D420033E010E01431A0F5D901EC91E03061F1AB
:106D520011960E9437620E94465E0CF5D901139685
:106D62000E943762AC81BD81EA17FB07C4F4F901C6
:106D720001801280D90115960E944B5EAE81BF81BF
:106D8200AE17BF0764F4F90103801480D901169687
:106D92000E944B5EAC81BD81AE17BF070CF004C0F0
:106DA200E12FEF5F0E2F04C0245F3F4F1F5FCACF5A
:106DB200003081F0E0914705F0914805A02FB0E046
:106DC200EA17FB0731F0A0914705B09148051097EB
:106DD20009F401C02BC00E949C55159791F40A93A7
:106DE200E1E0EA93A9DD0E947C57E0934705F09326
:106DF20048050E947C570E94505EE3E0F0E00E944A
:106E0200B1550E949C555E9721F4E4E0F0E00E94A7
:106E1200B155A0913B05B0913C05139734F0E5E0E4
:106E2200F0E0E0934505F093460508C00E94555EE8
:106E32000E944156E0E0F0E00E94505E0C94FE3861
:106E4200E0914705F09148053097A1F00E949C55CA
:106E5200999734F4E0914705EA93E2E0EA936CDD16
:106E62000E949C55DD9734F0E0914705EA93E4E0F7
:106E7200EA9362DD0E9441560E94555EE0E0F0E036
:106E8200E0934705F09348050E94505EE0E0F0E091
:106E9200E0934305F093440508950E94083880DB8F
:106EA200E5E1E093C30508953FC1F894E5B3E07EC0
:106EB200E1600E945C5EAFE3B5E00E94A155789468
:106EC2000E9450560E94176193C0F894E5B3E07E89
:106ED2000E945C5E78940E9450560E94176188C09E
:106EE200E8E3EA93F2DFE4E1F0E00E946856E8E3C7
:106EF2000E94685EECE00E94685EE1E00E94685ECB
:106F0200E6E00E94685EE0E80E94685E0895AA8159
:106F1200BB81E4E1F0E00E94F061EA83FB83A88197
:106F2200B981E2E0F0E00E94F061E883F9830E9417
:106F320045610E944161AA81BB81AE0FBF1FE0E89B
:106F4200F0E0EA2BFB2BEA93C0DFEA81FB81E093BE
:106F52003F05F0934005E881F981E0934105F09304
:106F62004205E2C01A9310913F050E946F5EA09104
:106F72003F05B09140055497C4F3E12F0E94F254AB
:106F82000E94A55CC4DF1991089532C0EA81E093A2
:106F92006305E881E0936405E091F103E061E09329
:106FA200F103C2C0A0916305A43120F4A09164054D
:106FB200A33008F01DC0E09163050E94F254E091F5
:106FC20064050E94F254A3DFE881E03071F0E091A1
:106FD2006305A3E0EA9FF001E859FA4FDF01E0916F
:106FE20064050E94FB5AEC9101C0E0E2EA935DDF86
:106FF20021960895E091F103E07141F0E2E0EA9315
:10700200D1DFE091F103EF7EE093F10308951A934B
:107012000E9428560E94135610E0143120F40E9458
:107022006F5E1F5FFACF0E9428560E9428566FDFBC
:1070320010E0143120F40E946F5E1F5FFACF0E94AD
:1070420028560E94285663DF0C94E93CE0DF08953D
:1070520086C00895E0E0E0937100E0937400E2B32B
:10706200E360E2BBE3EFE1BB85E38A95F1F7E0EF92
:10707200E1BBE4E4E093740080E991E00197F1F769
:1070820008951A9314EAE4EA0E94735E41F40E949E
:10709200785E183011F0103111F4E0E099C4E2E0AA
:1070A20097C4E4E9E0937400E0E008951A93E9815B
:1070B200E1600E947D5E31F40E94785E103411F42A
:1070C200E0E04CC04AC01A93E9810E947D5E31F42F
:1070D2000E94785E183111F4E0E040C03EC01A937D
:1070E200E9810E947D5E31F40E94785E183211F4CB
:1070F200E0E034C032C01A93E981E03011F0E4ECF0
:1071020001C0E4E80E94735E69F40E94785EE09137
:107112007300AA81BB81EC93103511F0183511F47C
:10712200E0E001C0E1E01881249608951A93E98114
:10713200E093740010E0E0917400E07811F41639E5
:1071420008F005C08BE18A95F1F71F5FF4CFE0915B
:107152007400E07811F0E0E001C0E1E018812296CD
:1071620008950E941D643D810C8120E08ADFE03099
:1071720009F5EE810E949F58E9F43A93B0DFE030BE
:10718200C9F40E94815EB1F47CDFE03099F4EE81B3
:10719200EA938CDFE03071F4EDB7FEB7FA93EA932D
:1071A2001F93E0E0EA93A7DF1F91E03019F479DF43
:1071B200E12F02C04FDFDACF0E94246427960895A0
:1071C2000E941D6430E00E811D815BDFE03099F486
:1071D200EF810E949F5879F40E94815E61F41A93B4
:1071E2007EDFE03041F4EC81EA9379DFE03019F49C
:1071F20058DFE0E002C02EDFE8CF0E942464289628
:10720200089522970E941B6450E02B853A85A89529
:1072120038DFE03011F00C946139EE850E949F58FE
:1072220011F00C9461392A935ADFE03011F00C947A
:1072320061393A9354DFE03011F00C94613921DF67
:10724200E030F1F5EE85EA9331DFE030C9F5E0E0B8
:10725200EE83EF83EC85FD8531970E94465E51F403
:10726200EDB7FEB7FA93EA931F93E0E0EA9343DFA8
:107272001F9109C0EDB7FEB7FA93EA931F93E1E0BD
:10728200EA9339DF1F910E2FEE81FF81A885B98520
:10729200EA0FFB1F10830E94865E003039F4EC85F2
:1072A200FD85AE81BF81AE17BF0708F001C0D2CF06
:1072B200EC85FD850E94465E19F4F3DEE0E002C033
:1072C200C9DEA6CF0E9422642F96089568970E9475
:1072D2001B6420E0E0E0EC8FED8F31E0A895E9A19E
:1072E200FAA1662777270E94F2620E94C655EE8DA8
:1072F2000E948C5E0E94D255EE81FF81688579855D
:10730200AA85BB858C859D850E94C863EA8BFB8B11
:107312006C8B7D8B0E945462FE017296FA93EA9303
:107322000E94BE54EE8BFF8B688F798F0E94925E13
:107332000E94B962AF010E94925EAE8DBB27882780
:1073420099270E945B620E94A55EDE015A960E9406
:10735200B962ED93FC930AA119A193DEE030E1F545
:10736200EDA10E949F58C1F50E94815EA9F51A9372
:10737200B6DEE03089F5303061F14F5F5F4FEC8D62
:10738200FD8D3196EC8FFD8FAC8DBD8D1197EBA1EC
:10739200FCA1EA17FB0711F430E01AC0EC8DFD8D59
:1073A2003197AF8DB8A1AE0FBF1FEC91EA9397DE74
:1073B200EE8DDA01F0E0EA17FB0751F472DEEA8D96
:1073C200FB8DA9A1BAA1EA0FFB1FE9A3FAA387CFFC
:1073D200D2CF67DEE0E002C03DDEBFCF0E94226472
:1073E200A69608950E94AA5E99F0E0E0E0935409FF
:1073F20010E000E00E9485570E94B05E49F00E94B2
:1074020085570E94B55E0E9485570E94B85EF2CFF2
:107412000991199108951A930A930091F30BAA8185
:10742200A53411F4E0E062C0AA81A23539F4A0913A
:107432005008A13019F40E948D5609F405C00E942B
:107442003D1AE0E0E0935008AA81AB3411F0A33575
:1074520099F4E02FE470E43011F414E001C013E079
:10746200E02FE270E23009F41C5FE02FE170E130BE
:1074720009F41F5FE12F3AC0AA81A13511F0A137AB
:1074820099F4E02FE470E43011F417E001C016E043
:10749200E02FE270E23009F41C5FE02FE170E1308E
:1074A20009F41F5FE12F22C0AA81A33441F413E043
:1074B200E02FE170E13009F41F5FE12F17C0AA81CC
:1074C200A73741F417E0E02FE170E13009F41F5FC4
:1074D200E12F0CC0AA81A03441F415E0E02FE17045
:1074E200E13009F41F5FE12F01C0EFEF198108813C
:1074F2002396089524970E941B64A0915B09A534EA
:1075020011F00C942C3BE0E0E09350080E948A5B5F
:10751200E0E0E093790BE091F70BE03081F5E09148
:107522002C08A0912D08EA1739F00E94BE5EED5298
:10753200F84FE081E13009F022C0E7E7EA930E94C8
:10754200174D0E94BE5EEA52F84FE0810E94F2544B
:107552000E94C45EEC52F84FDF010E9429580E943B
:10756200C45EE952F84FE0810E942D57E2E0E093B9
:1075720050080E94BE5EED52F84FA2E0A083E09157
:107582005008E03011F00C941E3B0E948D5611F40D
:107592000C940C3B0E94321AE1E0E0935008A09157
:1075A200F30BA87081F00E949E56E8EEF3E00E9471
:1075B200BE61DF010E94116414F4E1E301C0E0E363
:1075C200EA930E94174DE091440C0E94F2540E94EB
:1075D200CB5E0E94804DA091F30BA47059F00E94E3
:1075E2009E56E0E1F7E20E94F061FA93EA93E4E04A
:1075F200F0E008C00E949E560E94B15CFA93EA93A2
:10760200E3E0F0E0FA93EA930E94804D0E949756DD
:10761200E3E0F0E00EC018E0A091F30BA47009F0D3
:107622001F5FA091F30BA87009F01F5F0E942E55F7
:10763200F0E0FA93EA930E94804DA091F30BE1E00F
:10764200EA23E13029F4E091790BEA930E94174D85
:107652000E94955BC7DEA0915B09A73729F4E2E09F
:10766200E0935008E03009F47BC00E948A5BE2E5B7
:107672000E94AB5BB7DE0E944C5C1E2FE3E0EA93F4
:107682000E948F4CAF01E1E0EA930E948F4C0E2FD3
:10769200E0912C08A0912D08EA1739F00E94BE5EF5
:1076A200ED52F84FE081E23009F057C00E94BE5E11
:1076B200EC52F84FDF010E9437624E175F0711F05C
:1076C2000C94A73B0E94BE5EE852F84F00801180E6
:1076D2000E946C560E942A57EA17FB0779F10E9412
:1076E200BE5EE852F84FDF010E94D05E0E94BE5E8D
:1076F200E852F84FDF010E943762EA57F44F0E94C6
:10770200DA5E0E949B580E94DE5EE12F0E94F254D4
:107712000E947856E5EAF8E00E949356003029F07C
:107722005A934A930E94464D04C0E0E3EA930E94B2
:10773200174D0E94AE560E94A14E08C0003031F093
:107742000E94E25E18F40A930E94315CE0912D08D7
:10775200EA930E94842FE0932D08E0E0E093500822
:10776200A0915B09A33421F40E948F2FE03009F429
:107772000DC00E948A5BE2E50E94AB5B33DE0E9491
:10778200B9560E94285630D30E94F01AA0915B0984
:10779200A03421F40E948F2FE03009F425C00E940A
:1077A2004C5CE887F987E2E0EA930E948F4C1E2F37
:1077B2000E94F9560E94E2150E940E57EF5FF74FA2
:1077C2000E94E6560E940E57ED5FF74F10830E940B
:1077D2000E57E050F84FA7E00E9417570E948A5BAD
:1077E200E2E50E94AB5BFEDDA0915B09AB3439F0B0
:1077F200A33529F0A13519F0A13709F078C00E940C
:10780200D01A339724F00E948F2FE03009F469C018
:107812000E948A5B0E94E95EECE5F9E00E947158E1
:10782200A091F30BE2E0EA23E23029F4E4E0EA93E8
:107832000E948F4C02C0E1E0F0E0E887F987A09156
:107842005B09A13511F0A13731F4E3E0EA930E941C
:107852008F4C1E2F02C01091090CA091F30BE4E093
:10786200EA23E43011F4E4E001C0E3E0EA930E9489
:107872008F4CAF01A0915B09A33511F0A13731F410
:10788200E885F9850E942C61E887F9870E94E25E0B
:1078920020F0A091F70BA130C9F41A935A934A939E
:1078A200EB85FC85FA93EA930E940F1BEE83FF831C
:1078B200AF81AA235AF40E948A5BE6E6EA930E9409
:1078C200174D0E94865EAF81AA23BAF31A935A9388
:1078D2004A93EB85FC850E9420570E94955B82DDCE
:1078E20006C00E94B9560E9428560E940F1B0E9491
:1078F20022642A9608950E94ED5EE89422F80E947E
:107902009658E2E7EA930E94174DE0915608EA93EF
:107912000E94174DEFE0EA930E94174DA091530881
:10792200AA3221F41A930E94A90B1BC0A0915608F7
:107932000E948557EA57F44FE081EA1721F4E0915B
:107942005608E03351F40E942E58AA57B44FE091E2
:107952005608EC931A930E94A90B22FC02C00E94C3
:10796200A14E36C00E94ED5EE0915608E053AE2F64
:107972000E948557E956F44FE081EA1749F51A93B8
:107982000E94A90BA0915108A23019F40E94F55E41
:1079920009F402C00E94FB5EA0915108A33019F4C1
:1079A2000E94F55E09F402C00E94FB5EE0E0E093F3
:1079B2005108E093330D0E948557E956F44FBF01F9
:1079C200E081EF5FAE2FEAE00E94ED61DB01EC9314
:1079D200199108950E941D6425FC02C20E94F55E61
:1079E20011F40C943D3E0E942457E150F84F9F0140
:1079F200D9011196EC91E43071F50E94035F0E9467
:107A0200065F0E940D5FF901A481A03021F4A281DA
:107A1200B381109709F007C0E8EAF8E00E94935694
:107A22000E94AE5615C00E94DE5E0E94145F0E9444
:107A32007856EBEAF8E00E9493560E94195F0E9482
:107A42001F5FF901A681B781BA93AA930E94464D9E
:107A52000E94235FC5C1E730C9F40E94035F0E9400
:107A6200065F0E940D5FEEEAF8E00E9493560E94C4
:107A7200195F0E947856E1EBF8E00E9493560E944B
:107A8200145F0E94464D0E94235FAAC1E93099F417
:107A92000E94035F0E94065F0E940D5FE4EBF8E024
:107AA2000E949356D901EC910E94F2540E9478569A
:107AB2000E94235F95C1E63029F5EAE2EA930E942B
:107AC2008E4EE7EBF8E00E949356D901EC910E94AA
:107AD2002D57E091F10B0E942D57EBE4EA930E949F
:107AE200174D0E94145F0E94464DE4E5EA930E94FE
:107AF200174D0E94195F0E94464D0E94A14E0E949E
:107B0200FB5E6EC1E530E1F4D90116960E94D05EAB
:107B1200D901EC91EA930E94174D0E949B580E9452
:107B2200DE5E0E94145F0E947856E5EAF8E00E9449
:107B320093560E94195F0E94464D0E94235F50C1D6
:107B4200E830C1F40E94D15D0E94E95E0E942A5F82
:107B52000E949B58EAEBF8E00E949356D901EC91FF
:107B6200E0580E94F2540E9478560E942E5F0E94B2
:107B7200435F36C1EA30D9F40E94D15D0E94E95ECA
:107B82000E942A5F0E949B58EDEBF8E00E949356F8
:107B9200D901EC910E94F2540E941F5F0E94145F6F
:107BA2000E9478560E942E5F0E94435F19C1E13005
:107BB20011F00C941C3EA0913508A53029F4E091F7
:107BC200F10BE65F1E2F01C011E0E12FE05D0E9484
:107BD200485F0E948557E956F44FE0810E942D5775
:107BE2000E949B580E94DE5E0E94145F0E9478569B
:107BF200E0ECF8E00E9493560E94195F0E941F5F1A
:107C0200D9011596EC910E94F2540E94464DA09122
:107C12003508A53059F40E947857F901A085AA9336
:107C22000E947D160E9423560E9449580E94D95DE7
:107C32000E944C5FD5C0E330F9F4D90116960E9438
:107C42003762F0960E94485FD90116960E94376209
:107C5200E956F44FE0810E942D570E949B58E3ECB5
:107C6200F8E00E9493560E94195F0E94464D0E94BE
:107C7200D95D0E944C5FB4C00E948D5661F0A09104
:107C82005108A03041F4A091F60BA13021F40E94DA
:107C92006C56E13009F427C0A091A70BA03059F02F
:107CA200E091A90BF091AA0BFA93EA93E8EEF3E0C4
:107CB2000E94C55CC1F40E94D15D0E94E95E0E94EF
:107CC2002A5F0E949B580E946C56EA930E94630BA3
:107CD200E09351080E94D95DE093310DF093320D8B
:107CE200E0E0E093A70BA0915108A03059F0E09199
:107CF200310DF091320DFA93EA93E4E6F0E00E943E
:107D0200C55C09F02BC0A0915108A23019F40E9461
:107D1200F55E09F402C00E94FB5EA0915108A330F7
:107D220019F40E94F55E09F416C0A091330DA33038
:107D320030F00E94FB5EE0E0E093330D0CC00E9445
:107D42002457DF01E050F84FBF01FD01EF5FF74F0D
:107D5200E081DB01EC93E0E0E0935108A091A80BF5
:107D6200A130F1F5E091590CA091580CEA1799F164
:107D7200EAE20E94485FE091960B0E942D570E9412
:107D82009B58E091590CEA930E94641C0E94DE5EAB
:107D9200E091490C0E94F2540E947856E6ECF8E019
:107DA2000E9493560E940C5A0E944D580E94785786
:107DB2000E9404570E945B570E94A14EE091590C09
:107DC200EA930E94E71AE091590CEA930E94BA1AC8
:107DD200E093590C05C0E0E0E093A80B689420F80A
:107DE2000E942464249608950E948F2FE030E9F0C7
:107DF2000E940E57EF5FF74FAA81BB81A083B18328
:107E02000E940E57EB5FF74FA881B981A083B1831F
:107E12000E940E57ED5FF74FAC81A0830E940E5770
:107E2200E050F84FA4E00E9417570C94A542A88195
:107E3200A03310F0AA3308F004C0E881E0530C9498
:107E42002642A881A13410F0A73408F004C0E881CA
:107E5200E7530C942642EFEF0C942642A881AA30F5
:107E620020F4E881E05D0C942642A881AA3020F03B
:107E7200E881E95C0C942642E8E50C9426421A93C8
:107E82000A93F8940091840B1091850B7894F80171
:107E9200C8C21A930A93F3DF8F01EA81FB81AC8196
:107EA200BD81EA0FFB1FE01BF10BDF010E94116491
:107EB20024F4E0E019810881FFC2E1E01981088120
:107EC200FBC268970E941B64EAECF8E00E94DD5D49
:107ED2000E945B340E940334E0913E08E03061F07E
:107EE200E5EDF8E00E94DD5D0E945B34E0913E0822
:107EF2000E94F2540E94545F0E9403340E941E1892
:107F020030E03A3090F43A930E944355EFE0EA931E
:107F12000E943534E32F0E9453550E9457550E9408
:107F22005C550E94585F3F5FECCF0E941734EEED24
:107F3200F8E0FA93EA93EFE0EA930E945B340E943E
:107F420038550E94585F0E9419340E94033400E0A1
:107F5200003110F00C9460400E946C56E01711F052
:107F62000C94F43FE4EEF8E00E94DD5D0E945B3485
:107F7200E02F0E94F2540E94545FE0E0E0933A083E
:107F8200A0913A08A03458F5E0913E08EA93E091B6
:107F92003A08EA930E9464170E9469553097C9F023
:107FA200E0913A08EA930E947D160E946955FA937D
:107FB200EA930E945C5F0E945B340E940E56EAE0E4
:107FC200EA930E9435340E9472550E9454620E94C4
:107FD200585FE0913A08EF5FE0933A08D1CF0E94F0
:107FE20003340E9403340E947C570E94825911F08C
:107FF2000C945E40E4EEF8E00E94DD5D0E945B348A
:10800200E02F0E94F2540E94545F0E94615FE0E3FD
:108012000E948E5951F413E0EDB7FEB7FA93EA933A
:108022001F930E944E4E1F91AF01042E052A11F498
:108032000C945A401F5FEDB7FEB7FA93EA931F9371
:108042000E941A4E1F91EA8FFB8F6C8F7D8F1F5FEC
:10805200EDB7FEB7FA93EA931F930E94195E0E944E
:108062006D4E1F915A934A930E945C5F0E945B344B
:10807200FE013696FA93EA93EAE0EA930E943534D7
:10808200EA8DFB8D6C8D7D8D0E9454620E94585F3B
:108092000E94615FE1E30E948E5951F413E0EDB753
:1080A200FEB7FA93EA931F930E944E4E1F91AF01BF
:1080B200BCCF0E9403340E9403340F5F49CF0E9459
:1080C200EC330E9422646E9608950E941D64AC8176
:1080D200BD81EC91E1702E2F0E94695FE12F0E9419
:1080E200F254E02F0E94F2540E948837E4E0EA93AF
:1080F2000E94C637203019F4E1EFF8E002C0E6EF43
:10810200F8E0FA93EA930E9428330E94A05C349725
:108112000E946E5F0E94735F333409F431E20E9461
:10812200FB373D3311F0313209F402C0E1E02E2772
:108132003D3311F0313209F401C0D0CF3D3319F48F
:10814200AC81BD812C93E32F0E942464B5C10E94AF
:108152001D64AD81BE812C910E94695FE12F0E9456
:10816200F254E02F0E94F2540E948837ECE3EA9323
:108172000E945637EC81EA930E94C6372A93ED811A
:10818200EA930E94F032EEE3EA930E9456370E948D
:10819200795F0E94735F0E94FB37333409F431E246
:1081A200313320F0EC81E05DE31708F407C0E32FE0
:1081B2000E94B65CE255FF4FE4912E273D3311F049
:1081C200313209F401C0CACF3D3319F4AD81BE8109
:1081D2002C93E32F0E942464279608950E941B6427
:1081E20020E0AF81B8855C910E94695FE12F0E9417
:1081F200F254E02F0E94F2540E947C5F5A930E9434
:1082020016330E94795F0E94735F0E94FB373033FE
:1082120010F03A3308F00EC0203009F450E021E0AB
:10822200A52FEAE00E94ED61AAE0EA9FF001E30FC8
:10823200E0535E2F333429F4203009F431E250E068
:1082420020E03D3319F4EE81E51708F005C0AF8157
:10825200B8855C9130E020E03D3311F0313209F411
:1082620001C0C4CF3D3319F4AF81B8855C93BDC062
:108272000E941B6420E0AF81B8854D915C910E9401
:10828200695FE12F0E94F254E02F0E94F2540E9493
:108292002D56AE81A23021F4FA010E94205604C06C
:1082A2005A934A930E940D330E94795F0E94735F32
:1082B2000E94FB37303310F03A3308F020C02030F0
:1082C20011F440E050E021E04031E7E25E0734F093
:1082D200DA01E0E1F7E20E94F061AF01493BEBE035
:1082E2005E0724F0DA010E94B15CAF01DA010E945C
:1082F200825FDF01EE27A30FBE1FD097AD0133349B
:1083020031F4203009F431E240E050E020E03D3326
:1083120011F0313209F401C0B4CF3D3321F4AF8101
:10832200B8854D935C9361C00E941B640E94695F93
:1083320020E050E04FEFE12F0E94F254E02F0E9424
:10834200F2540E942D56EF81F885FA93EA93E8855C
:10835200EA930E944133E52FE10F0E94F254E02F8D
:108362000E94F2540E94735F0E94FB37303310F078
:108372003A3308F022C03053431729F04F3F09F037
:108382005F5F20E005C0A22FAF5FEA2FE3702E2FC0
:10839200E52FAF81B8850E94875F0F01E32FA2E826
:1083A200B6E0F0E00E944561AE0FBF1FE22F0E94CF
:1083B200875FE491D001EC93432F3B3219F4EE81B5
:1083C2005E1708F002C05F5F4FEF3D3211F451308B
:1083D20008F402C051504FEFEE815E1720F43132A3
:1083E20011F03D3309F401C0A6CFE32F0E942264AD
:1083F200299608951A930A93A091BE0BECEDEA23F5
:108402001E2F00E00B3040F40E94D4573A96E491BC
:10841200E11711F00F5FF6CF0E94D4570E94345536
:10842200E02F099119910895AEEBBBE0E8810E941B
:10843200FB5AEC91E17019F4EBEFF8E002C0EFEFB8
:10844200F8E0FA93EA930E942833219608950E9455
:108452001B640E94695FE12F0E94F254E02F0E9488
:10846200F2540E942D56C6DF5E2F0E94795F0E9451
:10847200735F0E94FB37303310F03A3308F013C0B9
:108482005F5F5B3008F050E0A091BE0BE1E0EA23B1
:108492002E2FACE05A9FF001E053FC4F3A96E49144
:1084A200E20FE093BE0B3D3311F0313209F401C00B
:1084B200D2CFE32F0E942264269608950E941D6463
:1084C2000E94695FE12F0E94F254E02F0E94F25451
:1084D2000E942D56EC81EA93A7DF0E94795F0E94E9
:1084E200735F0E94FB37303310F03A3308F012C04A
:1084F200AEEBBBE00E94D458EA0FFB1F0F01AEEBBC
:10850200BBE00E94D458AE0FBF1FAC91E1E0EA2756
:10851200D001EC933D3311F0313209F401C0D2CFD6
:10852200A091BE0BE2E0EA232E2FE091BF0BED7F7C
:10853200E22BE093BF0BE091C00BED7FE22BE093C7
:10854200C00BE32F0E942464259608950E948B5F3E
:108552000E94A7050E9428560E9428560E9488372A
:108562000E940E56EAE0EA93DFDEE13209F42BC301
:108572000E9428560E9428560E942D56E3E0F9E0F8
:108582000E943455E9EBFBE00E94DD5D71DEE132D1
:1085920009F419C30E9428560E9428560E942D569B
:1085A200E9E0F9E00E943455EBEBFBE0FA93EA9341
:1085B200EAE00E948F5F09F406C30E9428560E94D7
:1085C20028560E942D56E2E1F9E00E943455E0ED72
:1085D200FBE00E94945F09F4F6C20E9428560E94B2
:1085E20028560E942D56E8E1F9E00E943455E2ED4A
:1085F200FBE00E94945F09F4E6C20E9428560E94A2
:1086020028560E942D56EEE1F9E00E943455EDEB1A
:10861200FBE0FA93EA93E3E60E948F5F09F4D3C288
:108622000E9428560E9428560E942D56E7E2F9E041
:108632000E9434550CDFE13209F4C5C210E0133058
:1086420010F00C94B2430E9428560E9428560E94B1
:108652002D56E12F0E94565CEDE2F9E00E9434555E
:108662000E944E550E9428560E948837A1ECBBE01A
:108672000E9485570E949C5F09F4A5C2E9E0F0E0E0
:10868200FA93EA930E9428560E948837A4ECBBE032
:108692000E9485570E949C5F09F495C20E94285649
:1086A2000E9428560E942D56E12F0E94565CE8E354
:1086B200F9E00E9434551A9301DFE13209F483C2D2
:1086C2000E944E550E9428560E948837AEEBBBE0AE
:1086D2000E946C5AE17049F40E94A1590E941358F9
:1086E2000E94945F09F46FC20AC00E94A1590E94BD
:1086F20013580E94DD5DBCDDE13209F464C20E94C0
:1087020028560E9428560E942D56E12F0E94565C40
:10871200EAE3F9E00E9434550E944E550E94285621
:108722000E948837ADECBBE0EE27A10FBE1F2C9153
:108732003327EDB7FEB73197FA93EA933F932F931E
:10874200E0E0EA9395DD2F913F91E13209F43BC2DB
:10875200ADECBBE00E948557EA0FFB1F20831F5F31
:108762006ECF31C20E941D6410E01A930E947D16E2
:108772000E9408380E949D050E9428560E94285691
:108782000E94A25F0E940E560E944A550E945558AE
:108792000E946E550E9428560E9413560E9423562C
:1087A2000E942056E7E0F0E0FA93EA930E94135603
:1087B200E091D20BF091D30B0E9420560E942856D2
:1087C2000E94CB5E0E948837E1E4F9E00E943455B2
:1087D200E091BB0BEA930E941633E7E0F0E0FA93D4
:1087E200EA930E94CB5E0E94883704DE0E946F5E8D
:1087F20000E00330D0F50E942856E02FED5F0E9482
:10880200F2540E9488370E94B35BEA930E941633A7
:10881200EBE2EA930E9456370E94BA5BEA930E9407
:10882200AD5F0E94C15B41F40E94DA5B0E9419565F
:108832000E942056E3E707C00E94DA5B0E941956A5
:108842000E946E55E9E4EA930E9456370E946F5ED9
:10885200ADECBBE00E94D55BEA930E941B33E3E7D9
:10886200EA930E9456370F5FC4CF0E94B5343E2F61
:108872003B3211F4103408F001C01F5F3D3211F495
:10888200113008F401C011503D3439F41A930E949A
:108892007D165CDE1A930E94A716313209F065CF6D
:1088A20092C10E941D6410E00E940838012F0E94AC
:1088B20028560E9428560E948837E5E4F9E00E9473
:1088C200345531E03C3028F5103808F50E9428561E
:1088D200E32F0E94F2540E9488371A930E94F116E5
:1088E200E12FEF5FEA930E94AD5FA091540CE1E0AB
:1088F2000E94B05FA091550CE7E00E94B05FE0914A
:10890200E105EA93E8E0EA930E94F03213953F5FB3
:10891200D9CF0E949D050E94B5343E2F3D3411F0FF
:108922000C94D2440E948A5C102F1038D0F51A930E
:108932000E94F1160E9428560E9428560E942D5627
:10894200E9E5F9E00E9434550E94B55F0E94625940
:108952000E9428560E948837ECE5F9E00E943455BF
:10896200E4E5FCE0FA93EA93E1E00E948F5F09F408
:108972002AC10E9462590E9428560E942D56E2E6A0
:10898200F9E00E943455E5E5FCE0FA93EA93E7E06A
:108992000E948F5F09F417C11A930E9425171F5F67
:1089A200C4CF313211F0103808F001C07DCF0BC1B5
:1089B2000E948B5F0E949D050E9428560E942856A5
:1089C2000E948837E8E6F9E00E94345510E0103141
:1089D200E8F41A930E9431170E942E55EF5F0E940D
:1089E200F2540E94A25FE0914F0C0E94BE5FE091A0
:1089F200520C0E94BE5FE091500C0E94BE5FE0915B
:108A0200510CEA930E941B331F5FE1CF0E94B534E1
:108A12000E2F0D34A1F50E948A5C10E0103178F51A
:108A22001A930E9431170E9428560E9428560E94CB
:108A32002D56EBE7F9E00E9434550E94B55F30E015
:108A42003430C0F40E9462590E9428560E942D566A
:108A5200A6E13A9FF001E65DF94F0E943455A6E186
:108A62003A9FF001E65DF94F0E94C25F09F4ABC084
:108A72003F5FE6CF1A930E944E171F5FCFCFA3C06E
:108A82000E948B5F0E94A70500E0033210F00C9455
:108A9200E4450E9427380E9428560E9428560E94C8
:108AA20088370E94CC5F31960E9434550E946F5ED7
:108AB2000E94CC5F0E94C557A9F40E946C561E2FDB
:108AC200EDB7FEB7FA93EA931F93E0E1EA9386DBF0
:108AD2001F91E13209F477C0E12FA9E0B0E00E94D2
:108AE2007B626DC0E138A0E0FA07D1F40E942458FD
:108AF2001E2FEDB7FEB7FA93EA931F93E6DA1F91A2
:108B0200E13209F460C00E9427380E942458E1171C
:108B120031F0E12FA8E0B0E00E947B62FFCF4FC0AE
:108B2200309749F40E94CC5F0E94D25FCEDAE132E4
:108B320009F449C044C0E130A0E0FA0739F40E94C8
:108B4200CC5F0E94C25F09F43EC039C0E230A0E0AF
:108B5200FA0769F40E94CC5FDF010E94D25FFD0137
:108B62007296E491EA9384DBE13269F128C0E33042
:108B7200A0E0FA0769F40E94CC5FDF010E94D25F95
:108B8200FD017296E491EA93E2DAE132E1F017C074
:108B9200E430A0E0FA0799F40E94CC5F3E960E946E
:108BA2005062E093340DF093350DFA93EA930E94EC
:108BB200CC5F7296E491EA93B7DBE13221F00E9436
:108BC200CC150F5F62CF0E942464249608950E9400
:108BD2008A5C0E9428560E9428560E948837EEE737
:108BE200F9E00E943455E1E0E0933E08EEE3F8E05C
:108BF200FA93EA93E5E0EA93F1DA089522970E9464
:108C02001B640E94B5340E2FE0913708E03011F05A
:108C12000C94AF470132D1F4E6EFF4E0A0915A0C84
:108C2200B0915B0CEA17FB0761F4E7E0E0933408CC
:108C3200EAE2EA93E7E8F9E00E94DD5D0E94DA4E9B
:108C4200DFC1E0E0E093A4050E94D85F0D3319F480
:108C52000E94105504910D3441F4EAE2EA93EAE8E5
:108C6200F9E00E94DD5D0E94DA4E063449F4ECEA36
:108C7200F5E0E0935A0CF0935B0CE0E0E093A4057E
:108C8200003311F00B3229F4E091A405EF5FE09379
:108C9200A4050D3229F4E091A405E150E093A40566
:108CA200013329F494DFED3311F40E94DF5F0333C3
:108CB20021F48DDFED3309F404D9063321F4E0E029
:108CC200E0933E08FED8043329F4E0E0E0933E0846
:108CD2000E94DF5F093411F40E941A05A091400836
:108CE200A13010F40C942347023301F570DFED3309
:108CF200E9F40E94EC5FD1F4E0913E08EA930E940D
:108D0200BE1830E0303190F40E947F590E9482599F
:108D120059F4E32FE05DEA93EDE8F9E00E94875908
:108D2200E0E3EA930E94FD4E3F5FECCF053331F55D
:108D3200E0E0E0933E080E94EC5F01F511E016309E
:108D4200E8F41A930E94BE1830E03031A8F40E9471
:108D52007F590E94825971F4E32FE05DEA93EDE8B6
:108D6200F9E0FA93EA93E12FE05DEA93E0E3EA9314
:108D72000E94FD4E3F5FE9CF1F5FE1CF013451F406
:108D8200EAE2EA93E0E9F9E00E940D5DE1E0E093B6
:108D9200340836C1073311F00C9423470E94083877
:108DA2000E949305E1E0E0933808E0E0F0E0E09310
:108DB2003008F093310830E0303130F40E947F59AE
:108DC2000E94E05A3F5FF8CF0E94403FEE83FF834C
:108DD2000E94F55FEEE1F0E00E94275DE03031F0A5
:108DE2000E9434090E94403FEE83FF830E94555641
:108DF2000E94D13440E050E000914B05003089F0F0
:108E0200E02F0E94715AE050FD4FE081EF573E2F54
:108E1200313010F0313108F004C0E32F0E94315696
:108E2200AF014093300850933108E02F0E94715AED
:108E3200E050FD4FE081E13259F6E0E0E09338087E
:108E4200E093C405A0914008A23011F00C94A84709
:108E5200093309F415DE053409F4AADD033611F4E9
:108E62000E941B05083309F47DDC073421F4A0912C
:108E7200080CA33009F01BC0E1E0E093830B0E94D1
:108E82000838E091830BE03091F0E4E6F0E0FA93E9
:108E9200EA930E94D1340E94CB5E0E94CB5E0E9474
:108EA2007C5FE091830BEA930E941633EACF02348F
:108EB20009F4F7DC0334B1F51091590C0E9408381B
:108EC20000E0E091580CE11711F00C3008F01DC0E1
:108ED2000E942856E02F0E94F2540E9488371A936B
:108EE2000E94641C1A930E94AD5FE091490C0E949B
:108EF200BE5FE0914C0C0E94BE5F0E940C5A0E9421
:108F02006E550E94F6590395DCCF0E949D050E9482
:108F1200B5340E2F013221F0E091580CE11709F41B
:108F220001C0CCCF043499F40E94EC5F81F4A0918B
:108F3200F70BA03021F4A091F50BA03031F00E9484
:108F4200B9560E9428560E94F53E0E94F01AE091FE
:108F52003708E03011F40E9496054DC0E130B9F4B3
:108F6200A0913D08AB3010F4013209F405C00E9413
:108F7200B1050E949D050AC0E0E0E0933A080E9414
:108F8200FA5F0E940360E2E0E093370834C0E23007
:108F920091F5013269F4E0E0E09337080E94083865
:108FA200EAE2EA93EAE8F9E00E940D5D0E94960582
:108FB2000B3281F4E0913A08EA5FE0933A08A0911B
:108FC2003A08A03418F0EAE3E0933A080E94FA5F04
:108FD2000E9403600D3279F4A0913A08AC3020F07F
:108FE200E0913A08E65001C0E0E0E0933A080E94BE
:108FF200FA5F0E940360A0913408A33009F401CE05
:109002000E942264289608951A93E3E0E0933508BB
:109012000E942455E6E9F9E00E9434550E94285640
:109022000E94135610E0103140F40E948557E3531A
:10903200FA4FA0E0A0831F5FF6CF10E0E091ED0BA6
:109042001E17E0F4E12FE05DEA93EEE9F9E0FA930E
:10905200EA93E0E3EA93E0E00E948E5949F40E9429
:109062008557E353FA4FA1E0A083E12FE05D01C0F1
:10907200EEE2EA930E9456371F5FE0CF0E94D85F6C
:10908200E0E0E093A405E09337080E94960534C21D
:10909200AC81A03310F0AA3308F006C00E940A6027
:1090A200E0530E94126057C4AC81A13410F0A7347F
:1090B20008F006C00E940A60E7530E9412604BC487
:1090C200A881B981E0E0EC9346C4AA93EA93FA93AB
:1090D200EFB7EA931A930A931BB10CB1E091700DAA
:1090E200F0E0E25CF24F0083A091700DAF5FA093BD
:1090F200700DA23319F4E0E0E093700D099119911B
:1091020014C31A93E091710DA091700DEA17D1F377
:10911200F0E0E25CF24F1081A091710DAF5FA0937D
:10912200710DA23319F4E0E0E093710DE4C1E09116
:10913200710DA091700DEA1709F0A1C3A2C30E949C
:10914200D7550E941C6049F0A0915409A03021F02B
:109152000E941C05E13009F401C006C00E94226091
:1091620019F4E0E0E093D70DE991EFBFF991E991AD
:10917200B991A9919991899179916991F9901990EF
:10918200099018951A930E941C6059F45D9B09C0BE
:10919200A0915409A13021F40E941C05E03009F08D
:1091A20013C01091D60D0E948557EE58F24FA98137
:1091B200A0831F5F143609F410E0E091D70DE11788
:1091C200E1F31093D60D02C0E981ECB995C40E9477
:1091D2001C6021F40E941C05E13009F001C04FC35C
:1091E20050C30E941C6061F05D9B0AC0A0915409AB
:1091F200A13021F40E941C05E13009F001C001C038
:1092020006C00E94226019F4E0E0E093D70D0895B1
:109212000E941D648CDFE03011F40C94354A71DF3A
:109222001E2FA091390DA53618F0E0E0E093550904
:1092320030915509E0915509E03011F00C946149E3
:10924200A091080CA13021F0A091080CA23041F4A9
:10925200E12FEF77E0935B09EBE4E0935A09FCC05E
:10926200A091080CA33011F41E3709F002C0EEE100
:10927200F1C01A3511F4E1E0EDC0123021F4E4E15D
:109282000E943060E9C01A930E940C3AE093570999
:10929200A0915709AF3F99F010935B09E1E0E09389
:1092A200560910935809E0915709E03011F4E5E4AA
:1092B20004C0EAE0E0935509E0E0E0935A09CCC02B
:1092C200E13069F4103039F4E2E0E0935509E0E06E
:1092D200E0935A0903C0E0E0E0935509BDC0E230D3
:1092E20049F41093570910935809E0E0E0935609A6
:1092F200E3E0B0C0E330E9F40E9438600E943E60CF
:109302000E944860A9F4E0915809E03071F4E4E069
:10931200E0935509E09156090E940E590E9452604D
:109322000E943860A0E0A08303C0E0E0E09355090A
:1093320093C0E43031F41D3019F4EAE5E0935A09A0
:1093420088C0EA30A9F40E9438600E943E60EA2791
:10935200E0935809E0915709E150E0935709E03052
:1093620031F4E0E0E0935509E5E4E0935A0974C072
:10937200E431B9F40E9438601083E12FA0915809BA
:10938200EA27E0935809E0915609EF5FE093560906
:10939200E0E0E093380D133019F4E5E1E09355096C
:1093A2005BC0E53111F0E63159F41A93E8E3FDE0D0
:1093B200FA93EA93E5E5F9E0FA93EA9369DE4CC0A1
:1093C200E73181F4E0E0E0935509173131F4E0919F
:1093D200380DA0915809EA1709F003C0E3E4E093BD
:1093E2005A093AC0EE3141F4103011F4EFE101C0F4
:1093F200E0E0E093550930C0EF3149F4E0E0E0935A
:109402005A0910935709E0E20E94306025C0E03209
:1094120059F40E9438600E943E600E94486019F42C
:10942200E1E2E093550918C0E132B1F4A091580984
:10943200EFEFEA1B1E1769F40E943860A0E0A083D8
:10944200E0915609F0E0E45AF64FA083E8E5E09394
:109452005A09E0E0E0935509A09155093A1719F02D
:10946200E0E0E093390DD6CE55C2AA93BA93EA93BF
:10947200FA93EFB7EA931A930A9310919B00009123
:109482009C00E12FEC71A9F4E091A00EF091A10EE5
:10949200E852F24F0083A0EABEE00E94A155E83CE8
:1094A200A0E0FA0731F4E0E0F0E0E093A00EF093E0
:1094B200A10E09911991E991EFBFF991E991B99141
:1094C200A99118951A930E9457600E945C60D9F383
:1094D2000E945760E852F24F1081A2EABEE00E9459
:1094E200A155E83CA0E0FA0731F4E0E0F0E0E093B7
:1094F200A20EF093A30EE12F199108950E945760D6
:109502000E945C6009F0BBC1BCC10E941D64F6DF11
:10951200E03021F0A091370DA03009F0E5C0D2DF94
:109522001E2FA091AC0EA53618F0E0E0E093A60E37
:109532003091A60EE091A60EE03059F4113019F4E4
:10954200E4E0E093A60E1A3519F4EAE0E093A60EE1
:10955200C3C0E430C1F4E0E0E093A60E1A3229F071
:109562000E946C56E05DE11769F410935308109362
:10957200A70EE5E0E093A60EE0E0E093370DE1E010
:10958200E093A90EA9C0E530A9F4E0E0E093A60EAD
:109592000E946C56E05DE11761F00E9463600E94D8
:1095A2006C60E091A90EEF5FE093A90EE6E0E09314
:1095B200A60E92C0E63091F4E091A90E0E946C6072
:1095C2000E946360EF5FE093A90EE0E0E093AA0ED1
:1095D200133019F4E7E0E093A60E7EC0E73011F0F5
:1095E200E83059F41A93EAEAFEE0FA93EA93E6EADB
:1095F200FEE0FA93EA934CDD6FC0E93081F4E0E0DB
:10960200E093A60E173131F4E091AA0EA091A70EB5
:10961200EA1709F003C0E4E5E093370D5DC0EA30D4
:1096220041F4103011F4EBE001C0E0E0E093A60E4B
:1096320053C0EB3071F4E0E0E093A90E1093A80E52
:109642001093A70EECE0E093A60EE0E0E093370D56
:1096520043C0EC30A1F5E091A90EF0E0E55AF64FD7
:1096620010830E946360EF5FE093A90EE091A80E61
:10967200E150E093A80EA091A80EA03021F4A09191
:10968200A70EA03009F00EC0EDE0E093A60EE09127
:10969200A90E0E940E590E945260E091A90EF0E0BC
:1096A2000E945260A091A80EA03021F4A091A70EB2
:1096B200A03009F403C0E0E0E093A60E0DC0ED3047
:1096C20059F4E0E0E093A60E1D3031F4EAE5E093B0
:1096D200370DEFEFE093360DE091A60EE31719F088
:1096E200E0E0E093AC0E13CF15C1AA93EA93FA938C
:1096F200EFB7EA93E091AE0FA091AD0FEA1791F0A8
:10970200E0915208E03019F0E89426F80AC00E946D
:109712007160F0E0E030A1E0FA0719F4E0E0E093D4
:10972200AE0F03C0E89425F826F8E991EFBFF9914E
:10973200E991A99118951A93E091AE0FA091AD0FFE
:10974200EA1721F4E0919B00E072C1F4E091AD0FC1
:10975200F0E0E355F14FA981A0831091AD0F1F5F97
:109762000E942E58A030E1E0BE0709F410E0E0911B
:10977200AE0FE117E1F31093AD0F03C0E981E0935F
:109782009C00BAC1E0E0E093AE0FA091AD0FA13012
:1097920020F00E947160689426F80895AA93BA9303
:1097A200EA93EFB7EA93E0E0E093AE0F0E946C56C3
:1097B200EF5FE0935208E991EFBFE991B991A99166
:1097C20018950E947E56A03220F00E947E56AB333E
:1097D20009F403C00E948A56F4CF0E947E56AB332E
:1097E20011F40E948A5608950E947E56E881EA1773
:1097F20029F40E948A563197E1E001C0E0E0219607
:1098020008950E947F60EEE20E94B55701F520E0C4
:1098120030E0EC81D901F0E0AE17BF07C4F4D80103
:109822000E94825F8F010E947E56A03320F00E9428
:109832007E56AA3308F008C00E9484560E94B65C85
:109842000E0F1F1F0E948A562F5F3F4FE2CFF80173
:1098520080C00E947E56A03228F00E947658E18194
:10986200E03208F40EC00E948456E0935D0B0E9421
:109872008A560E948456E0935E0B0E948A56E1E06B
:109882000895E0E008951A930A9310E00E94845824
:109892000C910B3311F0003208F412C0013310F0B6
:1098A200093308F007C0E02F0E94B65CE255FF4F73
:1098B200E4911E2B0E948A560E9484580C91E9CF93
:1098C200E12F8EC30E947F600E947E56AD3229F442
:1098D2000E948A562FEF3FEF02C021E030E00E9443
:1098E2007E56A03320F00E947E56AA3308F00EC0A6
:1098F200D8010E94825F0F010E9484560E94B65CCA
:10990200E00DF11D8F010E948A56E9CFF901D801BD
:109912000E9493610E942464249608950E941D640B
:1099220020E030E000E010E0EC810E94CC5D84F4A5
:10993200D9010E94825F0F010E9484560E94B65C88
:10994200E00DF11D9F010E948A560F5F1F4FECCF61
:10995200F9010E942464259608950E947F6020E008
:1099620030E00E947E56A03320F00E947E56AA3339
:1099720008F018C0AC81A13058F0D8010E94825F73
:109982000F010E9484560E94B65CE00DF11D8F010A
:1099920031E0213018F0AC81A13008F403C0EC8131
:1099A200E150EC830E947E56AE3211F422E031E0A7
:1099B200313011F40E948A56313091F2AC81A130DB
:1099C20040F0D8010E94825F8F01EC81E150EC836C
:1099D200F5CFF8010E9424640C94F5511A9310E01B
:1099E2000E943157E030E9F00E947E56A03258F0D2
:1099F2000E947E56A23239F00E947E56AB3319F095
:109A0200E9811E1708F00DC00E948557E15AF44FF4
:109A12000F010E948456D001EC931F5F0E948A5668
:109A2200E3CF0E9485570E94B05766C0E8810E942A
:109A32007E58E881A091780BEA0FE093780BE881D9
:109A4200A091790BEA27E093790B0C9455521A9363
:109A520010E00E948460E491E03031F00E94846062
:109A6200E4910E948860F5CFE1C01A9310E00E9451
:109A720085570E948D6041F00E948557E15AF44F4C
:109A82000E94DA5E1F5FF3CFE9C20E94C057E2EA8A
:109A9200F9E0FA93EA93EC81FD810E945A580E9400
:109AA2005F58E3DF2AC01A930E94C057E5EAF9E043
:109AB200FA93EA93ED81FE810E945A580E945F5800
:109AC200D4DFB4C01A93ECE3EA93B0DF11E01930AB
:109AD20080F40E948557E255FF4FE491A981EA2361
:109AE20019F0E12FE05D01C0E0E2EA939FDF1F5F22
:109AF200EECFEEE3EA939ADF1881229608951A9345
:109B02000E94C057EAEAF9E0FA93EA93EF81F885F6
:109B12000E945A580E945F5810E00E948557E15AED
:109B2200F44FE081E03241F40E948557E15AF44F4C
:109B3200A0E3A0831F5FF1CFA981BA81EAE0F0E040
:109B4200EA1B1E2F0E9485570E948D6041F00E94E1
:109B52008557E15AF44F0E94DA5E1F5FF3CF1881F6
:109B62000C94F5510E94905DE2EAF9E0FA93EA93CF
:109B7200EE85FF85688979890E9454620E945F5848
:109B820074DF0E94AE562E9608951A93E2E2EA938B
:109B92004DDF10E00E948D5DE03029F00E948D5D66
:109BA2000E948860F7CFE2E2EA9340DF3FC01A9357
:109BB20010E00E948D5DE03029F00E948D5D0E94D0
:109BC2008860F7CF33C01A930E94C057EFEAF9E0DA
:109BD200FA93EA93AD81BE81E4E6F0E00E94BE61B1
:109BE2000E945A58A985BA85E4E6F0E00E94F06125
:109BF2000E945A5888E00E943F542C9610E00E941E
:109C020085570E948D6091F00E948557E15AF44F6A
:109C1200E081E03211F4E0E305C00E948557E15A89
:109C2200F44FE081EA9302DF1F5FE9CF18812396A8
:109C3200089524971A93E0E0E983EA83EB83EC83A7
:109C42000E949260103310F01A3308F01FC0A981ED
:109C5200BA818B819C81EAE0F0E060E070E00E94D2
:109C62009861DF01CB01E12FE053FF2766277727B9
:109C72000E942761E983FA836B837C83AD81BE8175
:109C8200EC91EF5FEC930E949260DCCFE981FA8164
:109C92006B817C8118810C947C520E947F600E94AF
:109CA2009A60303310F03A3308F012C0D8010E94A3
:109CB200825FDF01E32F0E94B65CEA0FFB1F8F0178
:109CC200AC81BD81EC91EF5FEC930E949A60E9CF89
:109CD200F8010E9424648EC01A9310E00E94A260D0
:109CE200E03210F0EB3708F010C00E9484600F01E0
:109CF2000E94A260D001EC93AB81BC81EC91EF5F3A
:109D0200EC931A3008F41F5FE9CFA981BA810E944F
:109D1200AD59E12F18810C94F551EDEAFEE0E09384
:109D22007A0BF0937B0B0E94915BE0E0E093780B5F
:109D32000E94AA600E946C560E942D570C945552A4
:109D42001A930A93E091360DE03009F049C1E3E03D
:109D5200EA936CDEE091780BE295EF70EA930E9451
:109D62002F3F1E2FE091780BEF70EA930E942F3F56
:109D72000E2F1A935BDE0A9359DEE7E1EA9356DE71
:109D8200EDEAFEE00E94AE600E946462EA1BE0938C
:109D9200AD0F689425F824C1EE81EA93BEDFEC8111
:109DA200FD810E9493560E94B360DCDEC9DF0C94F1
:109DB2007C52EB81EA93B1DFE981FA810E949356EA
:109DC2000E94AA60BDDF0C94BC54ED81EA93A5DF2A
:109DD200EB81FC810E949356EA81EA9327DEE981B6
:109DE200E03011F0EA9322DEE881E03011F00E94C7
:109DF200AA60A6DF269608950E941B6410E0E6EB97
:109E0200F9E0A885B985EA17FB0719F444E150E0A7
:109E120002C048EC50E0EA85E0935309E89431F837
:109E2200EA93E985FA85FA93EA93EA85EA93EA8561
:109E3200EA93E0E0EA93C9DF0E94403F9F010E945B
:109E42009A083A932A935A934A930E944A3F0E2FB2
:109E520031FC02C0003009F001C0F1CF31FE04C074
:109E6200E89431F8E1E004C01F5F1230A0F2E0E0B4
:109E72000E9422642B9608950E94AA5E09F4B0C043
:109E8200E0E0E0935409E2E0EA937CD910E003E0D9
:109E92000E9485570E94B05E61F00E9485570E9421
:109EA200B55E0E948557E55AF54FE0810E271F5F88
:109EB200EFCFE3E0EA9366D9E02FE295EF700E94DC
:109EC200BA60E02FEF700E94BA60E7E1EA935AD9D4
:109ED20087C00E941B64EBE5FAE00E94AE60AE1BF5
:109EE200BF0B9D01EEE70E94C0602A934BD950E060
:109EF20000E010E00217130784F4ABE5BAE0A00F0C
:109F0200B11FEC91EA933ED9ABE5BAE0A00FB11FC5
:109F1200EC915E0F0F5F1F4FEDCFEFEFE51BEA9362
:109F220031D90E9422640C94EA540E94AA5E09F478
:109F320057C0E0E0E0935409EAE50E94C06010E0F7
:109F42000E9485570E94B05E11F01F5FF9CF1F5F1C
:109F5200012F0A9317D910E00E9485570E94B05E24
:109F620049F00E9485570E94B55E0E9485570E9463
:109F7200B85EF2CFE02FE195EA9304D9EDE0EA93DF
:109F820001D92EC00E94AA5E59F1EAE5EA93D3DB19
:109F9200E0E0EA93D0DB10E00E9485570E94B05EB9
:109FA20011F01F5FF9CF1F5F012F0A93C4DB10E08E
:109FB2000E9485570E94B05E61F00E948557E55A63
:109FC200F54FE081EA93B7DB0E9485570E94B85EA5
:109FD200EFCFE02FE195EA93AEDBEDE0EA93ABDB66
:109FE2000991199108951A93E0915D09EA9395DE1A
:109FF200EAE5EA931BDDE0915B09EA9317DD13E0E2
:10A002000E948557E55AF64FE081E03041F00E9408
:10A012008557E55AF64F0E94DA5E1F5FF1CF90DE58
:10A022001DC00E946958E09156080E94A45BE0910D
:10A032005408EA93FBDC14E00E948557ED5AF74F6F
:10A04200E081E43040F00E948557ED5AF74F0E94BC
:10A05200DA5E1F5FF1CF0E94955B67DF1991089569
:10A062000E941B640E948A5B0E94915B0E94955B26
:10A072000E94995B0E94915B00917A0B10917B0B7D
:10A082000E94955B0E94955B0E94E95EE2E1E0938B
:10A09200780BE4E4EA93CADCE8E3EA93C7DCA09134
:10A0A200830BA13051F40E94D55DECE4EA93BEDC4F
:10A0B200E1E3EA93BBDC0E94AE56A091830BA2308F
:10A0C20010F0A23408F038C0E0E5EA93AFDC0E9459
:10A0D200D55DE091830BE1500E94F2540E947856C4
:10A0E200E0E5EA93A3DCEEE4EA93A0DCE091830BE3
:10A0F200E250EA930E947D1640E04A3078F40E94D2
:10A102004C5DE15AF44F0F01AEEABBE0EE27A40F1B
:10A11200BE1FEC91D001EC934F5FEFCF0E943158FC
:10A1220034DD0E94AE56E0E50E94A45BE091C70BCD
:10A13200F091C80B0E945B57A091830BA23438F0B8
:10A142000E94D55DE4E5EA9371DC0E94AE560E945E
:10A15200AE60A01BB10BE1E0F0E00E946462EA1B7A
:10A162005E2FE52FA091780BEA0FE093780BE19533
:10A172000E94F25498DC20917A0B30917B0B009371
:10A182007A0B10937B0BE52F0E94F2548CDC209308
:10A192007A0B30937B0B9DDE0E9422640C94EA546E
:10A1A20037D8E0915A09E030B9F1A0915A09AA359D
:10A1B20041F4A0915609A33020F0E0915C09E43407
:10A1C20009F00FC00E946C56E05DA0915D09EA178C
:10A1D20021F40E94DA14A9DE04C005DFEAE5E09367
:10A1E2005909A0915A09A53411F40E947B3AA09111
:10A1F2005A09A33411F40E945428A0915A09AB348D
:10A2020011F40E944D28A0915A09A83511F40E9418
:10A212009828E0E0E0935A09A091080CA33011F0CD
:10A222000C949751E0917E0BE03019F40E94C760C4
:10A232007AC0E13011F00C9468510E94CE600E9405
:10A242004A3FE030A1F1E2E0E0937E0B0E94C7605A
:10A25200E0917F0BEF5FE0937F0BA0917F0BA03229
:10A2620010F0A13718F0E0E2E0937F0B0E948A5BC6
:10A272000E94915BE0917F0BEA93D8DBEFEFEA93C8
:10A28200D5DBEFEFEA93D2DB0E94915B0E94915BF8
:10A29200E0E4EA93CBDB0E94E95EEAE2EA93C6DB02
:10A2A200E6E3EA93C3DB0E94D55D13DE3FC0E09193
:10A2B200830BE03059F0E3E0E0937E0B0E94403FD5
:10A2C200E0933C0DF0933D0DCBDE30C02FC0E23069
:10A2D200E1F40E94CE600E944A3FE030A9F0E0E043
:10A2E200E0937E0BE091800BEF5FE093800BA091F7
:10A2F200800BA33049F49698EAE0F0E00E94685699
:10A30200969AE0E0E093800B11C0E33079F4E0919B
:10A312003C0DF0913D0DFA93EA930E94115C0E946C
:10A322004A3FE03019F0E1E0E0937E0B37C0EDD810
:10A33200A091370DA43529F4A0E025FCA1E0A030BE
:10A3420009F022C0E0915508EA3519F40E944E1531
:10A3520018C0EA3711F465DE14C0E23519F40E9420
:10A362007C3C0FC0E23719F40E94B33C0AC00E9441
:10A372004A2CE0915408A0915309EA1711F4689409
:10A3820031F8E0E0E093370DA091370DAA3531F4B2
:10A392000E94DA14F7DDE0E0E093370DE0E0089583
:10A3A200A0E025FCA1E0A13049F4A0E026FCA1E058
:10A3B200A03021F4A0915208A03009F001C0E2D9E6
:10A3C200E0915208E03019F0E150E093520808950C
:10A3D200B981A881109631F0FC81EB816A81619389
:10A3E2001197E9F7EB81FC8125960895E991F9919E
:10A3F200A991B9911D900590011421F40020D1F783
:10A40200EE2708951018E1F3E1E008F4E250089510
:10A41200E991F991A991B991CD0161916D93662369
:10A42200E1F7FC010895A991B991EE27FF276D91FB
:10A43200662311F03196FBCF0895AA27BB27E99135
:10A44200F9910590002011F01196FBCFFD010895BE
:10A452007991E991F991A991B991CD01772351F0BF
:10A462007A9561916D936623C9F7772319F07A95EE
:10A472006D93FBCFFC0108956991E991F991A9913E
:10A48200B991CD01662351F06A9505900D92002095
:10A49200C9F7662319F06A950D92FBCFFC01089566
:10A4A2005D9BFECFE881ECB9219608951A930A9339
:10A4B200AC81BD810E9437623097C1F0AA81BB8115
:10A4C2000E9437628F01309749F00230E0E01E07A8
:10A4D20060F0F80131978F01ED93FC93AC81BD815F
:10A4E2000E94A1553197AE81A08303C0EE81EA9309
:10A4F200D7DF19810881279608952C970E941B6443
:10A5020010E0E88DF98D3196E88FF98F3197E4915B
:10A512002E2FE03011F40C943B54E12FE03039F44B
:10A52200253211F411E002C00E94D560A2C1E130CF
:10A53200C1F4253219F40E94D5609AC112E0E0E01C
:10A54200E98B00E02D3211F401E093C12B3219F4B2
:10A55200EBE2E98B8EC1203219F4E0E2E98B89C18A
:10A5620002C0E23039F450E013E0203311F4006805
:10A5720080C102C0E330A1F4203310F02A3308F086
:10A5820009C0A52FEAE0EA9FF0015E2FE22FE05317
:10A592005E0F6FC140E02E3211F414E06AC110C0A8
:10A5A200E430A1F4203310F02A3308F009C0A42FBC
:10A5B200EAE0EA9FF0014E2FE22FE0534E0F59C11D
:10A5C2002C3619F4026015E054C104C0E53011F0D4
:10A5D2000C943A54E22FE33649F40E94E060EE898B
:10A5E200FF89A481AA930E94E66042C1E33741F445
:10A5F2000E94E0600E94F0600E9414521E2F0AC066
:10A60200E037A1F40E94E0600E94F0600E941E52B6
:10A612001E2F08600F77403011F0411708F001C07B
:10A62200142F40E0E0E0E88B30E078C0E43611F02F
:10A63200E93611F4046002C0E537A1F4EAE0E88BE0
:10A6420001FF08C0E0E0FAEC6AE97BE30E94F860EF
:10A652001AE023C0E0E1F7E260E070E00E94F860F7
:10A6620015E01BC0E83511F4086004C0E83711F0AA
:10A672000C943954E0E1E88B01FF08C0E0E0F0E01F
:10A6820060E070E10E94F86018E007C0E0E0F0E1ED
:10A6920060E070E00E94F86014E0403011F00F7743
:10A6A20001C041E001FF08C00E94E060AE89BF899D
:10A6B20014960E943B6215C002FF0AC00E94E0602D
:10A6C200AE89BF8914960E9437620E94556109C003
:10A6D2000E94E060AE89BF8914960E9437626627A5
:10A6E2007727EC87FD876E877F8702FF16C0AF85CD
:10A6F200AA2362F4EC85FD856E857F850E94306118
:10A70200EC87FD876E877F87EDE2E98BE989E03090
:10A7120019F01F5F4F5F01C00B7F342F00FD14C083
:10A72200151710F4351708F00FC007FF08C002FF15
:10A7320004C00B7F2989115001C020E301C020E22F
:10A742000E94D5605150ECCF1417B0F4006102FFA3
:10A752000AC00B7FE989EA930E94E660503009F053
:10A76200515011504150E0E3EA930E94E6605030AC
:10A7720009F051504150E8CF312FE889E030B9F467
:10A782003030A1F003FF05C00E94865E3197E4914C
:10A7920005C0AE81BF81ED91AE83BF83EA930E9473
:10A7A200E660503009F051503150EACF57C00E9454
:10A7B200FD600E94C3612E2F2A3030F003FF02C0D9
:10A7C200295C01C0295A01C0205D04FD25C0213346
:10A7D20060F4A885B9858A859B85A130E0E0BE0733
:10A7E200E0E08E07E0E09E0709F40BC0431740F457
:10A7F200531710F000FF01C014C020E207FF0CC085
:10A8020020E3006102FF08C00B7FE989EA930E94FE
:10A81200E660503009F051500E94D560503009F086
:10A82200515031500E94FD600E94FE61EC87FD870D
:10A832006E877F87E889A885B9858A859B85FF27EA
:10A84200662777270E94C3610E94F860E885F98530
:10A852006A857B850E940D6409F0A9CF00FF08C0BC
:10A86200503031F05150E0E2EA930E94E660F8CFB6
:10A8720010E047CE0E9422646A960895FF92F82E55
:10A8820022971A930A93DE010E9423618D01DE0151
:10A8920016960E9423610E943762EA83FB83DE01DF
:10A8A20014960E9423610E9429581A930A93FE016A
:10A8B2003696FA93EA930E9428561FDEAA81BB813C
:10A8C200E0E0EC93198108812496FF9008957B8142
:10A8D2006A81F981E88177FB770F67FD7160972FB5
:10A8E2009E5781F078F0983190F4AA27BB278827E9
:10A8F20008948795B795A7959A95D1F7EA23FB23F4
:10A90200682305C0E8947727EE27FF2766276F772D
:10A91200769508F4606877F9A991B991899199912E
:10A92200EA17FB076807790797FB08950E94B3604F
:10A932000E94066119F40E940D611DC0E6F7A8810C
:10A94200B9818A819B81E0E0F0E060E87FE30E94C8
:10A95200A55E11C00E94B3600E94066119F40E94B4
:10A962000D6109C0E6F30E940D61A0E0B0E080E84D
:10A972009FE30E942C63249608950E9412610E9414
:10A982000D6439F4A881B9810E9471590E9446620E
:10A9920020C0AA81BB818C819D810E94156434F400
:10A9A2000E9412610E945462C1DF05C00E941261BE
:10A9B2000E945462CFDFA881B9810E944662A881B9
:10A9C200B9810E943B62AA81BB818C819D810E94D8
:10A9D200A55E26960895ACE01A9FF001E050FD4F67
:10A9E2000895F0E0FA93EA930895ECE0F0E0FA9328
:10A9F200EA930895EA93E0E0F0E0FA93EA93FA9397
:10AA0200EA930C9467350E9430050E940838E0E012
:10AA1200F0E0FA93EA93FA93EA930C948837E09180
:10AA2200A405F0E0A0915A0CB0915B0CBD01AEE020
:10AA3200B0E00E946B61E60FF71F0895E881F9818B
:10AA4200FA93EA9308950E940838E0E0F0E0FA935E
:10AA5200EA93FA93EA930C948837E0E0F0E0FA93F1
:10AA6200EA93E12F0895FA93EA930C942833E09144
:10AA72004508F091460860914708709148080E9485
:10AA8200546208950E94B816E7EDFBE0FA93EA9348
:10AA92000895EAE0EA930C944133E6E0F0E0FA9399
:10AAA200EA930895A2EDB6E0F0E008950E944561B0
:10AAB200AE0FBF1F08950E943B620E945462089528
:10AAC200EA930E947D16EEEAFBE0FA93EA93E1CF65
:10AAD200E0913E0CF0913F0C0895FA93EA930C94A6
:10AAE2000D33E091400CF091410C6091420C709159
:10AAF200430C08950E9454620C940733E09151056F
:10AB0200F09152050895E0914D05F0914E0508959A
:10AB1200AE0FBF1FE3E0F0E00E94BE610895FA931A
:10AB2200EA931A930A930C943806FA93EA933A93A7
:10AB32002A930C943806A0914905B0914A050895CC
:10AB4200ED91FD913196FE93EE930895A0915505F6
:10AB5200B09156050895A0915705B09158050895F2
:10AB6200E0933B05F0933C050895E093A705F0932D
:10AB7200A8056093A9057093AA0508950E946462CE
:10AB8200EA1BFB0B0E9455610895EA87FB876C87DD
:10AB92007D8708950E946B62DF01F001EA1BFB0BC7
:10ABA2000895EE83FF836887798708950A921A923F
:10ABB200FA926A937A938A939A93AA93BA93EA93AC
:10ABC200FA93EFB7EA930895ADE3B5E0ED91FD9105
:10ABD2003197FE93EE930895E1E0EA930C942938BD
:10ABE200E2E0EA930C942938E0914B05F0914C0590
:10ABF2003197ACE0B0E00E946B61E050FD4FE08124
:10AC02000895E0E0F0E0FA93EA93E1E0F0E0FA93ED
:10AC1200EA930E9488370C94B337EEEAFBE0FA938A
:10AC2200EA930895E1E0F0E0FA93EA930C9488370E
:10AC3200EE0FFF1FAE0FBF1F0E94376208950E94E2
:10AC4200556158CFE091D00BF091D10B0895E0E01F
:10AC5200F0E0FA93EA9308950E9488370C94B33790
:10AC6200ACE8B0E0F0E0EE0FFF1FEA0FFB1F0E941E
:10AC720050620895E12FF0E0EE51FA4FE08108951D
:10AC8200E0E0F0E06DCFECE2F1E0FA93EA930C94AD
:10AC92001761E4EFF1E0FA93EA930C941761E1E0B3
:10ACA200F0E0FA93EA930895E5E0F0E0FA93EA938C
:10ACB2000895E1E0EA930E942405E2E3F0E0FA93CA
:10ACC200EA930E941761E0E0EA930C942405FA9358
:10ACD200EA930C941761A9E0B0E00E946F620895B4
:10ACE2000E94464DECE2EA930E94174DA7CE0E94C5
:10ACF200464DEBE3EA930C94174DA0917C0BB09177
:10AD02007D0BAC910895A0917C0BB0917D0BEC91E1
:10AD12000895ACE7BBE014CFE091570CA091560C1C
:10AD2200EA170895FA93EA930C94284DE091470CA0
:10AD3200F091480CFA93EA930895A091450CB091D2
:10AD4200460C0895F0E0A4E6B0E00E9493610895F5
:10AD5200E093450CF093460C0895EBE3EA930C94D0
:10AD6200174DA0917A0BB0917B0BE0E0EC93089524
:10AD7200E0E0EA936CCFEE81FF81E093470CF09321
:10AD8200480C1093440C0E94201AE1E3089541E01C
:10AD920050E00E94634CE887F987EAE3EA930E9455
:10ADA200F54BE1300895FA93EA930C942B161A931B
:10ADB200E985FA85FA93EA935A934A930895E091C2
:10ADC2002C08A9E0EA9FF0010895A885B985A0831F
:10ADD200B1830895DF01EA85F0E0ED93FC930895D5
:10ADE200E0912C08EA930E94842FE0932C080895A6
:10ADF2001A93E985FA85FA93EA930895A0914C0C87
:10AE0200B0914D0C0895E0914C0CF0914D0C0895C9
:10AE1200E0934C0CF0934D0C0895E0912E08A9E0BC
:10AE2200EA9FF0010895EA85F0E00895A083E09199
:10AE32002E08EA930E94842FE0932E080895FA9335
:10AE4200EA930C94F53EE0912F08A9E0EA9FF00105
:10AE52000895D001F0E00895E05DEA930C94174D57
:10AE6200E2E2EA930C94F54B0E94634CE058FF4FE8
:10AE72001E2F0895E32FF0E0EE52F94F0895ACED46
:10AE8200B6E0EE27A30FBE1F0895E32FF0E0EE50C9
:10AE9200FA4F08950E94464DEAE3EA930E94174D45
:10AEA200E32F0895A2E2B6E0F0E00895A2E4B6E04E
:10AEB200F0E00895FA93EA931ACFA0E0B0E0A083FD
:10AEC200B183E0E00895EAE3EA930E94F54BE130B2
:10AED20008950E94464DECE2EA930C94174DACEDB6
:10AEE200B6E0E32FF0E0EA0FFB1F0F01C8CFEAE361
:10AEF200EA930C94174DE02FF0E00895EFEFE09302
:10AF0200730BE093740B0895E12FF0E008950E9413
:10AF1200634C3197E0935B0BE091740BA0915B0B58
:10AF2200EA1708950E94FC0EE0915B0BEA930895E4
:10AF3200E0915B0BE093740B0895E0915B0BF0E002
:10AF4200EE52F94F0895ECE2EA930E94F54BE0309D
:10AF52000895A7EDBBE0EE27A10FBE1F0895E15AA9
:10AF6200F44FA0E0A0830895EA930E94F54BE130EC
:10AF72000895A6E11A9FF001E854FF4F0895EFE506
:10AF8200FBE0FA93EA93089570960E945062E038CB
:10AF9200A0E0FA07089572960E945062A02FB0E0D6
:10AFA200AE17BF070895ACE00A9FF001E053FC4FD3
:10AFB2000895A1ECBBE0E0915C0BF0E00895A4ECF5
:10AFC200BBE0E0915C0BF0E00895E0915C0BEF5F79
:10AFD200E0935C0B0895ADECBBE0E0915C0BF0E01C
:10AFE2000895A7ECBBE0E0915C0BF0E0EE0FFF1FD1
:10AFF200EA0FFB1F0895AEEBBBE0E0915C0BF0E0C3
:10B002000895AE0FBF1FEC91E160D001EC9308955B
:10B01200AEEABBE0EE27A10FBE1F0895E0915C0BE4
:10B02200F0E00895EE0FFF1FEA0FFB1F0895FA9359
:10B03200EA930C940C0BE0915B0BA6E1EA9FF00102
:10B04200E854FF4F0895A8E0B0E00E946F620895AF
:10B052000E943762FA93EA930895A12FB0E008950F
:10B06200E0E0E093690B8BCFECE2EA930C94174D8E
:10B07200E091BC0BE295EF70B4CC0E94464DEFE834
:10B08200F7E050CE0E94010BE0E0E0935C0B0895E4
:10B09200FA93EA930C94E44DFA93EA930C94464D96
:10B0A200AE0FBF1FEC919DCCE091B90BF091BA0BA2
:10B0B20008950E9455610E945462089584E00E949E
:10B0C2003F5428960895A091540CE1E0EA2389CCDC
:10B0D2001A93EBE5FAE0E0937A0BF0937B0B089579
:10B0E200E0937C0BF0937D0B0895E0917C0BF09143
:10B0F2007D0B0895AAE7BBE023CDA0917A0BB09116
:10B102007B0BEC93F7CFA0917C0BB0917D0B089554
:10B11200A0917A0BB0917B0B13970895E0E0EA932C
:10B122000E94630BE09350080895E0915408EA935B
:10B132000C948E4EEEE0EA930C94174DEA930E9423
:10B142006438E0300895E0EAEA93EAE5F0E0FA9341
:10B15200EA93E0E0FFE0FA93EA93E2EEFBE008957F
:10B16200FA93EA93E0E2EA930C946739E0EAEA930D
:10B17200E981FA81E050FE4EFA93EA930895EA815A
:10B18200F0E0A8E2B0E00E9493610895E0EAEA9359
:10B19200E2E0F0E0FA93EA931A930A930895FA939D
:10B1A200EA930C940239EC81F0E00895E0EAEA9324
:10B1B200E8E2F0E0FA93EA931A930A932ECDAEEA0C
:10B1C200BBE0EE27A30FBE1F0895ABE0B0E00E94E4
:10B1D2009361E050F24F8F010895E0EAEA93EBE0C9
:10B1E200F0E0FA93EA931A930A93E6EDFBE00895EE
:10B1F200EE27A30FBE1FEC9308951A930A93EA81D8
:10B20200F0E00895EA81F0E00895EE0FFF1FE050AC
:10B21200F04F8F01AA81A0380895E150F0E008951F
:10B222000E944561E058F14F8F01AA81A031089533
:10B23200E0EAEA93E4E0F0E0FA93EA931A930A93DD
:10B24200EFE4FCE00895E093500CE0E0E093510C51
:10B25200E093520C0895E0E0F0E0E0933E0CF093AE
:10B262003F0CE0E0F0E060E070E0E093400CF0932F
:10B27200410C6093420C7093430C08950E94456107
:10B282000E944161DF01CFCDAE0FBF1FE8E0F0E0C9
:10B292000E949361E050FA4E8F01E0EAEA93E8E0FF
:10B2A200F0E0FA93EA931A930A93ECE3FCE077CF87
:10B2B200E093400CF093410C6093420C7093430C6A
:10B2C2000895E8E0F0E0FA93EA930895E0914308E4
:10B2D200F0914408E093470CF093480C0C94201A28
:10B2E200E0E0F0E060E070E00895E0934508F0935C
:10B2F200460860934708709348080895E32FF0E0EA
:10B302000895E353FA4FE081E1300895FA93EA9306
:10B31200E0913E08E05DEA930895EA930E94FD4EB3
:10B32200E1300895A981AF5FEAE00E949D61E05D8E
:10B332000895A981AF5FEAE00E94ED61E05D0895A2
:10B34200A7ECBBE0E1CDEE0FFF1FAE0FBF1FE0E0A9
:10B35200F0E0ED93FC930895EE27A10FBE1FEC934E
:10B362000895EA930E94563710E008957496E49186
:10B37200D901EC930895E881F0E0A5E0B0E00E94E5
:10B3820093610895E0EAEA938FCCEA930E94151A3A
:10B39200FA93EA93E4E4FCE008950E946462EA1BF3
:10B3A200FB0B0895EFEFE093490CEFEFFFEF30CD89
:10B3B200EFEFFFEFE0934A0CF0934B0C0895A0914E
:10B3C2004A0CB0914B0C0895E0E0E093580CE093E6
:10B3D200590C0895A88DB98DEA0FFB1F0895E0E07E
:10B3E200E093490C1A930C94721C1A930E94BA1A95
:10B3F2001E2F08950E944361DF01EA53FA4FE08154
:10B40200E03008950E944361EB53FA4F08951A9376
:10B412000E94641CF3CCE0914A0CF0914B0C08950D
:10B42200E881EA930E94BA1AE8830895EB81EA93CD
:10B432000E94E11AFA93EA93E9E4FCE008951A9370
:10B442000A93A09135080895E0E0E093B50CE093EB
:10B45200B40C0895A0913208B0913308EA2BFB2B6B
:10B46200E0933208F09333080895E12FA6EBBCE095
:10B47200F0E00895F0E0D6CDEE59F94FAFEFA0839A
:10B482000895A2EBB6E0F0E00895EE0FFF1FAE0FB5
:10B49200BF1F0895EE52F94FA0E0A0830895AEE0D9
:10B4A200B7E032CDBD01A6E0B0E00E946B61DB01E6
:10B4B200AE0FBF1F20CD0E94931D0E94D71DE2EF49
:10B4C200F5E0FA93EA93E0E0EA93E0E1F0E0FA9340
:10B4D200EA930C94E951EE27A10FBE1FEC91089557
:10B4E200E150ACE0EA9FF0010895E55FFC4FBF0137
:10B4F200E0810895D901E2E0F0E00E94BE619F017F
:10B502000895EE52F94FE081E0300895A0EFB6E0E1
:10B51200FBCCBD01A3E0B0E00E946B61DB01AE0F8A
:10B52200BF1FEE27A00FBE1FEC930895A1EEB6E059
:10B53200EBCCBD01A3E0B0E00E946B610895BD01B8
:10B54200A6E0B0E00E946B61DB010895EA5EF24F73
:10B552000081E12FA1E0B0E00E943861E887F9871D
:10B56200E423F52330970895E150F84FEE83FF83EB
:10B57200AE81BF811196EAE0EC93E12FEF5FAE81DD
:10B58200BF81EC9314960895EC93E0912E08EA9310
:10B592000E94842FE0932E080895E081EA930C9490
:10B5A200541DEE5FF94FE08138CEEE51FA4FE08143
:10B5B200F0E0EA0FFB1FD001ED93FC930895EE51EA
:10B5C200FA4FA0E0A0830895A0914B05B0914C05DD
:10B5D20010970895AEEBBBE0E0913608F0E00895D5
:10B5E200A1ECBBE0E0913608F0E0AE0FBF1FEC919A
:10B5F200EA930895F0E0AE0FBF1F0895A2E5B7E009
:10B602007DCEF0E0EA0FFB1FD001ED93FC937CCCE2
:10B61200A1EEB6E070CCE60FF71FE40FF51FE08154
:10B622000895AEE0B7E067CCAE0FBF1FFA0100CBC2
:10B63200ACEDB6E0EE27A00FBE1FEC910895ED91A0
:10B64200FD913197FE93EE930895A0EFB6E053CCAF
:10B65200E12FA6EDBCE0F0E018CFEE52F94FE08109
:10B66200EA93E3E0EA930C949D34A6EDBCE0F0E0AB
:10B672006ACEE60FF71FE40FF51F8FCFAFEFB6E0EC
:10B682003ACCEA930E948C1DE0300895ACE2B7E018
:10B6920032CCE60FF71FDF0131960F01FD01E18188
:10B6A2000895E60FF71FDF0132960F01FD01E281D7
:10B6B2000895E150F84FEE83FF83AE81BF8111966A
:10B6C2000895DB01AE0FBF1FEC9108951696F0E0CE
:10B6D200ED93FC9308951296F0E0ED93FC93089598
:10B6E200E0912E08EA930E94842FE0932E08089599
:10B6F200E12FA2E8B6E0F0E09BCAE12FA2E8B6E0B3
:10B70200F0E0C3CEE3E0E093280DE0E00E94226483
:10B712000895EBE5FAE0E0937A0BF0937B0B089542
:10B72200E1E0EA930C94174DE0E0EA930C94174D94
:10B73200E091820BEA930E94174DE091810BEA930C
:10B742000E94174DEDCFEA930E94174DE4E4EA936D
:10B752000C94174DEA930E94174DE6CFDB01AE0F12
:10B76200BF1FC9CBA1ECBBE0EE27A00FBE1FEC911F
:10B772000895A4ECBBE0EE27A00FBE1FEC91089544
:10B78200AEEBBBE0EE27A00FBE1FEC91E170089577
:10B79200EA0FFB1FCF01F001DB01AE0FBF1FEE2747
:10B7A200A00FBE1FEC910895EE27A00FBE1FEC91D3
:10B7B2000895A7ECBBE09FCBDF01E60FF71F0F0157
:10B7C200FD017FCFEA81ACE0EA9FF001E75FFC4F29
:10B7D200A0E0A083EA81EA9308950E944361E553C1
:10B7E200FA4F0895AFEFBFEFA083B18308950A9394
:10B7F200FE013596FA93EA930C94D930FE01359600
:10B80200FA93EA930C942335EE55F94FAFEFA083E8
:10B812000895E0912E0DF0912F0DFA93EA93089579
:10B82200E4EFF1E0FA93EA9308950E94403FE09337
:10B832002E0DF0932F0D0895FA93EA93E0E0F0E1D4
:10B84200FA93EA930C942D05FA93EA93E091290D69
:10B852000895E150F84FFA93EA930E94032740CFEC
:10B86200E091AE05EA930C94F923E0914308F0913C
:10B872004408FA93EA930895E0E0E0932B0DE1E3A4
:10B88200E0932C0D0E94F2270C94A0230E94174DE6
:10B89200E0E8EA930895ECE5F9E022DCE3E0EA93DC
:10B8A2000C948F4CE0935D0CD2C9EF5CEA930C943C
:10B8B2005637A2E5B7E028CBA7ECBBE0E09136080B
:10B8C200D9CDE7E0E0933408EA9352CAEA930E94A2
:10B8D2009E320E94B5341E2F0895EAE2EA93E2E313
:10B8E200F8E0FA93EA93E0E0EA930C94DA4E0E94CD
:10B8F2003F29E1E0EA930C941829E05DEA930C9465
:10B90200DA4E1F771A930E947D16E091BD0BE0304C
:10B9120008950E9408380C94A705E0E0F0E0E09357
:10B922004108F0934208E2E00895E091610CE5508D
:10B932000C94F254E0914108F0914208CEC8E09193
:10B942003F05F09140050895E0914105F0914205CF
:10B95200FA93EA930895A0914108B091420808959C
:10B96200E8EEF3E00E94F0610895E053F0E00895FC
:10B97200A0E024FCA1E0A0300895E0914E08F091EF
:10B982004F08FA93EA930895FA93EA930E944A3F82
:10B99200E13008950E94403FE0934E08F0934F0833
:10B9A2000895E0E0E093B40C0895D5DFEA17FB07B1
:10B9B2000895E0934308F09344080895E09334080F
:10B9C200E0E0E0934C080895E0913508EA93E0E066
:10B9D200EA930E94552A0E94BE260E94B234E030A9
:10B9E20008950E94B5341E2F1A930E94CA2A103855
:10B9F2000895E091AE05EA930E945F1EEF3F08951D
:10BA02000A93E091AE05EA930C942D27E091570832
:10BA1200E053E0933E080895FA93EA93E0E3EA9351
:10BA22000C94DA4EE081EA930C94C348E091350815
:10BA3200A0913408EA170895E89423F8E0E0F0E0D2
:10BA4200B8DF0A93E1E0EA930C94552AFA93EA9359
:10BA52000C944A3F0E944361E853FA4FA0E0A0834E
:10BA620008950E944361EA53FA4FA0E0A08308952B
:10BA72000E944361E853FA4FA1E0A08308950E9417
:10BA82004361EA53FA4FA1E0A08308950E94436103
:10BA9200E653FA4F0895E42FF0E00895FA93EA93FB
:10BAA200E8E7F8E0FA93EA93BEC9FF27662777270B
:10BAB2000E94546203CBAC81BD81EE27A00FBE1F52
:10BAC2000895E02FAC81BD81F0E0EA0FFB1F0895DD
:10BAD200EA0FFB1F0F01A2E7B7E0EE27A30FBE1F7D
:10BAE2000895A2E7B7E0EE27A30FBE1F0895EE2741
:10BAF200A30FBE1FAC910895E32FA0913A08EA0F5D
:10BB0200EA930895EE27A30FBE1FEC910895E093E8
:10BB1200A505F093A6050895A981BA81DCCC2A97E0
:10BB2200FE01FA93EA930895E6E8F8E0FA93EA93BD
:10BB3200AE85BF8588899989E4E6F0E060E070E02F
:10BB42000E94E8610E945462AA89BB898C899D89FE
:10BB5200E4E6F0E060E070E00E9402620E9454625B
:10BB620088E00E943F542C96FE01FA93EA930895CE
:10BB7200EFE8F8E0FA93EA93EE85FF859ACAFE01B0
:10BB8200FA93EA930C94C332F801AA81BB81EA0FBB
:10BB9200FB1FE4910895D801F0E0AE17BF070895A6
:10BBA200E1E3EA930C948E4EE3E2EA930C94174D90
:10BBB2000E94A14E0C94403FFA93EA93E0E0EA938C
:10BBC2000895EA930E94B8331F5F0895E12FAB8175
:10BBD200BC81F0E0EA0FFB1FE4910895AFEAB5E003
:10BBE20049CCAF5FEAE00E94ED610895E981ACE0E3
:10BBF200EA9FF0010895ABE00A9FF001EE50FC4F7E
:10BC0200DF010895EA0FFB1F0F01AC81BD817ACFDE
:10BC1200A5E10A9FF001E253FB4FDF010895EE8197
:10BC2200FF8101801280AE81BF811596EC9111C90E
:10BC3200FE013896FA93EA930895A5E10A9FF0016E
:10BC4200E253FB4FE081E0300895FA93EA93FE015C
:10BC52003A96FA93EA930E94095230E0E02F08954F
:10BC6200ABE00A9FF001EE50FC4FE081E030089516
:10BC7200E091A505F091A6050895A5EAB5E0ED913C
:10BC8200FD913296FE93EE930895AE81BF81EA173D
:10BC9200FB070895EC91F0E0E00DF11D0895E093AB
:10BCA2004B05F0934C050895E0E0F0E0E093490580
:10BCB200F0934A050895E5BBE881EBBB85E08A95E0
:10BCC200F1F71F9A85E08A95F1F71F980895EA9394
:10BCD2000E946637EAE0F0E00C946856E0E2EA93EC
:10BCE2000C945637EA930E949738E0300895E09119
:10BCF2007100E87F1E2F0895E0937300E4E8F2CF0D
:10BD02000A930E947038E0300895EE81FF813196E7
:10BD1200EE83FF830895FF27662777270E94F2624A
:10BD22000895EE8DAE85BF8588899989F4DF0E94DA
:10BD32007A63A9A1BAA1882799270E945B620E940F
:10BD42005E620E94256308950E945E620E942563DE
:10BD520008951A930A93E0915B0AE0300895E55A38
:10BD6200F54FE081E0300895E55AF54F5BCEE55A94
:10BD7200F54FE0810E0F1F5F0895E0912D08A9E0B5
:10BD8200EA9FF0010895E3E0F0E0FA93EA930E945B
:10BD9200804DF3CFE2E0F0E0FA93EA9308950E9437
:10BDA2003762F096EA930E948E4EE2E7EA930C9491
:10BDB200174DE081EA930C94174DE2EAF8E00C94F7
:10BDC20093565A934A930E942B160E2F00340895CD
:10BDD200E2E5EA930C94174D1A93E0915408E0536C
:10BDE2001E2FE8E5F8E07CC9E0912E08A0912F080B
:10BDF200EA170895E0912F08EA930E94842FE093B6
:10BE02002F080895A091960BECCEE093960BEAE2F0
:10BE1200EA930E948E4EDCCFE091960BE05AEA93B1
:10BE22000E94174D87C9D9011496EC910C94F254D3
:10BE3200F901A281B381BA93AA9308950E94464D53
:10BE42000C947857D9011196E0E0EC930E94A14E30
:10BE5200D1CFE091980B0C942D570E94A14EE3E0B4
:10BE6200E0935108E091330DEF5FE093330D0E94B0
:10BE7200403FE093310DF093320DD9011196EC91D0
:10BE8200D90129CCD9011196E2E0EC930895EA9305
:10BE92000E948E4E9DCFE093310DF093320DE2E081
:10BEA200E0935108EFCF0E9429340C9403340E948E
:10BEB20020340C9403340E942934EBEEF8E07CCE5B
:10BEC20040E050E0E02FE05DEA93EEEEF8E01ECABB
:10BED20010913F05009141050895FA93EA93E02FEE
:10BEE2000C94F2540E94C7370E94B5343E2F089535
:10BEF20026DD3197F2CF0E948837E2E0EA930C9474
:10BF0200C637EAE0F0E00E9493610895F0E0EA0F9C
:10BF1200FB1F08950E941D640C940838EA930E9446
:10BF2200EF40E1320895FA93EA93E2E0EA930E9445
:10BF32003941E1320895EA0FFB1FFA93EA93E0E1F7
:10BF4200EDCF0E948837E12FEF5FEA930E9416330C
:10BF5200EAE3EA930C9456370E941633BFCEEA23E3
:10BF6200EA930E941B33BACEE12FEF5FEA930E945D
:10BF72001633EAE3EA930C945637EA930E941B3392
:10BF8200ADCEDF013E960E945062FA93EA93FD0124
:10BF92007296E491C3CFA6E10A9FF001E854FF4FE5
:10BFA20008953E960E945062FA93EA930895E6EF4E
:10BFB200F4E0E0935A0CF0935B0C08950E941E1873
:10BFC200E0E0E0933D080E94B1050E949D05E1E09A
:10BFD200E093370808950E9408380E949E050E9447
:10BFE200B5340E2F0D330895EE81FF81FA93EA9353
:10BFF2000895EAE2EA93E3E9F9E0FA93EA93E09139
:10C002003A087BCCE0913A08EA930E94FB050C9433
:10C012009D05AA81BB81EC91E295E07FAE2FEC8178
:10C022000895EA0FAA81BB81EC93A881B981EC91B2
:10C03200EF5FEC930895E091D70DA091D60DEA172A
:10C042000895E091D70DF0E0EE58F24FE081ECB99F
:10C05200A091D70DAF5FA093D70DA4360895E093BA
:10C062005509E0E0E0935609E09358090895E091FC
:10C072005609F0E0E55AF64F08951083E09156090B
:10C08200EF5FE0935609E12FA09158090895EA0F56
:10C09200E0935809E0915709E150E0935709E030E5
:10C0A2000895E55AF64FA0E0A0830895E091A20E0C
:10C0B200F091A30E0895A091A00EB091A10EEA17DF
:10C0C200FB070895E12FA091A70EEA0FE093A70EB8
:10C0D200E091A90E0895F0E0ED5AF74F108308950C
:10C0E200E091AE0FF0E0E355F14FE081E0939C0068
:10C0F200E091AE0FEF5FE093AE0F08950E941D64D2
:10C1020000E010E00895E12FA981BA81FFCEEA9301
:10C112000E94174D1F5F0895E15AF44FE081E0300D
:10C122000895AD81BE81EC91F0E0ED5AF74F108198
:10C132000895AC81BD81EC91F0E0ED5AF74F30816A
:10C142000895AB81BC81EC91F0E0ED5AF74FE081AC
:10C152000895E881EA930C94174DA0917A0BB0915F
:10C162007B0B0895E881F9816A817B810E94546288
:10C172000895EA930E942F3FEA930C94C348EA93EE
:10C182000E94C348E0E0EA930C94C3480E94403FF7
:10C19200E0933A0DF0933B0D0895E0913A0DF09142
:10C1A2003B0DFA93EA933CCB2A93ED89FE89FA93ED
:10C1B200EA93FE017596FA93EA930C945752EE892C
:10C1C200FF893497EE8BFF8B0895ED89FE89FA93F0
:10C1D200EA93FE017596FA93EA930C945752AE894C
:10C1E200BF8914960E943762EE83FF83FDCEE887F3
:10C1F200F9876A877B870895E885F9856A857B8553
:10C20200AC85BD858E859F8508950E946854E8831C
:10C21200F9836A837B830895E881F9816A817B814E
:10C222000895EA81FB816C817D810895E991F991FC
:10C23200309639F080EA9FE00197F1F7A89531979F
:10C24200C9F708950024AF0DB01D0895EA0FFB1F32
:10C25200681F791F0895F195E195F0400895F095D2
:10C2620060957095E195FF4F6F4F7F4F0895EE23D4
:10C272000E2EFD0121F0EE0FFF1F0A94E1F7089543
:10C28200EE0FFF1FEE0FFF1FEE0FFF1FEE0FFF1F40
:10C292000895EF2FFF27E7FDFFEF0895FE2FFF0F11
:10C2A200FF0B6F2F7F2F08956F2F660F660B762F70
:10C2B2000895BA2FBB0FBB0B8B2F9B2F08958B2F8B
:10C2C200880F880B982F0895EA17FB07E1E00CF01E
:10C2D200EE270895FA9FF02DEB9FF00DEA9FE02DD7
:10C2E200F10D08957A9F702D6B9F700DF89F700D60
:10C2F200E99F700D6A9F602D710DFB9F600D711D8E
:10C30200E89F600D711D8827FA9FF02D610D781F3F
:10C31200EB9FF00D611D781FEA9FE02DF10D681F64
:10C32200781F089582D0D6DF0EF495DF08958BD062
:10C33200D9DF0EF494DF0895002498E0AA0F001CC0
:10C342000E1A10F40E0E01C0A1609A95B9F7EA2FE9
:10C35200A02D08950024112490E1AA0FBB1F001CF8
:10C36200111C0E1A1F0A18F40E0E1F1E01C0A16026
:10C372009A9599F7FD01D001089557D0EBDF0EF49D
:10C382006ADF08953F934F935F930024112444275B
:10C39200552730E2AA0FBB1F881F991F001C111CD2
:10C3A200441F551F0E1A1F0A460B570B28F40E0E78
:10C3B2001F1E461F571F01C0A1603A9559F7FD0184
:10C3C200BC01D001CA015F914F913F9108953BD0CA
:10C3D200D9DF0EF444DF0895AFDFEA2F0895E89421
:10C3E200B7FF04C0A095B09511966894F7FD33DFAE
:10C3F200B1DFFD010EF42FDF0895C4DFFD01BC01A2
:10C402000895E89497FF09C0A095B09580959095FE
:10C41200AF5FBF4F8F4F9F4F689477FD20DFB2DF32
:10C42200FD01BC010EF41BDF0895E894F7FF02C082
:10C4320012DF6894B7FF06C0A095B095119600F878
:10C44200039400FA0895E89477FF02C008DF689425
:10C4520097FF0BC00024A095B095809590951196FA
:10C46200801D901D00F8039400FA0895ED91FC914F
:10C4720011970895ED91FD916D917C911397089517
:10C48200ED91FD916D917D910895ED93FD936D93E5
:10C492007C9308957E936E93FE93EE930895059098
:10C4A200F491E02D08957A936A93FA93EA930895AA
:10C4B200689401C0E89401D095D0182E862F612D82
:10C4C200192E972F712D1B2EBF2FF12D1A2EAE2F45
:10C4D200E12D0895119602D0FE2F1197E199FECF1A
:10C4E200FF93FFB7F894AEBBBFBBE09AEDB3FFBFBB
:10C4F200FF910895E19B02C0A895FCCF9FB7F894E5
:10C50200AEBBBFBBE09A8DB3E81719F0EDBBE29A60
:10C51200E19A9FBF0895552342F4503811F4E0FF89
:10C5220004C03196691F791F6BF050E8572711F448
:10C532005F93CDC05F3F31F0660F000C5795679552
:10C54200752F08955F9300200AF0CDC0C6C050E851
:10C55200192E1522880F991F9527550F879550E898
:10C56200072E0522660F771F7527550F67950895C9
:10C57200689401C0E8945F93F2DF703818F07F3F4F
:10C5820008F4A5C056E1571BAAF4519558300EF491
:10C59200593030F0EFEFFFEF6FEF7FE777F91AC016
:10C5A20077275523B9F0EE0FFF1F661F771F5A95A5
:10C5B200D1F710C07727583028F0EF2FF62F672FCA
:10C5C2005850F9CF552331F076956795F795E79551
:10C5D2005A95D1F700200AF442DE5F9108956894DB
:10C5E20001C0E894309760407040B1F0002426F01A
:10C5F200772312F4009433DE172E7EE1112032F0FD
:10C602007A95EE0FFF1F661F111CF9CFEF2FF62F41
:10C61200612D5F938ADF5F9108954F93AF01FD0112
:10C62200DA01AB01BC01CA01402D012C142E4F913D
:10C632000895EA0FFB1F681F0895E095F095609535
:10C64200EF5FFF4F6F4F08955F9381DF903871F175
:10C6520050E8152604C05F937ADF903839F17038BC
:10C6620021F1572F591B13F112F4D7DFFACF5831AA
:10C6720018F0AA27BB278827583028F0AB2FB82FED
:10C6820088275850F9CF552329F08695B795A79555
:10C692005A95D9F7502D512562F0CBDF38F46795C2
:10C6A200F795E795739513F41EC0B7DF3EDF5F91F0
:10C6B2000895EA1BFB0B680B51F010F40094BDDFE8
:10C6C2006623A2F3EE0FFF1F661F7A95CBF7EE27C4
:10C6D200FF27662777275F910895EFEFFFEF6FE758
:10C6E2007FEF5F910895EFEFFFEF6FE77FE75F91D5
:10C6F20008955F932CDF703851F3903841F3012491
:10C702000894791F23F41CF300203AF3ECCF0F9224
:10C712001F932F933F934F93112722279927689FA7
:10C72200A0018F9F302D410D591F6B9F300D411D70
:10C73200591F8E9F27D0BF9F25D06A9F23D0BE9FAF
:10C742001DD0AF9F1BD0AE9F110D291F391F491F4E
:10C75200591FE32FF42F652F522F4F913F912F91A5
:10C762001F910F9066232AF0550FEE1FFF1F661FC1
:10C7720002C073954BF2CFDE5F910895100D211D1B
:10C78200391F02C0200D311D491F591F08955F93A3
:10C79200DEDE703821F411200AF49FCFA4CF903846
:10C7A20009F495CF01240894970B1BF4D4F30020CD
:10C7B200F3CF792F1F932F933F934F931124112778
:10C7C200222733274427552790E2AE17BF07860753
:10C7D200410730F0AE1BBF0B860B410B089401C022
:10C7E2008894551F221F331F111CAA1FBB1F881FAD
:10C7F200441F9A9551F7F901612D4F913F912F9165
:10C802001F91662332F0550FEE1FFF1F661F7A95A8
:10C8120043F281DE5F910895309760407040089541
:10C8220000240A160B06089500240A160B060806B1
:10C83200090608955A934A933A932A931A930A93AC
:10C8420008955D814C813B812A8119810881089577
:00000001FF
